:100000000C94A60A0C94C70A0C94C70A0C941E10F0
:100010000C9458100C94C70A0C94C70A0C94C70A85
:100020000C94C70A0C94C70A0C94C70A0C94C70A0C
:100030000C94C70A0C94C70A0C94C70A0C94731347
:100040000C94C70A0C94C70A0C94C70A0C94C70AEC
:100050000C94C70A0C9457680C94C70A0C94C70AEE
:100060000C94C70A0C94D2680C94C70A0C94C70A63
:100070000C94C70A0C94C70A0C94C70A0C94C70ABC
:100080000C9481810C94C70A0C94C70A0C94C70A7B
:100090000C9401690C94C70A0C94C70A0C94C70A03
:1000A0000C94C70A0C94C70A0C94C70A0C94C70A8C
:1000B0000C94C70A0C94C70A0C94C70A0C94C70A7C
:1000C0000C94C70A0C94C70A0C94C70A0C94C70A6C
:1000D0000C94C70A0C94C70A0C94C70A0C94C70A5C
:1000E0000C94C70A0C94926F0C949C6F0C94886FBC
:1000F0000C94486F0C94C86F0C94BE6F0C94B26F44
:100100000C94A66F0C94C70A0C94C70A0C94C70AE7
:100110000C94C70A0C94C70A0C94C70A0C94C70A1B
:100120000C94C70A0C94C70A0C94C70A0C94C70A0B
:100130000C94C70AAF87CE8747883989598979894E
:1001400081892E89084AD73B3BCE016E84BCBFFD16
:10015000C12F3D6C74319ABD56833DDA3D00C77F97
:1001600011BED9E4BB4C3E916BAAAABE0000008030
:100170003F07634236B79BD8A71A39685618AEBAFC
:10018000AB558C1D3CB7CC5763BD6DEDFD753EF690
:10019000177231BF000000803F08000000BE9224AB
:1001A00049123EABAAAA2ABECDCCCC4C3E000000E0
:1001B00080BEABAAAAAA3E00000000BF00000080DB
:1001C0003F0000000000084178D3BB4387D1133DB6
:1001D000190E3CC3BD4282AD2B3E68EC8276BED97F
:1001E0008FE1A93E4C80EFFFBE01C4FF7F3F0000BE
:1001F000000000000C9459770C94445E0C94EA6C57
:100200000C94337C0C94448B0C94A56D0C94087B5B
:100210000C942E890C94CF6E0C9423110C940B7BB0
:100220000C945E770C94AA6A0C9417760C947D6BF0
:100230000C940D770C9432160C94DD380C94AC0EA3
:100240000C9481890C94AF1D0C9405710C94920E42
:100250000C9462690C9423760C941D4E0C9479894D
:100260000C94BA690C94526D0C943F150C94E66989
:100270000C94746B0C94A77B0C94037B0C94BA8A3B
:100280000C9461770C94B1760C9454770C944F775E
:100290000C94244F0C9494910C9459890C94018BD8
:1002A0000C94928E0C94E36F0C94B56A0C9439897B
:1002B0000C94958A0C942F6C0C9447880C9420799C
:1002C0000C94C18F0C94AF870C946A8A0C94F18DB6
:1002D0000C94C64E0C94DA760C94CE870C944A7724
:1002E0000C94C27B0C942A7C6E616E00696E660071
:1002F000256300496E76616C6964206932632073FE
:100300007065656420696E20454550524F4D2E2022
:1003100053657474696E67203130206B6269742F85
:10032000730025730A00776474206E6F7420656E05
:1003300061626C65640A005854414C5F5452494DE7
:100340003D25640025730A0025730A005465737403
:1003500020362025730A00546573742035202573D8
:100360000A005465737420342025730A00546573A1
:100370007420332025730A005465737420322025BD
:10038000730A005465737420312025730A00636872
:10039000616E3D25640A0074787077723D25640AA9
:1003A000003530306B0A003235306B0A00313135A0
:1003B0006B0A0035366B0A0033386B0A0025730A66
:1003C00000765F6C6F773D252D332E32660A00254F
:1003D000730A0073656E743D252D75206475703D3C
:1003E000252D752069676E6F7265643D252D75201A
:1003F00074746C5F7A65726F3D252D750A00253720
:100400002E33662025372E33660025352E326620A2
:10041000004572726F72203020566F6C74004E6F00
:100420007420737570706F727465640A004572721F
:100430006F72203020566F6C74004572726F72209C
:100440003020566F6C740062756C6B5F64656C6114
:10045000793D252D750062756C6B3D252D75005617
:10046000616C7565206E6F7420616C6C6F7765646C
:100470000062756C6B3A206D61783D257520737450
:100480006172743D25752C20656E643D25752C20A8
:10049000696E5F7573653D25750A007062323D2592
:1004A000730A007062313D25730A00256C750041A6
:1004B0006C6C6F77656420737065656420312F31D3
:1004C000302F3130302F343030206B6269742F730D
:1004D0000025630074746C3D252D64200074746CD9
:1004E0003D252D6420004E65772074746C3D252DCC
:1004F0006420002563004D533536313120503D25B1
:100500002D372E326620252D372E32666D0A004299
:100510004D5030383520256C6420432000424D502A
:1005200030383520256C642050612020252D372E51
:1005300032666D00256300545F484541545F49446D
:10054000583D252D352E32662000545F4445573DD9
:10055000252D352E3266200041483D252D352E3281
:10056000662000545F53485432583D252D352E32B5
:1005700066200052485F53485432583D252D352E91
:1005800032662000545F52483D252D342E316620BE
:100590000052483D252D342E31662000256300256C
:1005A00063002563002563002563007265706F7228
:1005B000745F616C6C3D007265706F72743D0025F4
:1005C0006300256300256300256300204F534343E8
:1005D000414C3D2564200020467573653A206565D1
:1005E0003D253032782068663D25303278206C66B3
:1005F0003D25303278206C623D25303278004D4305
:10060000553D2530366C780025630074785F6C6545
:100610006E3D252D6C752C765F6C6F773D252D6CAE
:10062000752C73687432783D252D6C752C62756C51
:100630006B3D252D6C75002563004F4B0A0025632B
:100640000025630025630025630025630025630002
:1006500025630025630064656275675F616C6C3DAE
:100660000064656275673D0064656275673D0025DD
:10067000730A00646565700A006E6F6E650A00702B
:100680007772733D007764743D25730A007062329F
:100690003D25730A007062313D25730A00696E744E
:1006A000725F7365635F70313D252D372E33660AA7
:1006B00000696E74725F70313D252D6C640A0069AB
:1006C0006E74725F7365635F70303D252D372E3316
:1006D000660A00696E74725F70303D252D6C640A85
:1006E00000765F6D63753D252D352E32660A0074E8
:1006F0005F6D63753D252D352E32660A007070776B
:10070000723D25730A0064656275673D0072636D12
:10071000643D25730A0025730A006175746F0A0031
:100720006C6F675F6D6F64653D007573625F7077B6
:10073000723D25730A0072656C61793D25730A006C
:1007400074746C3D252D640A0052494D455F616407
:1007500064723D252D642E252D640A006E6569673F
:1007600068626F725F7461626C655F73697A653D20
:1007700025640A00765F6C6F773D252D332E326637
:100780000A00747870773D25640A006368616E3DE5
:1007900025640A0069643D006932635F6275733DD8
:1007A000006932635F73706565643D252D6C750A61
:1007B000007478743D25730A0053797374656D2055
:1007C00053756D6D6172790A002530366C78004181
:1007D000744D656761323536524652320041744D70
:1007E000656761313238524652320041744D656757
:1007F000613634524652320041744D656761313280
:100800003852464131004D43553D006D61736B3D9B
:10081000002C00696E74657276616C3D252D750043
:1008200023252D642C00705F626D653238300072B4
:10083000685F626D6532383000745F626D653238B2
:1008400030007062320070623100745F68656174FC
:100850005F69647800745F64657700616800705F49
:100860006D73353631310072685F736874327800A9
:10087000745F736874327800706100700061643472
:1008800000616433006164320061643100613300EF
:10089000613200613100765F696E007268006572D6
:1008A0007200757074696D650070315F6C737400EF
:1008B00070315F740070310070305F6C7374007061
:1008C000305F7400703000765F6D637500745F6D2B
:1008D0006375007431007400696400653634007417
:1008E0007874002D002B006175746F006E6F6E655B
:1008F0000062756C6B00706F7765725F736176650F
:100900005F6C656472790072656C61795F6C6564B7
:100910007900636F6D7061737300616363656C0070
:100920007072657300705F7077720061657300703C
:10093000315F6C6564790070305F6C65647200656E
:1009400076656E74006C6564006F7700706B740080
:1009500074785F6C6564790072785F6C65647200AE
:100960006F706572006E6F6E6500253032780076AC
:100970005F6164343D252D382E3666002000765F99
:100980006164333D252D382E3666002000765F6188
:1009900064323D252D382E3666002000765F616476
:1009A000313D252D382E3666002000765F6C696754
:1009B00068743D252D382E3666002000765F613242
:1009C0003D252D372E3366002000765F61313D25B1
:1009D0002D372E3366002000765F696E3D252D355C
:1009E0002E326600204E657665722D757365642023
:1009F000737461636B203E20256420627974657393
:100A00000A00757074696D653D252D642D646179EA
:100A1000732D253032643A253032643A2530326401
:100A20002D686F7572730A0074657374205B6F664E
:100A3000667C317C327C337C347C355D2020202008
:100A4000202020202D2074657374206D6F646573E1
:100A50000A0D007478205B706B74207061796C6F84
:100A600061645D2020202020202020202020202DB7
:100A70002073656E6420726164696F20706B7420EE
:100A80006B6579626F6172640A0D00776474205B34
:100A90006F6E7C6F66667C746573745D20202020A9
:100AA000202020202020202D207761746368646F2F
:100AB000670A0D00765F6C6F77205B765F6C6F77EF
:100AC0005D202020202020202020202020202020E9
:100AD0002D206C6F77657374207265706F7274204F
:100AE000766F6C746167650A0D00757067722020FF
:100AF00020202020202020202020202020202020F6
:100B00002020202020202D207265626F6F742076B7
:100B1000696120626F6F746C6F616465720A0D00A9
:100B200075617274205B33386B7C35366B7C313188
:100B3000356B7C3235306B7C3530306B5D202D2051
:100B4000736574207465726D2F7561727420737093
:100B50006565640A0D00626F6F74202020202020DC
:100B60002020202020202020202020202020202085
:100B700020202D207265626F6F740A0D00707772ED
:100B800073205B646565707C6E6F6E655D202020F0
:100B90002020202020202020202D206D6375207310
:100BA0006C656570206D6F64650A0D007265737405
:100BB00020656570726F6D2020202020202020206D
:100BC00020202020202020202D20726573746F7239
:100BD0006520656570726F6D0A0D00707077722008
:100BE0005B6F6E7C6F66665D2020202020202020B9
:100BF000202020202020202D2070726F6772616DD0
:100C00006D61626C65207077720A0D00706232202F
:100C1000205B6F6E7C6F66665D2020202020202088
:100C200020202020202020202D2070726F677261EC
:100C30006D6D61626C652070696E2062320A0D0014
:100C400070623120205B6F6E7C6F66665D202020B5
:100C50002020202020202020202020202D206275F0
:100C60006C6B204750494F2070696E0A0D007478F4
:100C700074205B737472696E675D202020202020D1
:100C8000202020202020202020202D20536574208B
:100C90007265706F727420746578742073747269F1
:100CA0006E670A0D0074787077205B31352D305DEA
:100CB0002020202020202020202020202020202034
:100CC000202D205458205077722E2048696768657F
:100CD0007374203020283364426D290A0D00747427
:100CE0006C205B302D31355D2020202020202020FD
:100CF000202020202020202020202D2074696D65B8
:100D00002D746F2D6C69766520666F72207061633B
:100D10006B6574730A0D007373202020202020203F
:100D200020202020202020202020202020202020C3
:100D30002020202D2073797374656D2073756D6D7F
:100D40006172790A0D00727320202020202020205B
:100D50002020202020202020202020202020202093
:100D600020202D20726164696F2073746174730A8E
:100D70000D007269205B236E5D205B696E745D20DF
:100D800020202020202020202020202020202D2056
:100D90007265706F727420696E74657276616C0A28
:100DA0000D0072636D64205B6F6E7C6F66665D2004
:100DB00020202020202020202020202020202D2026
:100DC000616C6C6F7720636D642066726F6D206E4E
:100DD00065746F726B0A0D007265205B236E5D2077
:100DE0005B2B7C2D5D205B6D61736B7C6175746F1B
:100DF0002C6D61736B5D202D206D6F7465207265A5
:100E0000706F7274207365742F6D6F646966790AF0
:100E10000D006F772020202020202020202020205F
:100E200020202020202020202020202020202D20B5
:100E30006F6E652D776972652073656E736F72735F
:100E40000A0D006C6F67205B6175746F7C6F6E7C40
:100E50006F66665D20202020202020202020202D6D
:100E6000206D6F7465732064617461206F6E20550E
:100E700053420A0D006E65205B666C7573685D20D9
:100E80002020202020202020202020202020202062
:100E9000202D206E65696768626F72207461626CD4
:100EA000650A0D006572722020202020202020205D
:100EB0002020202020202020202020202020202032
:100EC0002D206572726F722073746174730A0D0045
:100ED0006D6375202020202020202020202020202D
:100EE0002020202020202020202020202D206D6365
:100EF0007520696E666F0A0D00693263205B70723F
:100F00006F62657C737065656420236E5D202020B0
:100F100020202020202D206932632070726F6265AE
:100F2000206275737C7365742062757320737065BD
:100F300065640A0D006964205B72657365745D20E9
:100F400020202020202020202020202020202020A1
:100F5000202D2069642068616E646C696E670A0DDB
:100F60000068756D202020202020202020202020B7
:100F7000202020202020202020202020202D20681C
:100F8000756D69646974792073656E736F720A0D8B
:100F90000072656C6179205B6F6E7C6F66667C7336
:100FA000746174735D20202020202020202D207269
:100FB000656C6179206E6574776F726B20726570F5
:100FC0006F7274730A0D006465205B6D61736B5DF5
:100FD0002020202020202020202020202020202011
:100FE0002020202D2064656275670A0D006368610A
:100FF0006E205B31312D32365D20202020202020D4
:101000002020202020202020202D206368616E20B9
:1010100031312D32362028322E3430352D323438CD
:1010200030204D687A290A0D0063616C69205B5B92
:10103000765F696E7C61317C61325D20766F6C74A5
:101040007C72657365747C6E6F6E655D202D2063A8
:10105000616C6962726174650A0D0062756C6B2067
:101060005B5B73686F777C666C7573685D205B7320
:1010700065742074687273682064656C61795D5D65
:1010800020202D2062756C6B696E67207061636B28
:10109000657473200A0D00616463202020202020E5
:1010A0002020202020202020202020202020202040
:1010B0002020202D2073686F7720765F696E2C20AA
:1010C00061312C20613220766F6C74616765730A20
:1010D0000D007520202020202020202020202020EE
:1010E00020202020202020202020202020202D20F3
:1010F000757074696D650A0D00762020202020200F
:1011000020202020202020202020202020202020DF
:1011100020202020202D2076657273696F6E0A0DC5
:101120000068202020202020202020202020202097
:10113000202020202020202020202020202D20685A
:10114000656C700A0D00256300756E6B6E6F776EAF
:1011500020636D640A00484D4335383833002573E9
:1011600000257300202573002025362E32662000CE
:10117000253032780074656D705F65787465726EC5
:101180003D252D362E326600202573002025362E73
:101190003266204F6E2D426F6172640025303278C6
:1011A0000074656D705F626F6172643D252D362E2F
:1011B0003266000A0042756C6B2072656D3A2073CE
:1011C000746172743D25752C20656E643D25752C07
:1011D00020696E5F7573653D25750A0042756C6BFD
:1011E000206164643A2073746172743D25752C200B
:1011F000656E643D25752C20696E5F7573653D25B0
:10120000750A0042756C6B207468726573683A20C9
:1012100074696D65723D25750A00503A20256C642D
:101220002050612020252D372E3266206D0A00497E
:1012300032433A20004A5441472072657365747402
:10124000210A005761746368646F67207265736573
:1012500074210A0042726F776E6F75742072657325
:101260006574210A0045787465726E616C20726540
:10127000736574210A00506F7765722D6F6E20724E
:1012800065736574212E0A004F6E6C696E650A00E5
:10129000526F7574696E6720456E61626C65640A91
:1012A0000052504C20456E61626C65640A002573E3
:1012B0002025732C206368616E6E656C2025752077
:1012C0002C20636865636B2072617465202575202E
:1012D000487A20747820706F7765722025750A002F
:1012E0000A2A2A2A2A2A2A2A426F6F74696E6720DC
:1012F00025732A2A2A2A2A2A2A0A004A54414720E0
:101300007265736574210A005761746368646F675E
:10131000207265736574210A0042726F776E6F7573
:1013200074207265736574210A0045787465726E65
:10133000616C207265736574210A00506F77657265
:101340002D6F6E2072657365742E0A00726E6720B1
:101350006973737565732025640A00454550524FC3
:101360004D20697320636F72727570742C207265E2
:1013700077726974696E672077697468206465663E
:1013800061756C74732E0A006C6F63616C686F73A7
:10139000740041544D454741323536726672320011
:1013A000020000FFFE000001452025642E25642078
:1013B000636C6F636B20256C752063707520256CE2
:1013C00075206C706D20256C752069727120256CFC
:1013D0007520676C656420256C7520796C656420C8
:1013E000256C7520726C656420256C7520747820DE
:1013F000256C75206C697374656E20256C7520737F
:10140000656E736F727320256C75207365726961E8
:101410006C20256C750A0000407A10F35A00A07207
:101420004E18090010A5D4E80000E876481700001F
:10143000E40B54020000CA9A3B000000E1F50500ED
:101440000080969800000040420F000000A0860136
:10145000000000102700000000E803000000006406
:1014600000000000000A0000000000010000000071
:10147000002C76D888DC674F0823DFC1DFAE59E146
:10148000B1B796E5E3E453C63AE651997696E8E6B5
:10149000C28426EB898C9B62ED407C6FFCEFBC9C88
:1014A0009F40F2BAA56FA5F490055A2AF75C936B9A
:1014B0006CF9676DC11BFCE0E40D47FEF520E6B555
:1014C00000D0ED902E0300943577050080841E082F
:1014D0000000204E0A000000C80C333333330F984D
:1014E0006E12831141EF8D2114893BE65516CFFE14
:1014F000E6DB18D1844B381BF77C1D901DA4BBE4A0
:1015000024203284725E228100C9F124ECA1E53DE1
:10151000274E414E494E495459494E46CDCCCC3DBB
:101520000AD7233C17B7D13877CC2B329595E624D0
:101530001FB14F0A000020410000C84200401C4675
:1015400020BCBE4CCA1B0E5AAEC59D7411241FBED2
:10155000CFEFD1E8DEBFCDBF00E00CBF1AE0A0E0C6
:10156000B2E0E6E8FDE301E00BBF02C007900D9298
:10157000A43DB107D9F72AE3A4EDBAE001C01D925A
:10158000AD3BB207E1F70E9431670C94C19E0C9409
:1015900000002F923F924F925F926F927F928F92B4
:1015A0009F92AF92BF92CF92DF92EF92FF920F93F2
:1015B0001F93CF93DF93CDB7DEB763970FB6F89441
:1015C000DEBF0FBECDBF6C014B012A01FC011782AB
:1015D0001682838181FF43C3AE014F5F5F4F3A01A3
:1015E000F6019381F40193FD859193FF81914F0161
:1015F000882309F430C3853239F493FD859193FF34
:1016000081914F01853239F4B60190E00E948D9BA3
:1016100052012501E5CF10E0F12C20E02032A0F4AA
:101620008B3269F030F4803259F0833269F42061F2
:101630002CC08D3239F0803339F4216026C022600D
:10164000246023C0286021C027FD27C030ED380F5B
:101650003A3078F426FF06C0FAE01F9F300D1124BF
:10166000132F13C04AE0F49E300D1124F32E206294
:101670000CC08E3221F426FDEEC2206406C08C36EA
:1016800011F4206802C0883641F4F40193FD85917D
:1016900093FF81914F018111C1CF9BEB980F933044
:1016A00018F42061805E06C09BE9980F933008F023
:1016B00071C12F7E26FF16E02F73322E853619F466
:1016C0002064322E08C0863621F4F22FF0683F2EB7
:1016D00002C01111115037FE07C01C3350F4EE2424
:1016E000E394E10E27E00BC0183038F027E017E054
:1016F00005C027E04CE3E42E02C0212FE12C52016B
:1017000044E0A40EB11CF201608171818281938159
:101710000E2DA3010E94049A2C01098100FF02C032
:1017200003FF07C031FC08C032FE09C030E2232E9F
:1017300007C02DE2222E04C09BE2292E01C0212CDD
:10174000802F8C7019F0211068C2A8C237FE0FC01C
:10175000E40C04FF04C08A81813309F4EA941E1466
:1017600074F5F8E0FE1578F588E0E82E2CC036FC1C
:101770002AC0812F90E0841595059CF02CEF42162D
:101780002FEF520674F0432D4068342E0AC0E2E079
:10179000F0E0EC0FFD1FE10FF11D8081803319F4A3
:1017A00011501111F4CF37FE0EC0EE24E394E10E78
:1017B000812F90E0481659062CF4141904C0EE2429
:1017C000E39401C010E037FE06C01414150434F48D
:1017D000C201019605C085E090E002C081E090E082
:1017E00021100196112331F0212F30E02F5F3F4F60
:1017F000820F931F2F2D30E08217930714F4F81AED
:1018000001C0F12C832D897049F4FF2039F0B60115
:1018100080E290E00E948D9BFA94F7CF222029F07D
:10182000B601822D90E00E948D9B33FC09C0FF2001
:1018300039F0B60180E390E00E948D9BFA94F7CFD7
:1018400037FE5AC0942D852D57FE02C090E080E0EF
:10185000292E382E20E030E0A2014E1951095D8773
:101860004C87A201421953095F874E87612F70E0B0
:1018700044275527461B570B598B488B5FEF25167E
:10188000350649F4B6018EE290E02A8B3B8B0E942C
:101890008D9B3B892A89421453046CF04C855D85ED
:1018A0004215530544F4EE85FF85E20FF31FE60D64
:1018B000F71D818101C080E351E0251A31082F5FB7
:1018C0003F4F48895989241635064CF0B60190E0FF
:1018D0002A8B3B8B0E948D9B2A893B89CFCF241476
:1018E000350439F49A81963318F4953311F404FFD2
:1018F00081E3B60190E04BC08A81813309F00F7E0D
:10190000B60190E00E948D9B111105C034FC18C0F7
:1019100085E690E017C0B6018EE290E00E948D9BB4
:1019200082E0EE24E394E80EF301E80FF11D8081DC
:10193000B60190E00E948D9B11508E2D91F7E6CF5D
:1019400085E490E0B6010E948D9B57FC05C04114D0
:10195000510439F404FF05C05194419451088DE2BB
:1019600001C08BE2B60190E00E948D9B80E39AE07B
:10197000491651042CF08F5F5AE0451A5108F7CFF1
:10198000B60190E00E948D9BB601C201C0960E94F4
:101990008D9B57C1833631F0833779F0833509F059
:1019A00058C021C05201E2E0AE0EB11CF2018081AC
:1019B000898301E010E0230114C05201F2E0AF0E70
:1019C000B11CF2014080518026FF03C0612F70E0FE
:1019D00002C06FEF7FEFC2012A8B0E94399B8C01FE
:1019E0002A892F7715C05201F2E0AF0EB11CF20127
:1019F0004080518026FF03C0612F70E002C06FEF6E
:101A00007FEFC2012A8B0E94EE9A8C012A892068FE
:101A1000322E23FD1AC08F2D90E008171907A8F465
:101A2000B60180E290E00E948D9BFA94F4CFF2011F
:101A300037FC859137FE81912F01B60190E00E941D
:101A40008D9BF110FA94015011090115110579F7D8
:101A5000F8C0843611F0893659F5520127FF09C0C4
:101A6000F4E0AF0EB11CF20160817181828193813B
:101A70000AC0F2E0AF0EB11CF20160817181072E45
:101A8000000C880B990B2F76322E97FF09C090958A
:101A90008095709561957F4F8F4F9F4F2068322EB4
:101AA0002AE030E0A3010E949E9CE82EE6183FC089
:101AB000022F853721F40F7E2AE030E01DC0097F18
:101AC0008F3691F018F4883559F0C5C0803719F079
:101AD000883711F0C0C0006104FF09C0046007C06E
:101AE00024FF08C0066006C028E030E005C020E101
:101AF00030E002C020E132E0520107FF09C0F4E00B
:101B0000AF0EB11CF201608171818281938108C0A6
:101B1000F2E0AF0EB11CF2016081718180E090E0D3
:101B2000A3010E949E9CE82EE6180F77302E36FE09
:101B30000BC0332D3E7FE11650F434FE0AC032FC58
:101B400008C0332D3E7E05C00E2D332D03C00E2D53
:101B500001C0012F34FF0CC0FE01EE0DF11D80818C
:101B6000803311F4397E08C032FF05C00E5F04C017
:101B7000832F867809F00F5F33FD13C030FF06C056
:101B80001E2D0F1518F41F0D101B0F2D0F1568F4C7
:101B9000B60180E290E03B8B0E948D9B0F5F3B89FA
:101BA000F5CF0F1510F4F01A01C0F12C34FF12C05C
:101BB000B60180E390E03B8B0E948D9B3B8932FF16
:101BC00017C031FD03C088E790E002C088E590E0CF
:101BD000B6010CC0832F867859F031FF02C08BE22A
:101BE00001C080E237FD8DE2B60190E00E948D9B3E
:101BF000E11638F4B60180E390E00E948D9B11500D
:101C0000F7CFEA94F301EE0DF11D8081B60190E06B
:101C10000E948D9BE110F5CF14C0F4E0FF1558F53C
:101C200084E0F81A33FE1EC0211026C003FF2AC02C
:101C300008EE12E0F32DF0713F2EF801849181112E
:101C400024C0FF2009F4E5CCB60180E290E00E94B8
:101C50008D9BFA94F6CFF6018681978126C08FEF8F
:101C60009FEF23C0B60180E290E00E948D9BFA9422
:101C7000F110F8CFD9CFF12CB601822D90E00E945F
:101C80008D9BD4CF0CEE12E0D5CF31108052B6012F
:101C900090E00E948D9B0F5F1F4FCFCF23E02F1549
:101CA00010F483E0BECFF12CC1CF63960FB6F89449
:101CB000DEBF0FBECDBFDF91CF911F910F91FF907F
:101CC000EF90DF90CF90BF90AF909F908F907F90DC
:101CD0006F905F904F903F902F90089581159105E0
:101CE00011F00197F1F708958FE796E09F938F9396
:101CF0000E94D99B8091660290916702A091680230
:101D0000B09169020F900F9093FF03C089E796E0AE
:101D100002C083E796E09F938F930E94D99B0F9018
:101D20000F900895E091AC1DEF73F0E0E350F24E98
:101D300080838091AC1D8F5F8093AC1D809159365C
:101D40008860809359364CE452E061E1CA010E94F8
:101D5000477380E090E00895CF93DF93EC0180918A
:101D60002D1490912E14A0912F14B091301486FF51
:101D70001DC08E811F928F938D811F928F938C81B6
:101D80001F928F938B811F928F938A811F928F93C3
:101D900089EE92E09F938F930E94C59B8DB79EB76B
:101DA0000C960FB6F8949EBF0FBE8DBFBE018FE19B
:101DB0009BE00E944074BE0188E092E0DF91CF91E9
:101DC0000C94D17452985A981DBAE9E6F0E08081DB
:101DD00080628083EA9A53985B98EB9A808180684E
:101DE0008083E8E6F0E08081816080830895E2E608
:101DF000FEE11182128210820895CF92DF92EF925B
:101E0000FF920F931F93CF93DF93EC019B0180917F
:101E1000621E843108F0BBC08091641E64E10E94A0
:101E200054909093641EC0907F31D0908031E090A8
:101E30008131F0908231092F10E08DE8989FD00118
:101E40001124AE59B14E1396CD92DD92ED92FC92D3
:101E500016974115510559F0FA018081FD01EA57A5
:101E6000FF4F8083FA018181A957BF4F8C93209740
:101E7000A9F089819DE8909FF001919FF00D1124B8
:101E8000EE59F14EDF01A657BF4F8C93E557FF4F38
:101E900088818F70808388818F70808321153105C0
:101EA000E1F1D90116964C9116975DE8509FC0015B
:101EB000519F900D11248E59914EFC01E757FF4F11
:101EC000408315964C9115973197408334961B9615
:101ED0004D915D916D917C911E97452F562F672FE7
:101EE0007727518340837C01BEE8EB0EF11CF9019A
:101EF0002385348545855685A4E6B0E00E94EF90A1
:101F0000672F782F892F992724E630E040E050E0B2
:101F10000E948890D7016D937C938DE8809FD001BB
:101F2000819FB00D1124A759B14EFE0132968FE763
:101F300001900D928A95E1F78091641E8F5F8093E6
:101F4000641E9091621E9F5F9093621E40912D14BB
:101F500050912E1460912F147091301460FF2DC099
:101F60001F929F931F928F938091631E1F928F9356
:101F70008CED91E19F938F930E94D99BEDB7FEB7B3
:101F800038960FB6F894FEBF0FBEEDBF16C0809115
:101F90008F3190919031A0919131B0919231019611
:101FA000A11DB11D80938F3190939031A0939131F9
:101FB000B093923180E090E002C081E090E0DF9148
:101FC000CF911F910F91FF90EF90DF90CF900895E8
:101FD0002091621E222361F18091631E8F5F215048
:101FE0002093621E64E10E9454909093631E40917E
:101FF0002D1450912E1460912F147091301460FFA5
:102000001AC01F922F938091641E1F928F931F926C
:102010009F9385EB91E19F938F930E94D99B8DB7FE
:102020009EB708960FB6F8949EBF0FBE8DBF03C033
:1020300080E090E0089581E090E008951F920F9273
:102040000FB60F9211248F939F93AF93BF938091FC
:10205000680080FF24C08091283690912936A09195
:102060002A36B0912B360196A11DB11D80932836DA
:1020700090932936A0932A36B0932B3680912D1455
:1020800090912E14A0912F14B091301487FF07C0A7
:10209000749882E090E09093920280939102BF91B5
:1020A000AF919F918F910F900FBE0F901F90189539
:1020B0001F920F920FB60F9211248F939F93AF939D
:1020C000BF938091680080FF24C080912C3690914E
:1020D0002D36A0912E36B0912F360196A11DB11D3F
:1020E00080932C3690932D36A0932E36B0932F36B6
:1020F00080912D1490912E14A0912F14B091301432
:1021000090FF07C0739882E090E0909392028093D2
:102110009102BF91AF919F918F910F900FBE0F9041
:102120001F90189580937C0080917B00877F80931F
:102130007B0080917C00806C80937C0085E08093A4
:102140007A0080917A00806880937A0080917B0089
:1021500087FFFCCF80917B0085FFFCCF80917A00C8
:10216000806480937A0080917A0086FDFCCF109283
:1021700079001092780084E090E060E070E02091B7
:102180007A00206420937A0020917A0026FDFCCF0B
:102190002091780030917900620F731F019779F7D1
:1021A00010927C0080917A008F7780937A007695E8
:1021B00067957695679580E090E00E945D9408951C
:1021C00080E00E9492102091890230918A02409111
:1021D0008B0250918C020E94579621EE3AE744E917
:1021E0005EE30E94C89208950F931F93CF93DF93ED
:1021F0000FE110E0CBE5DEE00093510182E991E0D0
:102200000E946E0E8091510185FD0DC000311105B7
:1022100021F02CF0CB54D10903C0C4ECD9E0E297F3
:1022200001501109E9CFBE0180E090E00E945D9469
:1022300020E030E04AE754E40E94AB93DF91CF9175
:102240001F910F910895CF93DF93EC0188819981BD
:10225000009799F08037924121F01982188283E02B
:1022600011C0623171F40E94F41060937B3170935D
:102270007C3180937D3190937E3180E792E1998328
:10228000888381E0DF91CF91089580917B00886001
:1022900080937B0089EC80937C0085E080937A00BA
:1022A00080917A00806880937A0080917B0087FF1C
:1022B000FCCF80917B0085FFFCCF80917A00806409
:1022C00080937A0080917A0086FDFCCF80917A001D
:1022D000806480937A0080917A0086FDFCCF6091C3
:1022E00078007091790080917A008F7780937A00DE
:1022F00080E090E00E945D9427ED33EA40E95FE3DF
:102300000E94579626E636E648E853E40E94C792B4
:102310000895CF92DF92EF92FF921F93CF93DF93B6
:10232000CDB7DEB729970FB6F894DEBF0FBECDBF8D
:102330006C01109227148FEF898785EBE82E8DE1D1
:10234000F82E10E089858823E9F11830D9F1BE0113
:102350006F5F7F4FCE0109960E94086299859F3F6B
:1023600011F09E3F19F4909327142CC0CE010196D2
:10237000C114D10481F40E94226280934A36A2E4FF
:10238000B6E3FE01319688E08E0F91919D938E13F6
:10239000FCCF81E018C00E942262F7018087FE0115
:1023A000319620E030E08191D701A20FB31F8C93CA
:1023B0002F5F3F4F28303105B1F71F5FF9E0EF0E77
:1023C000F11CC0CF812F29960FB6F894DEBF0FBE47
:1023D000CDBFDF91CF911F91FF90EF90DF90CF9015
:1023E000089583EB91E19F938F930E94D99B0F9067
:1023F0000F9008952F923F924F925F926F927F922B
:102400008F929F92AF92BF92CF92DF92EF92FF9204
:102410000F931F93CF93DF93EC015B01009711F4AF
:1024200027E003C0019749F426E04AE250E06BE25E
:1024300070E089E290E00E94E260CE010E94891182
:102440009E01285D3B4E6901D9018C93CD2B69F02B
:10245000C5EBDDE1E12CF12C88E6282E81E1382E58
:1024600094E6892E91E1992E9EC082E496E30E9423
:10247000B362BC01990F880B990B0E945F946B01AA
:102480007C01AB2869F020E030E048EC52E40E9487
:10249000AB939F938F937F936F9381EA91E1A4C055
:1024A000C2E4D6E30CE911E189911F928F931F9347
:1024B0000F930E94D99B0F900F900F900F90B6E34F
:1024C000CA34DB0789F720E030E048EC52E4C7016A
:1024D000B6010E94AB939F938F937F936F938CE889
:1024E00091E19F938F930E94D99B0F900F900F9033
:1024F0000F900F900F9080914A36811103C08AE9A6
:1025000093E002C088E193E09F938F9388E891E184
:102510009F938F930E94D99B0F900F900F900F90D5
:102520006DC000E010E0FE01E00FF11F80811F92FE
:102530008F93A0E7B1E1BF93AF930E94D99B0F5F48
:102540001F4F0F900F900F900F900830110559F703
:1025500020E030E048EC52E4C301B2010E94AB93AA
:102560009F938F937F936F933F922F920E94D99B5B
:102570000F900F900F900F900F900F908885811102
:1025800051C08AE993E09F938F939F928F920E940C
:10259000D99B0E94F111FFEFEF1AFF0A29960F90C5
:1025A0000F900F900F90D6018C9190E0E816F906ED
:1025B000E4F5CE010E94B362BC01990F880B990B20
:1025C0000E945F942B013C01A114B10409F4A9CF2E
:1025D00020E030E048EC52E40E94AB939F938F934D
:1025E0007F936F9385E791E19F938F930E94D99B8F
:1025F0000F900F900F900F900F900F90DF91CF9151
:102600001F910F91FF90EF90DF90CF90BF90AF9010
:102610009F908F907F906F905F904F903F902F9002
:102620000C94F11188E193E0AECFDF91CF911F912F
:102630000F91FF90EF90DF90CF90BF90AF909F9061
:102640008F907F906F905F904F903F902F90089564
:10265000CF93DF931F921F92CDB7DEB7E2E4F6E38C
:102660008181898387818A83CE0101960E94757753
:102670000F900F90DF91CF910895CF93DF93EC01EE
:102680002091423630914336409144365091453640
:102690006091463670914736809148369091493620
:1026A000AFEF0E94BB92E1F427E04AE250E06BE218
:1026B00070E089E290E00E94E26080E090E00E9499
:1026C0008911C85DDB4E888349E050E06EE070E020
:1026D00082E496E30E94A49EDF91CF910C9428138C
:1026E000DF91CF9108951F920F920FB60F92112490
:1026F0000BB60F92FF920F931F932F933F934F931D
:102700005F936F937F938F939F93AF93BF93CF9379
:10271000DF93EF93FF93809159368260809359360F
:102720008091660286FD2B9A8091660287FD2B9A26
:1027300080919102909192021816190614F4749ADD
:10274000739A80912D1490912E14A0912F14B09112
:10275000301485FF02C0749873988091060290919E
:10276000070201979093070280930602892B09F0D4
:102770004CC18091E20A9091E30A01969093E30A9A
:102780008093E20A80917F3190918031A0918131D4
:10279000B09182310196A11DB11D80937F3190933C
:1027A0008031A0938131B093823180E190E09093A9
:1027B0000702809306028091660280FD02C01D9B85
:1027C00005C010922C1410922B1406C081E090E0EA
:1027D00090932C1480932B1480912D1490912E148F
:1027E000A0912F14B091301497FF08C080912B1442
:1027F00090912C14892B49F0749A73980CE51DE183
:10280000C4E9D1E3FF24F39421C0739A7498F6CFFE
:102810008091E20A9091E30A01960E946090892BD0
:10282000E1F0F8016085718561157105A1F5F80188
:10283000608571856115710509F03FC0065F1F4F06
:102840002596F1E3C83ADF0709F44CC0F80160852A
:1028500071856115710529F3DBCF4281417020E05C
:1028600030E050E060E070E080E090E0A0E00E94A6
:10287000BB92B9F2779880912D1490912E14A0916B
:102880002F14B091301492FFCCCF74981092920212
:1028900010929102C6CF8091E20A9091E30A0196CC
:1028A0000E946090892B19F61C821B82AE0162E1A6
:1028B00084E292E00E944773BACF8091E20A90913D
:1028C000E30A0E946090892B09F0B8CFF8821A833E
:1028D00009831C821B82AE0162E182E492E00E94C5
:1028E0004773ACCF60916C0270916D0261157105F8
:1028F000A1F18091E20A9091E30A0E946090892BF5
:1029000061F58091283690912936A0912A36B091B0
:102910002B364091712950917229609173297091E1
:102920007429841B950BA60BB70B8093841D909381
:10293000851DA093861DB093871D809128369091A8
:102940002936A0912A36B0912B3680937129909325
:102950007229A0937329B093742960916A027091CF
:102960006B0261157105A1F18091E20A9091E30A71
:102970000E946090892B61F580912C3690912D36C4
:10298000A0912E36B0912F3640917529509176291D
:102990006091772970917829841B950BA60BB70B52
:1029A0008093881D9093891DA0938A1DB0938B1DE1
:1029B00080912C3690912D36A0912E36B0912F36E5
:1029C0008093752990937629A0937729B0937829DD
:1029D0008091660286FD2B98809166029091670235
:1029E000A0916802B091690291FF0FC00E946D6CC6
:1029F0008A3119F0C1E0C80F01C0CBE00E94AA6A79
:102A00008C2F0E94856C0E94746B40E050E060E067
:102A100085EB92E00E944773FF91EF91DF91CF9198
:102A2000BF91AF919F918F917F916F915F914F91E6
:102A30003F912F911F910F91FF900F900BBE0F9020
:102A40000FBE0F901F9018958091AC1D90919331FF
:102A5000891B08950E942415882371F0E091933119
:102A6000EF73F0E0E350F24E808190E020919331DB
:102A70002F5F2093933108958FEF9FEF0895CF93A9
:102A8000DF93EC011092130B1092120B8881998145
:102A90000097C1F08D3E934021F01982188283E0A7
:102AA000BDC0613109F0B9C00E942A1599279093E1
:102AB0000E0B80930D0B8D30910509F444C08F3FB0
:102AC000910549F40E9424158111EECF8DEE93E01B
:102AD00099838883A2C08231910509F45AC08F3747
:102AE000910509F052C080910B0B90910C0B1816B8
:102AF00019060CF56091B73A7091B83A88E090E009
:102B00000E948D9B6091B73A7091B83A80E290E054
:102B10000E948D9B6091B73A7091B83A88E090E03E
:102B20000E948D9B80910B0B90910C0B01979093C1
:102B30000C0B80930B0B80910B0B90910C0B8F3730
:102B4000910509F0BFCF109293311092AC1D809186
:102B50000B0B90910C0BFC01E855FE4C10829093EE
:102B6000130B8093120B10920C0B10920B0B809195
:102B70004B3690914C36009709F4A4CF40E050E0DA
:102B8000609125140E9447739DCF8830910571F59F
:102B9000AACF6091B73A7091B83A8DE090E00E9468
:102BA0008D9B10920A0B1092090B2091090B30910A
:102BB0000A0B80910B0B90910C0B281739070CF026
:102BC000BACFF901E855FE4C80816091B73A709117
:102BD000B83A90E00E948D9B8091090B90910A0B6E
:102BE000019690930A0B8093090BDFCF6091B73A5F
:102BF0007091B83A0E948D9B20910B0B30910C0B79
:102C000080910D0BF901E855FE4C80832F5F3F4FFB
:102C100030930C0B20930B0B8ECF81E0DF91CF9183
:102C2000089580912B1490912C14892BD1F08091D0
:102C3000660290916702A0916802B091690293FDCB
:102C400010C00E94AA6A83B7817F866083BFF89410
:102C500083B7816083BF7894889583B78E7F83BF65
:102C600078940895CF93DF93FC0120813181211561
:102C7000310551F0273A324129F0FC0111821082CE
:102C800083E015C0653891F4EC010E94A8690E94A8
:102C9000111640E050E065E880916F159091701535
:102CA0000E94477387EA92E19983888381E0DF91EC
:102CB000CF910895CF93DF931F921F92CDB7DEB7C8
:102CC000892B81F05F934F9381E691E19F938F93DE
:102CD00069837A830E94D99B0F900F900F900F9079
:102CE0007A8169817F936F938EE591E19F938F93B2
:102CF0000E94D99B0F900F900F900F900F900F9004
:102D0000DF91CF910895CF93DF931F921F92CDB79C
:102D1000DEB74A8369830E9471636981862F0E94AE
:102D2000A2634A81842F0E94A2630F900F90DF91CB
:102D3000CF910C949A63AF92BF92CF92DF92EF92B1
:102D4000FF920F931F93CF93DF9300D0CDB7DEB7E1
:102D5000182F022F4A835B8369830E947163698104
:102D6000862F0E94A263812F81600E9498634A810E
:102D7000A42E5B81B52E10E0E12CF12C680181E0DE
:102D8000C81AD108E016F10689F0EC14FD0419F414
:102D90000E94BD6302C00E94B363F5018083FFEF10
:102DA000EF1AFF0A8FEFA81AB80AECCF0F900F9016
:102DB0000F90DF91CF911F910F91FF90EF90DF90D7
:102DC000CF90BF90AF900C949A63CF92DF92EF9226
:102DD000FF920F931F93CF93DF931F92CDB7DEB770
:102DE0000E94A86980EB0E943D6381111CC00E9473
:102DF0009A638091792D90917A2D816090937A2DAC
:102E00008093792D81E293E09F938F938EE591E1FA
:102E10009F938F930E94D99B0F900F900F900F90CC
:102E200001E010E002C000E010E08EB18470F82EE6
:102E3000729A64E278E680E090E00E941A630E9451
:102E4000A8698EE40E943D63811117C00E949A63B5
:102E50008091792D90917A2D826090937A2D809334
:102E6000792D68018FEFC81AD80A46EB59E069E25C
:102E700073E0C8010E945A168601F11001C07298D1
:102E800064E278E680E090E00E941A630E94A869FC
:102E90008EEE0E943D63811159C019820E949A638F
:102EA00021E030E0AE014F5F5F4F60ED70E08EEEED
:102EB00090E00E949B1689818535A9F48091792D37
:102EC00090917A2D846090937A2D8093792D78015A
:102ED0008FEFE81AF80A46EB59E061E373E0C801A6
:102EE0000E945A16870189818835A9F48091792D2D
:102EF00090917A2D806190937A2D8093792D78012D
:102F00008FEFE81AF80A46EB59E068E373E0C8016E
:102F10000E945A16870189818036C1F48091792DEB
:102F200090917A2D806290937A2D8093792D7801FB
:102F30008FEFE81AF80A46EB59E06FE373E0C80137
:102F40000E945A1681E00E94BE7C870164E278E606
:102F500080E090E00E941A630E94A86986EA0E94BD
:102F60003D63811117C00E949A638091792D9091E1
:102F70007A2D806490937A2D8093792D78018FEF4C
:102F8000E81AF80A46EB59E066E473E0C8010E94CB
:102F90005A16870164E278E680E090E00E941A63A6
:102FA0000E94A8698CE30E943D6381111FC00E94AA
:102FB0009A638091792D90917A2D806890937A2DE3
:102FC0008093792D78018FEFE81AF80A46EB59E0E3
:102FD0006EE473E0C8010E945A1686E591E19F9362
:102FE0008F930E94D99B0F900F90870164E278E63F
:102FF00080E090E00E941A630E94A86982ED0E941E
:103000003D63811117C00E949A638091792D909140
:103010007A2D916090937A2D8093792D78018FEF9E
:10302000E81AF80A46EB59E066E573E0C8010E9429
:103030005A16870164E278E680E090E00E941A6305
:103040000E94A86980E80E943D63811117C00E9418
:103050009A638091792D90917A2D986090937A2D32
:103060008093792D78018FEFE81AF80A46EB59E042
:103070006FE573E0C8010E945A16870164E278E6A2
:1030800080E090E00E941A630E94A86980ED0E948F
:103090003D63811117C00E949A638091792D9091B0
:1030A0007A2D946090937A2D8093792D78018FEF0B
:1030B000E81AF80A46EB59E065E673E0C8010E9499
:1030C0005A16870164E278E680E090E00E941A6375
:1030D0000E94A8698CEE0E943D63811117C00E9476
:1030E0009A638091792D90917A2D906190937A2DA9
:1030F0008093792D78018FEFE81AF80A46EB59E0B2
:103100006DE673E0C8010E945A16870187E0E82E39
:10311000F12C64E278E680E090E00E941A630E945D
:10312000A8698CE70E943D63811113C00E949A63D5
:103130008091792D90917A2D926090937A2D809341
:10314000792D46EB59E064E773E0C8010E945A16F6
:1031500004C081E0E81AF108E1F60E949A630E9437
:10316000F1110F90DF91CF911F910F91FF90EF9090
:10317000DF90CF900895BF92CF92DF92EF92FF92AF
:103180000F931F93CF93DF93CDB7DEB760970FB642
:10319000F894DEBF0FBECDBFF82EE42E6623D9F122
:1031A0008E010F5F1F4F80E1F80111928A95E9F7B8
:1031B00028E0A80168E980EB0E949B16FF2041F0FF
:1031C0008DE793E09F938F930E94C59B0F900F9084
:1031D00024E8C22E23E0D22E37E0B32EB00EF80141
:1031E00081918F011F928F93DF92CF920E94C59B96
:1031F0000F900F900F900F90B012F1CF88851F9213
:103200008F9389ED93E09F938F930E94C59B0F90BE
:103210000F900F900F90EE20D9F18E010F5F1F4F8E
:1032200080E1F80111928A95E9F720E1A80160E8B0
:1032300080EB0E949B16FF2041F089E893E09F936A
:103240008F930E94C59B0F900F9084E8E82E83E037
:10325000F82E9FE0D92ED00EF80181918F011F9298
:103260008F93FF92EF920E94C59B0F900F900F904B
:103270000F90D012F1CF88891F928F9389ED93E040
:103280009F938F930E94C59B0F900F900F900F906C
:1032900060960FB6F894DEBF0FBECDBFDF91CF9121
:1032A0001F910F91FF90EF90DF90CF90BF90089506
:1032B0000F931F93CF93DF931F921F92CDB7DEB76B
:1032C0001A82198222E0AE014F5F5F4F6AEA8EEEEA
:1032D0000E949B160DE31EE1898190E0982F8827BC
:1032E0002A81822BF8019183808322E0AE014F5F17
:1032F0005F4F6CEA8EEE0E949B16898190E0982FBA
:1033000088272A81822BF8019383828322E0AE01F1
:103310004F5F5F4F6EEA8EEE0E949B16898190E0B0
:10332000982F88272A81822BF8019583848322E0B5
:10333000AE014F5F5F4F60EB8EEE0E949B1689815E
:1033400090E0982F88272A81822BF801938B828B1B
:1033500022E0AE014F5F5F4F62EB8EEE0E949B1644
:10336000898190E0982F88272A81822BF801958BFC
:10337000848B22E0AE014F5F5F4F64EB8EEE0E94C4
:103380009B16898190E0982F88272A81822BF8014B
:10339000978B868B22E0AE014F5F5F4F66EB8EEE20
:1033A0000E949B16898190E0982F88272A81822B82
:1033B000F8019783868322E0AE014F5F5F4F68EB91
:1033C0008EEE0E949B16898190E0982F88272A8193
:1033D000822BF8019187808722E0AE014F5F5F4F1B
:1033E0006AEB8EEE0E949B16898190E0982F8827C9
:1033F0002A81822BF8019587848722E0AE014F5FF6
:103400005F4F6CEB8EEE0E949B16898190E0982FA7
:1034100088272A81822BF8019787868722E0AE01D0
:103420004F5F5F4F6EEB8EEE0E949B16898190E09E
:10343000982F88272A81822BF801918B808B0F90FF
:103440000F90DF91CF911F910F9108952F923F928E
:103450004F925F926F927F928F929F92AF92BF92A4
:10346000CF92DF92EF92FF920F931F93CF93DF9350
:10347000CDB7DEB76C970FB6F894DEBF0FBECDBFE9
:10348000182F042F2D8B19821A821B828091611EA6
:10349000811107C06C8F0E94581981E08093611ED2
:1034A0006C8D662309F472C04EE264EF8EEE0E94CA
:1034B000831662E174E380E090E00E941A6322E0E8
:1034C000AE014F5F5F4F66EF8EEE0E949B16298123
:1034D000822F90E0A0E0B0E04427582F692F7A2F88
:1034E0008A81482B8091531E9091541E9A01AB0102
:1034F000281B390B41095109A091511EB091521E50
:103500000E94EF906B017C013FE0F594E794D79423
:10351000C7943A95D1F760914B1E70914C1ECB0128
:10352000770FAA0BBB0BBC01CD014BE0660F771FD9
:10353000881F991F4A95D1F720914D1E30914E1E3C
:103540004901330FAA08BB08A7019601280D391DB0
:103550004A1D5B1D0E94AA90C20ED31ED092481E27
:10356000C092471E28E0C20ED11C54E0D594C794E7
:103570005A95E1F70D2C000CEE08FF08C092551E7D
:10358000D092561EE092571EF092581E812F8295BF
:10359000880F880F807C8C5C8887212E312CA3E0DB
:1035A000B0E0012E02C0AA0FBB1F0A94E2F72AE680
:1035B0003AE00E94E8909B01AC012E5F3F4F4F4FD5
:1035C0005F4F29873A874B875C8780E593ECA0E0C3
:1035D000B0E09C01AD0104C05595479537952795FE
:1035E0001A95D2F7298B3A8B4B8B5C8B10E0412CD0
:1035F000512C320188E090E0AC01421953095B8FF5
:103600004A8F101709F43EC1488564EF8EEE0E9480
:10361000831669857A858B859C850E941A6323E0D1
:10362000AE014F5F5F4F66EF8EEE0E949B16E091FA
:10363000471EF091481EE05AFF409F01DF010E94A3
:10364000D1906C837D838E839F8380913F1E909168
:10365000401E9E878D8720913D1E30913E1E388BE7
:103660002F872091411E3091421E0E94D1906B0104
:103670007C01ADE0F594E794D794C794AA95D1F76F
:10368000A091431EB091441E2C813D814E815F81EB
:103690008CE055954795379527958A95D1F70E94E7
:1036A000FA90BB2797FDB095AB2F8C0D9D1DAE1DDD
:1036B000BF1D0296A11DB11D32E0B595A795979546
:1036C00087953A95D1F79C01AD0130584F4F5F4F28
:1036D000A0914F1EB091501E0E94EF904B015C01D3
:1036E0004FE0B694A794979487944A95D1F739817F
:1036F0008A8190E0A0E0B0E0BA2FA92F982F882708
:10370000A32B2B81822B9C01AD010A8C04C0559503
:103710004795379527950A94D2F72E8B3F8B488F84
:10372000598F4F8558896A01550FEE08FF0862E0EE
:10373000CC0CDD1CEE1CFF1C6A95D1F7A091451E38
:10374000B091461E2C813D814E815F810E94FA908E
:103750009B01AC0177E155954795379527957A956B
:10376000D1F72C833D834E835F832D853E85DF011A
:103770000E94D190DC01CB01EBE0B595A795979520
:103780008795EA95D1F72C813D814E815F81820F2B
:10379000931FA41FB51FC80ED91EEA1EFB1E022CC4
:1037A00004C0CC0CDD1CEE1CFF1C0A94D2F732E0E6
:1037B000C30ED11CE11CF11CF2E0F594E794D79400
:1037C000C794FA95D1F72E893F89488D598D2C19C8
:1037D0003D094E095F0969897A898B899C890E9414
:1037E000449097FD0BC0660F771F881F991FA50196
:1037F00094010E94889069017A010AC0A501940190
:103800000E94889069017A01CC0CDD1CEE1CFF1C23
:103810009927F7FC9A958F2D7E2D6D2D9B01AC017C
:103820000E9444909B01AC01AEEDBBE00E94EF9082
:103830004C01BB2497FCB094AB2CA3E4B3EEA701DE
:1038400096010E94FD90BB2797FDB095AB2F880E87
:10385000991EAA1EBB1E4FEC840E4EE0941EA11CA6
:10386000B11C44E0B594A794979487944A95D1F7F6
:10387000C80CD91CEA1CFB1C4C0C5D1C6E1C7F1C6C
:103880001F5FBFCE112381F0212F30E040E050E0D8
:10389000C301B2010E9488902093591E30935A1E92
:1038A00040935B1E50935C1E5D89552389F16091A6
:1038B000591E70915A1E80915B1E90915C1E61157D
:1038C00071058105910521F10E945F9420E836EE93
:1038D00045EC57E40E94AB9321E03EED42E45EE309
:1038E0000E94C4969B01AC0160E070E080E89FE319
:1038F0000E94C7922BE43AE34DEB57E30E94AB934F
:1039000060935D1E70935E1E80935F1E9093601E99
:103910006C960FB6F894DEBF0FBECDBFDF91CF918E
:103920001F910F91FF90EF90DF90CF90BF90AF90DD
:103930009F908F907F906F905F904F903F902F90CF
:1039400008950F931F93CF93DF9300D000D0CDB78E
:10395000DEB78E010F5F1F4F86E0F80111928A9546
:10396000E9F78091531D811113C040E061E386EABD
:103970000E9483164AE06CE286EA0E94831681E088
:103980008093531D68EF7CE780E090E00E941A630B
:1039900048E06DE286EA0E94831668EF7CE780E0EB
:1039A00090E00E941A6326E0A80162E386EA0E9482
:1039B0009B1647E06DE286EA0E9483168A8190E0BA
:1039C000982F88272981822B90934E1D80934D1D1F
:1039D0002C8130E0322F22274B81242B3093501D35
:1039E00020934F1D4E8150E0542F44276D81462B6C
:1039F0005093521D4093511D5F934F933F932F93CC
:103A00009F938F938DE893E09F938F930E94C59B24
:103A10000FB6F894DEBF0FBECDBF26960FB6F89452
:103A2000DEBF0FBECDBFDF91CF911F910F910895E3
:103A3000CF92DF92EF92FF920F931F93CF93DF937A
:103A4000CDB7DEB72A970FB6F894DEBF0FBECDBF55
:103A50008E010F5F1F4F86E0F80111928A95E9F7FA
:103A600041E062E08CE30E94831648E560E08CE36D
:103A70000E94831664E278E680E090E00E941A6378
:103A800026E0A80163E08CE30E949B1643E062E01D
:103A90008CE30E948316098110E0102F00278A8191
:103AA000082BEDE2FDE111830083EB80F12CFE2C6D
:103AB000EE248C81E82AF382E282CD80D12CDC2CAA
:103AC000CC248E81C82AD582C482B801012E000C74
:103AD000880B990B0E945F949B01AC01B7010F2CDE
:103AE000000C880B990B2F83388749875A870E94CF
:103AF0005F942F81388549855A850E94479320EE2F
:103B00003EE245E652E40E94579620E030E044E36E
:103B100053E40E94C8929F938F937F936F93DF9299
:103B2000CF92FF92EF921F930F938BE993E09F93B5
:103B30008F930E94C59B0FB6F894DEBF0FBECDBF1A
:103B40002A960FB6F894DEBF0FBECDBFDF91CF919E
:103B50001F910F91FF90EF90DF90CF900895CF933A
:103B6000DF93EC01888199810097A9F18C3892410B
:103B700021F01982188283E083C080EF9AE00E94CE
:103B8000D571892BA1F180912D1490912E14A091C3
:103B90002F14B091301493FD2CC080912D1490916E
:103BA0002E14A0912F14B091301493FD53C0809126
:103BB0002D1490912E14A0912F14B091301494FDD7
:103BC00051C080912D1490912E14A0912F14B0917A
:103BD000301495FD4EC040E850E060E070E080EFAA
:103BE0009AE00E94B7718CE892E19983888381E022
:103BF00047C08091792D82FFD0CF21E048E061E07D
:103C000083E00E94261A8091601E8F9380915F1E30
:103C10008F9380915E1E8F9380915D1E8F93809114
:103C20005C1E8F9380915B1E8F9380915A1E8F93A1
:103C30008091591E8F938AE192E19F938F930E9406
:103C4000D99B8DB79EB70A960FB6F8949EBF0FBE4C
:103C50008DBFA3CF8091792D85FFA9CF81E00E94F0
:103C6000B27DA5CF8091792D86FFABCF0E94A11C9C
:103C7000A8CF8091792D87FFAECF0E94181DABCFC2
:103C8000DF91CF910895CF93DF93C82F8CEE0E94E0
:103C900098638C2F0E94A2636AE67AE080E090E04D
:103CA0000E941A638DEE0E9498630E94B363D82F1E
:103CB0000E94BD63C82F0E949A638C2F90E09D2BB9
:103CC000DF91CF9108951F93CF93DF93C82F8CEE90
:103CD0000E9498638C2F0E94A26364E278E680E0E1
:103CE00090E00E941A638CEE0E94986380E00E942C
:103CF000A2636AE67AE080E090E00E941A638DEEAB
:103D00000E9498630E94B363D82F0E94B363182F58
:103D10000E94BD63C82F0E949A63812F90E0A0E0AB
:103D2000B0E0BA2FA92F982F8827AD2BBC01CD0169
:103D30006C2BDF91CF911F9108952F923F924F925C
:103D40005F926F927F928F929F92AF92BF92CF922B
:103D5000DF92EF92FF920F931F93CF93DF93CDB734
:103D6000DEB7CB54D1090FB6F894DEBF0FBECDBF7E
:103D70008091040290910502892BE1F110920502D5
:103D8000109204028CEE0E9498638EE10E94A2635E
:103D90000E949A6366E37CE980E090E00E941A63E7
:103DA00082EA0E94431E9093E10A8093E00A84EA2B
:103DB0000E94431E9093DF0A8093DE0A86EA0E94E7
:103DC000431E9093DD0A8093DC0A88EA0E94431E1A
:103DD0009093DB0A8093DA0A8AEA0E94431E90934A
:103DE000D90A8093D80A8CEA0E94431E9093D70A7E
:103DF0008093D60A88E40E94631E6DAB7EAB8FABC6
:103E000098AF88E50E94631E4B015C018091D80A3F
:103E10009091D90A8C0120E030E040E050E0BA01F6
:103E200022968FAF229723961FAF239724962FAF0A
:103E3000249725963FAF259726964FAF269727962E
:103E40005FAF279728966FAF289729967FAF29975E
:103E50009C0140E050E060E070E080E090E008E02D
:103E60000E945D920E9416923901B42FA52FF62F61
:103E7000E72F8C019401A50160E070E080E090E004
:103E80005301CB2EDA2EEF2EFE2E0E9494922CA3FD
:103E90003BA349835A831B012C01C20131504109C4
:103EA0005F4F6F4F7F4F8F4F9F4F88248394912C8C
:103EB00021153F4F4F4F5140610571058105910517
:103EC00009F010F4812C912C34010091D60A109144
:103ED000D70A5801C12CD12CE12CF12C00E010E0C4
:103EE0002CA13BA149815A81B101C2010E940291DA
:103EF000F22E032F142FB52FF62FE72FD82EE92EF1
:103F0000A0E00E94BB9284F42150310940485F4FE9
:103F10006F4F7F4F8F4F9F4FF22E032F142FB52FD0
:103F2000F62FE72FD82EE92E2F2D302F412F5B2F84
:103F30006F2F7E2F8D2D9E2D07E10E9476922B8F65
:103F40003C8F4D8F5E8F6F8F78A389A39AA32053E8
:103F5000384F4F4F5F4F6F4F7F4F8F4F9F4F2B8B80
:103F60003C8B4D8B5E8B6F8B788F898F9A8F205611
:103F7000304F4F4F5F4F6F4F7F4F8F4F9F4F243DBD
:103F8000304341055105610571058105910529F011
:103F900020F03401BFEF6B1A7B0A8090DE0A90900C
:103FA000DF0A940140E050E060E070E080E090E0E3
:103FB00000E10E945D922B833C834D835E836F837F
:103FC00078874C014091DA0A5091DB0AACA0BBA083
:103FD000C980DA80710182019A0140E050E060E01E
:103FE00070E080E090E00E940291F22E032F142FE7
:103FF000B52FF62FE72FD82EE92EA0E00E94BB9216
:104000005CF4AFE70E949D92F22E032F142FB52F80
:10401000F62FE72FD82EE92E2F2D302F412F5B2F93
:104020006F2F7E2F8D2D9E2D07E00E9476925901D5
:104030006A017B018C012B813C814D815E816F8106
:104040007885C4010E9494922B833C834D835E83C8
:104050006F8378878F87988B2E5F3F4F434051093E
:104060006E4F7F4F8F4F9F4F22303105494F5F4F2B
:10407000644071058105910521F018F0FFEF6F1A7A
:104080007F0A6091E00A7091E10A80E090E020E010
:1040900030E840E050E00E945B9129873A874B87E7
:1040A0005C876D877E874C014091DC0A5091DD0A68
:1040B000ACA0BBA0C980DA80710182019A0140E006
:1040C00050E060E070E080E090E00E940291F22E0B
:1040D000032F142FB52FF62FE72FD82EE92EA0E0AF
:1040E0000E94BB9284F421503F4F4F4F5F4F6F4F60
:1040F0007F4F8F4F9F4FF22E032F142FB52FF62F88
:10410000E72FD82EE92E2F2D302F412F5B2F6F2F29
:104110007E2F8D2D9E2D08E00E94769259016A0116
:104120007B018C0129853A854B855C856D857E8573
:10413000C4010E94949229873A874B875C876D87D8
:104140007E87898B9A8B2F5F3F4F414051096109D0
:10415000710981099109213030484C4F5F47614016
:1041600071058105910521F018F01FEF611A710AA0
:104170002B893C894D895E896F89788D898D9A8DCF
:104180002F3C3740410551056105710581059105B9
:1041900011F00CF09CC1ACA0BBA0C980DA80710109
:1041A00082019501A601B101C2010E940291A12CD8
:1041B000B12CC12CE0E8DE2EE12CF12C00E010E067
:1041C0000E94889129AF3AAF4BAF5CAF6DAF7EAF25
:1041D0008FAF21969FAF2197AB8CBC8CCD8CDE8CA2
:1041E000EF8CF8A009A11AA19501A601B701C80199
:1041F0000E94029159016A017B01E82F192F02E008
:104200000E945D920E2F0E9494927901142F452EE8
:10421000F62FE72F6C01922EAF2CB42E052F362EE1
:10422000B72F582E8D2CA0E00E94BB925CF4A1E029
:104230000E949D92922EA32EB42E052F362EB72FBC
:10424000582E892E292D3A2D4B2D502F632D7B2F43
:10425000852D982D01E00E94769229A73AA74A0160
:104260002C966FAF2C972B967FAF2B978BA79CA785
:1042700029833A834BA39CA26DA37EA38FA398A707
:10428000B42D9701412F542D6F2F7E2FC601A0E032
:104290000E94BB924CF4A3E00E949D927901142FDE
:1042A000B52FF62FE72F6C019701412F5B2F6F2F52
:1042B0007E2FC60102E00E9476922DA73EA74FA74F
:1042C00058AB69AB7AAB8BAB9CAB2901B42FA52F54
:1042D00022966FAF2297F72F1C012B893C894D89BD
:1042E0005E896F89788D898D9A8D24323A4F4F4F30
:1042F0005F4F6F4F7F4F8F4F9F4F0CF08BC02B8DB9
:104300003C8D4D8D5E8D6F8D78A189A19AA124552C
:10431000324F4F4F5F4F6F4F7F4F8F4F9F4F59011E
:104320006A017B018C010E94029119012A01B62FBA
:10433000A72FFC0103E00E945D9251016201EB2E68
:10434000FA2E8F010E94A99259016A017B018C010A
:1043500029A53AA5A4012C966FAD2C972B967FAD7D
:104360002B978BA59CA50E94949229833A834BA3FB
:104370005CA36DA37EA38FA398A79101A2016B2FCD
:104380007A2FCF0102E00E945D9251016201EB2E73
:10439000FA2E8F010E94A99202E00E945D920E2FD8
:1043A0000E94A992122FD32EE42EB52FF62FE72FBD
:1043B000F82E092FA0E00E94BB925CF4A1E00E94BD
:1043C0009D92122FD32EE42EB52FF62FE72FF82E25
:1043D000092F212F3D2D4E2D5B2F6F2F7E2F8F2DDF
:1043E000902F01E00E94769259016A017B018C01B5
:1043F0002DA53EA54FA558A969A97AA98BA99CA965
:104400000E9494922901B42FA52F22966FAF229774
:10441000F72F1C012B813C814D815E816F81788556
:104420008F859889A980BA80CBA0DCA0EDA0FEA0E2
:104430000FA118A50E94A9922B833C834D835E8314
:104440006F8378878F87988B29853A854B855C8524
:104450006D857E8589899A895201CB2EDA2E229626
:10446000EFAC2297FF2E81010E94A99229873A87FB
:104470004B875C876D877E87898B9A8B2B893C89DC
:104480004D895E896F89788D898D9A8DA9ACBAAC7A
:10449000CBACDCACEDACFEAC0FAD21961FAD2197E3
:1044A0000E94A9922056304F4F4F5F4F6F4F7F4F62
:1044B0008F4F9F4F243D30434105510561057105E4
:1044C0008105910521F018F00FEF601A700A4DA9CF
:1044D0005EA96FA978AD9A01AB0160E070E0CB01F5
:1044E00022962FAF229723963FAF239724964FAF64
:1044F000249725965FAF259726966FAF2697279628
:104500007FAF279728968FAF289729969FAF299737
:10451000A984BA84CB84DC84ED84FE8409891A8959
:1045200060E070E080E090E00E940291122FD32EB4
:10453000E42EB52FF62FE72FF82E092FA0E00E94CA
:10454000BB9284F421503109404E5F4F6F4F7F4F33
:104550008F4F9F4F122FD32EE42EB52FF62FE72F1C
:10456000F82E092F212F3D2D4E2D5B2F6F2F7E2FE3
:104570008F2D902F05E10E947692AB80BC80CD807C
:10458000DE80EF80F8840F8518890E94A992122F8F
:10459000D32EE42EB52FF62FE72FF82E092FA0E00B
:1045A0000E94BB9284F4215030484F4F5F4F6F4FB1
:1045B0007F4F8F4F9F4F122FD32EE42EB52FF62F04
:1045C000E72FF82E092F212F3D2D4E2D5B2F6F2F1A
:1045D0007E2F8F2D902F0FE00E94769259016A0155
:1045E0007B018C01322E5B2CB42FAD2DF62F4F2C7E
:1045F0004C01285E33404109510961097109810963
:104600009109283D304D41405105610571058105F5
:10461000910509F010F4672869F09501A601B7012A
:10462000C8010E941692322E532EB42FA52FF62FBA
:10463000472E4C01232D352D4B2F5A2F6F2F742DC4
:10464000C4010E94579420E030E048EC52E40E94FC
:10465000AB93C55BDF4F0FB6F894DEBF0FBECDBF87
:10466000DF91CF911F910F91FF90EF90DF90CF904E
:10467000BF90AF909F908F907F906F905F904F9082
:104680003F902F9008954F925F926F927F928F92FA
:104690009F92AF92BF92CF92DF92EF92FF922B0147
:1046A0003C0169017A0123EC35EF4CE851E4C70184
:1046B000B6010E9457964B015C0128EB3EE143E7AF
:1046C00053E4C701B6010E94C8929B01AC01C50129
:1046D000B4010E94AB930E9425944B015C0120E041
:1046E00030E048EC52E4C301B2010E94AB9321E8F0
:1046F00035E943EC50E40E945796A50194010E94CD
:1047000057964B015C0123E333E948E853E4C701C2
:10471000B6010E94C8929B01AC01C501B4010E9480
:10472000AB9323E333EB48E553E40E945796FF90A5
:10473000EF90DF90CF90BF90AF909F908F907F9041
:104740006F905F904F9008954F925F926F927F921B
:104750008F929F92AF92BF92CF92DF92EF92FF9291
:1047600069017A010E94CB9520E030E040E050E4FE
:104770000E94C79222E93CE54EED5EE30E94AB93B6
:104780004B015C0123EC35EF4CE851E4C701B60165
:104790000E9457962B013C0128EB3EE143E753E48E
:1047A000C701B6010E94C8929B01AC01C301B201CE
:1047B0000E94AB939B01AC01C501B4010E94C89259
:1047C0006B017C0128EB3EE143E753E40E945796DE
:1047D0004B015C01A701960163EC75EF8CE891E455
:1047E0000E94C7929B01AC01C501B4010E94AB932A
:1047F000FF90EF90DF90CF90BF90AF909F908F9001
:104800007F906F905F904F9008954F925F926F925C
:104810007F928F929F92AF92BF92CF92DF92EF9250
:10482000FF922B013C0169017A0123EC35EF4CE842
:1048300051E4C701B6010E9457964B015C0128EB79
:104840003EE143E753E4C701B6010E94C8929B01D1
:10485000AC01C501B4010E94AB930E9425944B01A9
:104860005C0120E030E048EC52E4C301B2010E9458
:10487000AB93A50194010E94579620E030E040E2FE
:1048800051E40E94C79224EE38E34EE05FE30E94B9
:1048900057969B01AC01C701B6010E94C892FF90D8
:1048A000EF90DF90CF90BF90AF909F908F907F90D0
:1048B0006F905F904F90089580E80E9498638111F7
:1048C0000DC08EEF0E94A263811108C066E37CE9EF
:1048D00080E090E00E941A630C949A630E949A63AD
:1048E00080918B3190918C31A0918D31B0918E312E
:1048F0000196A11DB11D80938B3190938C31A093B3
:104900008D31B0938E310895FC01DC01AC014E5F16
:104910005F4F90E031E38D91982788E0292F220F97
:1049200097FF03C0922F932701C0922F8150B1F7B8
:10493000A417B50781F721E030E08281981711F0C4
:1049400020E030E0C9010895DF92EF92FF920F93CB
:104950001F93CF93DF930E945C2480E80E949863AA
:1049600081116DC08AEF0E94A263811168C08FE03F
:104970000E94A263811163C06AE67AE080E090E061
:104980000E941A6381E80E949863811158C00E94B6
:10499000B363D82F0E94B3630E94B363182F0E94A1
:1049A000B3630E94B363082F0E94B3630E94BD6388
:1049B000F82E80E80E949863811141C08CEF0E941C
:1049C000A26381113CC089EC0E94A263811137C0AF
:1049D0006AE67AE080E090E00E941A6381E80E9433
:1049E00098630E94B363E82E0E94B363D82E0E949E
:1049F000B3630E94B363C82F0E94BD631F92DF920E
:104A00001F92EF921F92FF921F920F931F921F937C
:104A10001F92DF931F928F931F92CF9380EB93E0AF
:104A20009F938F930E94C59B0E949A638DB79EB7F8
:104A300042960FB6F8949EBF0FBE8DBF17C00E945E
:104A40009A6380918B3190918C31A0918D31B0918E
:104A50008E310196A11DB11D80938B3190938C31C5
:104A6000A0938D31B0938E310E945C2420E030E021
:104A700040E050E060E070E080E090E0DF91CF91B6
:104A80001F910F91FF90EF90DF900895EF92FF92AA
:104A90000F931F93CF93DF9300D0CDB7DEB78C0178
:104AA00080E80E949863811154C00115110551F0EE
:104AB00085EE0E94A26381114CC062E07EE281E03B
:104AC00090E009C083EE0E94A263811142C062E3BC
:104AD00075E783E090E00E941A6381E80E94986382
:104AE000811137C00E94B363E82E89830E94B363AB
:104AF000F82E8A830E94BD638B830E949A63CE0145
:104B000001960E948424892B21F16F2D70E07E296B
:104B10006C7F80E090E0012B69F00E945D9420E0C2
:104B200030E04AEF5AE30E94579620E030E040EC34
:104B300050E40CC00E945D9422E538EB4FE25BE349
:104B40000E94579626E636E64BE352E40E94C7924F
:104B50001BC00E949A6380918B3190918C31A091FF
:104B60008D31B0918E310196A11DB11D80938B3195
:104B700090938C31A0938D31B0938E310E945C2440
:104B800060EF7FEF89E794E40F900F900F90DF9133
:104B9000CF911F910F91FF90EF9008950F931F9366
:104BA000CF93DF93729A8091660283FF08C08EE4F0
:104BB0000E943D63811165C0C0E5D0E009C0C0E539
:104BC000D0E08FED97E00E946E0E2197D1F7EFCFE6
:104BD0008FED97E00E946E0E2197D1F78FE40E942F
:104BE0003D630E94B363D82FDF730E94B363082F25
:104BF0000E94B363C82F0E94BD63182F0E949A635E
:104C00008091660283FF72986D2F70E0762F662781
:104C1000600F711D80E090E00E945D9420E134E01F
:104C200048EC5BE30E94579660936D2970936E2960
:104C300080936F29909370296C2F70E0762F6627F0
:104C4000610F711D769567957695679580E090E088
:104C50000E945D9424EA3CEF44E25CE30E94579694
:104C600020E030E040E252E40E94C79260935A365E
:104C700070935B3680935C3690935D3680E090E075
:104C800002C081E090E0DF91CF911F910F910895D4
:104C90007298729A8EE40E943D6380EA0E94A26339
:104CA00080E00E94A26380E00E94A2638FE40E94E1
:104CB0003D630E94B3638EE40E943D6380E80E94DE
:104CC000A26380E00E94A26380E00E94A2630E942F
:104CD0009A6380E090E0089589E491E19F938F9337
:104CE0000E94D99B809180020F900F90882361F0E1
:104CF0001F928F9386E491E19F938F930E94D99B9B
:104D00000F900F900F900F90089581E291E19F9383
:104D10008F930E94D99B89EF90E19F938F930E947C
:104D2000D99B82ED90E19F938F930E94D99B87E955
:104D300090E19F938F930E94D99B8BE590E19F9385
:104D40008F930E94D99B89E290E19F938F930E9459
:104D5000D99B8DEE9FE09F938F930E94D99B87EC08
:104D60009FE09F938F930E94D99B81E99FE09F933F
:104D70008F930E94D99B8091792D90917A2D82708A
:104D800098702DB73EB72E5E3F4F0FB6F8943EBFDA
:104D90000FBE2DBF892B41F081E69FE09F938F933B
:104DA0000E94D99B0F900F9085E39FE09F938F9374
:104DB0000E94D99B89EF9EE09F938F930E94D99B7D
:104DC00080ED9EE09F938F930E94D99B84EA9EE0A2
:104DD0009F938F930E94D99B85E79EE09F938F932B
:104DE0000E94D99B83E49EE09F938F930E94D99B5E
:104DF00082E19EE09F938F930E94D99B88ED9DE076
:104E00009F938F930E94D99B82EA9DE09F938F93FB
:104E10000E94D99B82E79DE09F938F930E94D99B2C
:104E200086E49DE09F938F930E94D99B87E19DE04C
:104E30009F938F930E94D99B8EED9CE09F938F93BD
:104E40000E94D99B85EA9CE09F938F930E94D99BF7
:104E50008EE69CE09F938F930E94D99B80E49CE018
:104E60009F938F930E94D99B8DB79EB780960FB664
:104E7000F8949EBF0FBE8DBF8CE09CE09F938F93F4
:104E80000E94D99B8BED9BE09F938F930E94D99BAF
:104E90008CEA9BE09F938F930E94D99B8DE79BE0C8
:104EA0009F938F930E94D99B86E59BE09F938F935E
:104EB0000E94D99B80E29BE09F938F930E94D99B95
:104EC0008AEE9AE09F938F930E94D99B84EB9AE09D
:104ED0009F938F930E94D99B8BE89AE09F938F9327
:104EE0000E94D99B83E59AE09F938F930E94D99B60
:104EF00088E29AE09F938F930E94D99B2DB73EB78B
:104F00002A5E3F4F0FB6F8943EBF0FBE2DBF0895E7
:104F10008FED93E00C94019C4F925F926F927F9281
:104F20008F929F92AF92BF92CF92DF92EF92FF92B9
:104F3000CF93DF93CDB7DEB728970FB6F894DEBFD7
:104F40000FBECDBF80917F3190918031A091813192
:104F5000B091823189839A83AB83BC8340907F3147
:104F600050908031609081317090823180917F319A
:104F700090918031A0918131B09182318D839E8357
:104F8000AF83B88760917F3170918031809181319A
:104F9000909182312CE3822E912CA12CB12CA50171
:104FA00094010E9488907F936F9330E1C32E3EE07E
:104FB000D32EE12CF12C6D817E818F819885A70104
:104FC00096010E948890A50194010E9488903F93C9
:104FD0002F9340E8842E41E5942EAA24A394B12C6B
:104FE000C301B201A50194010E948890A701960116
:104FF0000E9488903F932F9369817A818B819C8155
:10500000A50194010E9488903F932F9382E09AE03B
:105010009F938F930E94D99B0FB6F894DEBF0FBE6B
:10502000CDBF28960FB6F894DEBF0FBECDBFDF917F
:10503000CF91FF90EF90DF90CF90BF90AF909F9077
:105040008F907F906F905F904F900895EDEBFAE313
:10505000808191818234924479F0ED5BFA43FF9331
:10506000EF9384EE99E09F938F930E94D99B0F90CA
:105070000F900F900F9008953A96E53F81E8F8075A
:1050800038F30895CF93DF93EC018C9A0E94E010DF
:105090009F938F937F936F9388ED99E09F938F9366
:1050A0000E94D99B0F900F900F900F900F900F9030
:1050B000209719F00E94F11108C086ED99E09F93A6
:1050C0008F930E94D99B0F900F9081E00E949210C5
:1050D000209185023091860240918702509188028A
:1050E0000E9457969F938F937F936F938AEC99E0DA
:1050F0009F938F930E94D99B0F900F900F900F90CA
:105100000F900F90209719F00E94F11108C088ECC1
:1051100099E09F938F930E94D99B0F900F9082E00C
:105120000E9492102091810230918202409183026C
:10513000509184020E9457969F938F937F936F9311
:105140008CEB99E09F938F930E94D99B0F900F90C7
:105150000F900F900F900F90209719F00E94F1116F
:1051600008C08AEB99E09F938F930E94D99B0F9080
:105170000F9083E00E9492109F938F937F936F9381
:105180008BEA99E09F938F930E94D99B8C980F9004
:105190000F900F900F900F900F90209719F00E9492
:1051A000F11108C089EA99E09F938F930E94D99BDF
:1051B0000F900F908091792D90917A2D92FF83C05E
:1051C00021E042E161E080ED0E9404659F938F93AE
:1051D0007F936F938CE999E09F938F930E94D99B63
:1051E0000F900F900F900F900F900F90209719F045
:1051F0000E94F11108C08AE999E09F938F930E9461
:10520000D99B0F900F9021E042E162E080ED0E9477
:1052100004659F938F937F936F938DE899E09F939D
:105220008F930E94D99B0F900F900F900F900F902B
:105230000F90209719F00E94F11108C08BE899E0B7
:105240009F938F930E94D99B0F900F9021E042E192
:1052500063E080ED0E9404659F938F937F936F932B
:105260008EE799E09F938F930E94D99B0F900F90A8
:105270000F900F900F900F90CD2B19F00E94F1110D
:1052800008C08CE799E09F938F930E94D99B0F9061
:105290000F9021E042E164E080ED0E9404659F935D
:1052A0008F937F936F938FE699E09F938F930E94E4
:1052B000D99B0F900F900F900F900F900F90DF9150
:1052C000CF910C94F111CD2BD1F3DF91CF910895B3
:1052D0000F931F93CF93DF93882389F049E050E029
:1052E0006FEF70E082E496E30E94139B49E050E088
:1052F0006EE070E082E496E30E94A49E13C0C2E4D4
:10530000D6E30AE619E089911F928F931F930F93BA
:105310000E94D99B0F900F900F900F9086E3CA3494
:10532000D80789F7DF91CF911F910F910C94F1115C
:10533000882311F0299A089529980895882311F057
:105340002A9A08952A980895CF92DF92EF92FF92B9
:10535000CF93DF936B017C0160FF11C08CE194E07F
:105360009F938F938EE591E19F938F930E94D99B9A
:105370000F900F900F900F9081E090E002C080E0BE
:1053800090E0C1FE09C0EC01219646EB59E061E2D4
:1053900074E00E945A16CE01C2FE09C0EC012196AB
:1053A00046EB59E069E274E00E945A16CE01C3FE52
:1053B00009C0EC01219646EB59E061E374E00E94DC
:1053C0005A16CE01C4FE09C0EC01219646EB59E005
:1053D0006DEB75E00E945A16CE01C5FE09C0EC01C6
:1053E000219646EB59E065E374E00E945A16CE011F
:1053F000C6FE09C0EC01219646EB59E069E374E072
:105400000E945A16CE01C7FE09C0EC01219646EB58
:1054100059E06FE374E00E945A16CE01D0FE09C035
:10542000EC01219646EB59E067E474E00E945A16BD
:10543000CE01D1FE09C0EC01219646EB59E06FE4A4
:1054400074E00E945A16CE01D2FE09C0EC012196EA
:1054500046EB59E063E574E00E945A16CE012091B4
:10546000792D30917A2D24703071232B59F0D3FE91
:1054700009C0EC01219646EB59E069E574E00E9411
:105480005A16CE012091792D26FF0BC0D4FE09C0FB
:10549000EC01219646EB59E06EE574E00E945A1645
:1054A000CE012091792D27FF0BC0D5FE09C0EC015C
:1054B000219646EB59E064E674E00E945A16CE014C
:1054C000D6FE09C0EC01219646EB59E06CE674E08B
:1054D0000E945A16CE01D7FE09C0EC01219646EB78
:1054E00059E067E774E00E945A16CE01E0FE0CC056
:1054F00046EB59E068E874E0DF91CF91FF90EF90C0
:10550000DF90CF900C945A16CD28CE28CF2841F4A6
:1055100085E699E09F938F930E94D99B0F900F90FF
:10552000DF91CF91FF90EF90DF90CF900895CF92D1
:10553000DF92EF92FF92CF93DF93EC01C12CD12C3D
:105540007601209709F4A3C060E679E0CE010E94BD
:10555000E59A892B11F46894C0F868E579E0CE01EA
:105560000E94E59A892B11F46894C1F860E579E00E
:10557000CE010E94E59A892B11F46894C2F86CE47C
:1055800079E0CE010E94E59A892B11F46894C3F862
:1055900069E479E0CE010E94E59A892B11F46894C0
:1055A000C4F865E479E0CE010E94E59A892B11F4F4
:1055B0006894C5F86FE379E0CE010E94E59A892BE3
:1055C00011F46894C6F867E379E0CE010E94E59A89
:1055D000892B11F46894C7F86FE279E0CE010E943C
:1055E000E59A892B11F46894D0F86BE279E0CE014A
:1055F0000E94E59A892B11F46894D1F865E279E06C
:10560000CE010E94E59A892B11F46894D2F860E2E9
:1056100079E0CE010E94E59A892B11F46894D3F8C1
:105620006AE179E0CE010E94E59A892B11F4689431
:10563000D4F862E179E0CE010E94E59A892B11F459
:105640006894D5F867E079E0CE010E94E59A892B4D
:1056500011F46894D6F866EF78E0CE010E94E59ADE
:10566000892B11F46894D7F861EF78E0CE010E949D
:10567000E59A892B11F46894E0F860917E027091AC
:105680007F0280E090E00E94F99AEC015ACFC701B6
:10569000B601DF91CF91FF90EF90DF90CF9008950A
:1056A000AF92BF92CF92DF92EF92FF920F931F9330
:1056B000CF93DF93D22FC32F8A01F62EC72ED82E79
:1056C000E92E217030E040E050E060E070E080E0E2
:1056D00090E0A0E00E94BB9289F08DE894E09F9357
:1056E0008F938EE591E19F938F930E94D99B0F90AA
:1056F0000F900F900F90E1E0F0E002C0E0E0F0E0EA
:105700008091792D80FF19C02D2F247030E040E06A
:1057100050E060E070E080E090E0A0E00E94BB928A
:1057200061F05F018FEFA81AB80A46EB59E061E912
:1057300074E0CF010E945A16F5012D2F227030E03F
:1057400040E050E060E070E080E090E0A0E00E9487
:10575000BB9261F05F018FEFA81AB80A46EB59E0DF
:1057600065E974E0CF010E945A16F5012D2F2870CB
:1057700030E040E050E060E070E080E090E0A0E0E9
:105780000E94BB9261F05F018FEFA81AB80A46EB46
:1057900059E06DEA74E0CF010E945A16F5012D2FF1
:1057A000207130E040E050E060E070E080E090E0A8
:1057B000A0E00E94BB9261F05F018FEFA81AB80AC7
:1057C00046EB59E068E974E0CF010E945A16F501F2
:1057D0002D2F207230E040E050E060E070E080E08B
:1057E00090E0A0E00E94BB9261F05F018FEFA81AE9
:1057F000B80A46EB59E06BE974E0CF010E945A16F3
:10580000F5012D2F207430E040E050E060E070E0C2
:1058100080E090E0A0E00E94BB9261F05F018FEF1A
:10582000A81AB80A46EB59E061EA74E0CF010E9479
:105830005A16F5012D2F207830E040E050E060E06E
:1058400070E080E090E0A0E00E94BB9261F05F0118
:105850008FEFA81AB80A46EB59E067EA74E0CF0167
:105860000E945A16F50120E03C2F317040E050E0D4
:1058700060E070E080E090E0A0E00E94BB9261F008
:105880005F018FEFA81AB80A46EB59E06AEA74E0A4
:10589000CF010E945A16F50120E03C2F327040E003
:1058A00050E060E070E080E090E0A0E00E94BB92F9
:1058B00061F05F018FEFA81AB80A46EB59E06FEA72
:1058C00074E0CF010E945A16F50120E03C2F34709D
:1058D00040E050E060E070E080E090E0A0E00E94F6
:1058E000BB9261F05F018FEFA81AB80A46EB59E04E
:1058F00066EB74E0CF010E945A16F50120E03C2FC0
:10590000387040E050E060E070E080E090E0A0E0BF
:105910000E94BB9261F05F018FEFA81AB80A46EBB4
:1059200059E069EB74E0CF010E945A16F50120E0BE
:105930003C2F307140E050E060E070E080E090E0AB
:10594000A0E00E94BB9261F05F018FEFA81AB80A35
:1059500046EB59E06EEB74E0CF010E945A16F50158
:1059600020E03C2F307240E050E060E070E080E0EA
:1059700090E0A0E00E94BB9261F05F018FEFA81A57
:10598000B80A46EB59E065EC74E0CF010E945A1664
:10599000F50120E030E040E050E06F2D647070E0F1
:1059A00080E090E0A0E00E94BB9261F05F018FEF89
:1059B000A81AB80A46EB59E06CEC74E0CF010E94DB
:1059C0005A16F5018091792D81FF19C020E03C2FF6
:1059D000307440E050E060E070E080E090E0A0E0F3
:1059E0000E94BB9261F05F018FEFA81AB80A46EBE4
:1059F00059E060ED74E0CF010E945A16F5018091E4
:105A0000792D90917A2D93FF19C020E030E040E08D
:105A1000512F507160E070E080E090E0A0E00E94C3
:105A2000BB9261F05F018FEFA81AB80A46EB59E00C
:105A300063ED74E0CF010E945A16F5018091792D33
:105A400090917A2D93FF19C020E030E040E0512F73
:105A5000507260E070E080E090E0A0E00E94BB92B5
:105A600061F05F018FEFA81AB80A46EB59E066EDC6
:105A700074E0CF010E945A16F5018091792D909122
:105A80007A2D93FF19C020E030E040E0512F507490
:105A900060E070E080E090E0A0E00E94BB9261F0E6
:105AA0005F018FEFA81AB80A46EB59E06CED74E07D
:105AB000CF010E945A16F50120E03C2F307840E0DB
:105AC00050E060E070E080E090E0A0E00E94BB92D7
:105AD00061F05F018FEFA81AB80A46EB59E067EE54
:105AE00074E0CF010E945A16F50120E030E0402F0B
:105AF000417050E060E070E080E090E0A0E00E9443
:105B0000BB9261F05F018FEFA81AB80A46EB59E02B
:105B10006CEE74E0CF010E945A16F50120E030E0EF
:105B2000402F427050E060E070E080E090E0A0E044
:105B30000E94BB9261F05F018FEFA81AB80A46EB92
:105B400059E06FEE74E0CF010E945A16F50120E093
:105B500030E040E050E06F2D687070E080E090E051
:105B6000A0E00E94BB9261F05F018FEFA81AB80A13
:105B700046EB59E062EF74E0CF010E945A16F5013E
:105B800020E030E040E050E06F2D607170E080E098
:105B900090E0A0E00E94BB9261F05F018FEFA81A35
:105BA000B80A46EB59E066EF74E0CF010E945A163E
:105BB000F5018091792D90917A2D92FF19C020E006
:105BC00030E0402F487050E060E070E080E090E00E
:105BD000A0E00E94BB9261F05F018FEFA81AB80AA3
:105BE00046EB59E06AEF74E0CF010E945A16F501C6
:105BF0008091792D90917A2D92FF19C020E030E0AC
:105C0000402F407150E060E070E080E090E0A0E064
:105C10000E94BB9261F05F018FEFA81AB80A46EBB1
:105C200059E06EEF74E0CF010E945A16F5018091A1
:105C3000792D90917A2D92FF19C020E030E0402F0D
:105C4000407250E060E070E080E090E0A0E00E94F0
:105C5000BB9261F05F018FEFA81AB80A46EB59E0DA
:105C600062E075E0CF010E945A16F5018091792D0E
:105C700090917A2D92FF19C020E030E0402F4074BF
:105C800050E060E070E080E090E0A0E00E94BB9215
:105C900061F05F018FEFA81AB80A46EB59E066E0A1
:105CA00075E0CF010E945A16F5018091792D82FF8F
:105CB00019C020E030E0402F407850E060E070E014
:105CC00080E090E0A0E00E94BB9261F05F018FEF66
:105CD000A81AB80A46EB59E060E576E0CF010E94C9
:105CE0005A16F5018091792D82FF19C020E030E02D
:105CF00040E0512F517060E070E080E090E0A0E063
:105D00000E94BB9261F05F018FEFA81AB80A46EBC0
:105D100059E06AE075E0CF010E945A16F5018091C2
:105D2000792D90917A2D93FF19C020E030E040E06A
:105D3000512F527060E070E080E090E0A0E00E949F
:105D4000BB9261F05F018FEFA81AB80A46EB59E0E9
:105D50006DE075E0CF010E945A16F5018091792D12
:105D600090917A2D93FF19C020E030E040E0512F50
:105D7000547060E070E080E090E0A0E00E94BB9290
:105D800061F05F018FEFA81AB80A46EB59E065E1B0
:105D900075E0CF010E945A16F5018091792D9091FE
:105DA0007A2D94FF19C020E030E040E0512F587068
:105DB00060E070E080E090E0A0E00E94BB9261F0C3
:105DC0005F018FEFA81AB80A46EB59E06EE175E063
:105DD000CF010E945A16F5018091792D85FF19C0D7
:105DE00020E030E040E050E06F2D607270E080E035
:105DF00090E0A0E00E94BB9261F05F018FEFA81AD3
:105E0000B80A46EB59E067E275E0CF010E945A16E6
:105E1000F5018091792D85FF19C020E030E040E048
:105E200050E06F2D607470E080E090E0A0E00E9490
:105E3000BB9261F05F018FEFA81AB80A46EB59E0F8
:105E400060E375E0CF010E945A16F5018091792D2B
:105E500085FF1EC020E030E040E050E06F2D60780C
:105E600070E080E090E0A0E00E94BB9289F046EBF9
:105E700059E06AE375E0CF01DF91CF911F910F9157
:105E8000FF90EF90DF90CF90BF90AF900C945A1698
:105E90002D2F3C2FA8016F2D7C2D8D2D9E2DA0E048
:105EA0000E94BB9241F48CEE98E09F938F930E94E6
:105EB000D99B0F900F90DF91CF911F910F91FF9081
:105EC000EF90DF90CF90BF90AF900895AF92BF92C8
:105ED000DF92EF92FF920F931F93CF93DF93EC012A
:105EE0005B01FB01108267EE78E00E94E59A892B46
:105EF00089F58091792D1DE440E8F42E82FF03C0DE
:105F000034E8E32E02C024E0E22E00E0D12C81FF31
:105F100002C090ECF92E26E04AE250E06BE270E01D
:105F200089E290E00E94E26081E090E00E948911A5
:105F300081111DE58091792D90917A2D93FF02C0FA
:105F4000177F06E094FD086085FF09C0177F80EE8B
:105F5000D82E05C010E0F12CE12C00E0D12C65EE2C
:105F600078E0CE010E94E59A892B61F481E0F50189
:105F7000808360917E0270917F0280E090E00E94B9
:105F8000F99AEC0163EE78E0CE010E94E59A892B44
:105F900061F48FEFF501808360917E0270917F0242
:105FA00080E090E00E94F99AEC01209709F456C134
:105FB0006FED78E0CE010E94E59A892B09F411601B
:105FC0006BED78E0CE010E94E59A892B09F414600C
:105FD00068ED78E0CE010E94E59A892B09F4126001
:105FE00066ED78E0CE010E94E59A892B09F41860ED
:105FF00063ED78E0CE010E94E59A892B09F41061E7
:106000006DEC78E0CE010E94E59A892B09F41062CC
:1060100067EC78E0CE010E94E59A892B09F41064C0
:1060200064EC78E0CE010E94E59A892B09F41068AF
:106030006FEB78E0CE010E94E59A892B19F4FF2DD1
:10604000F160FF2E68EB78E0CE010E94E59A892B83
:1060500019F48F2D8260F82E65EB78E0CE010E9456
:10606000E59A892B19F4EF2DE460FE2E60EB78E0C1
:10607000CE010E94E59A892B19F4FF2DF860FF2EBE
:1060800069EA78E0CE010E94E59A892B19F48F2DF8
:106090008061F82E62EA78E0CE010E94E59A892BB1
:1060A00019F4EF2DE062FE2E6EE978E0CE010E9439
:1060B000E59A892B19F4FD2DF460DF2E6BE978E069
:1060C000CE010E94E59A892B19F48F2D8064F82E59
:1060D00066E978E0CE010E94E59A892B19F4EF2D4C
:1060E000E068FE2E63E978E0CE010E94E59A892BF4
:1060F00019F4FE2DF160EF2E60E978E0CE010E94E8
:10610000E59A892B19F48E2D8260E82E6DE878E0EF
:10611000CE010E94E59A892B19F4EE2DE460EE2E53
:1061200069E878E0CE010E94E59A892B19F4FE2DEA
:10613000F860EF2E65E878E0CE010E94E59A892BA1
:1061400019F48E2D8061E82E61E878E0CE010E947E
:10615000E59A892B19F4EE2DE062EE2E6DE778E0DA
:10616000CE010E94E59A892B19F4FE2DF064EF2EE2
:106170006BE778E0CE010E94E59A892B19F48E2D09
:106180008068E82E68E778E0CE010E94E59A892BC6
:1061900009F4016060E778E0CE010E94E59A892B5E
:1061A00009F4026067E678E0CE010E94E59A892B47
:1061B00009F404606EE578E0CE010E94E59A892B2F
:1061C00009F408606BE578E0CE010E94E59A892B1E
:1061D00009F4006165E578E0CE010E94E59A892B1B
:1061E00009F400626AE478E0CE010E94E59A892B06
:1061F00009F4006466E478E0CE010E94E59A892BF8
:1062000019F4ED2DE860DE2E62E478E0CE010E9404
:10621000E59A892B19F4FD2DF061DF2E69E378E012
:10622000CE010E94E59A892B19F48D2D8062D82E1B
:106230006FE278E0CE010E94E59A892B19F4ED2DEA
:10624000E064DE2E66E278E0CE010E94E59A892BBA
:1062500009F0A2CEFD2DF068DF2E9ECE212F3F2D1E
:106260004E2D502F6D2D70E080E090E0DF91CF91AA
:106270001F910F91FF90EF90DF90BF90AF90089526
:106280005F926F927F928F929F92AF92BF92CF92C6
:10629000DF92EF92FF920F931F93CF93DF93782EAD
:1062A000CCE5DDE100E010E080E2E82E88E0F82EA9
:1062B000872D8170582E872D8270682E9BE0C92E05
:1062C00098E0D92E23E1A22E28E0B22E31E1832ED0
:1062D00038E0932E772051F01F930F93FF92EF92A7
:1062E0000E94D99B0F900F900F900F905520A1F016
:1062F00089858F9388858F93BF92AF920E94D99B97
:106300000F900F900F900F906620C1F09F928F9288
:106310000E94D99B0F900F90662081F0DF92CF9260
:106320000E94D99B288139814A815B816C817D8162
:106330008E819F810E94502B0F900F900E94F1112F
:106340000F5F1F4F2A960430110521F6DF91CF9180
:106350001F910F91FF90EF90DF90CF90BF90AF9083
:106360009F908F907F906F905F90089586E098E067
:106370009F938F930E94D99B8091692990916A295C
:10638000A0916B29B0916C290F900F90813027EA72
:1063900092072EE1A207B10519F488EF97E01DC01E
:1063A000823026EA92072EE1A207B10519F48BEE9E
:1063B00097E013C0823027EA92072EE1A207B105C9
:1063C00019F48DED97E009C0823028EA92072EE19A
:1063D000A207B10549F48FEC97E09F938F930E9439
:1063E000D99B0F900F900895BF93AF939F938F9376
:1063F00089EC97E09F938F930E94D99B0F900F9009
:106400000F900F900F900F90089589EB97E09F9356
:106410008F930E94D99B0E9488270E94B6310E94C8
:10642000F11183E49DE19F938F9381EB97E09F931C
:106430008F930E94D99B609160027091610280915C
:1064400062029091630228EE33E040E050E00E9447
:1064500088905F934F933F932F9381EA97E09F93A8
:106460008F930E94D99B88E997E09F938F930E9416
:10647000D99B0E94E5168091792D2DB73EB7225FFA
:106480003F4F0FB6F8943EBF0FBE2DBF80FF05C033
:1064900041E061E081E00E94BB1884E997E09F93AE
:1064A0008F930E94D99B80E00E9468290E948C27CC
:1064B000809165021F928F938BE897E09F938F9353
:1064C0000E94D99B80912A141F928F9382E897E0B3
:1064D0009F938F930E94D99B809190028F9380917C
:1064E0008F028F9380918E028F9380918D028F9374
:1064F00084E797E09F938F930E94D99B1F9280E43B
:106500008F938CE597E09F938F930E94D99B809106
:1065100064381F928F93809163381F928F9389E420
:1065200097E09F938F930E94D99B809164021F9262
:106530008F9380E497E09F938F930E94D99B8091E3
:10654000660290916702A0916802B09169022DB72E
:106550003EB7225E3F4F0FB6F8943EBF0FBE2DBF31
:1065600096FD03C086E495E002C083E495E09F9326
:106570008F9386E397E09F938F930E94D99B83E04C
:106580000E9440310F900F900F900F901D9903C003
:1065900086E495E002C083E495E09F938F938AE2BE
:1065A00097E09F938F930E94D99B80E297E09F93FF
:1065B0008F930E94D99B809166020F900F900F904D
:1065C0000F900F900F9081FF09C08AE197E09F9391
:1065D0008F930E94D99B0F900F9013C080FD03C032
:1065E00086E495E002C083E495E09F938F9386E173
:1065F00097E09F938F930E94D99B0F900F900F90DD
:106600000F908091660290916702A0916802B0910C
:10661000690297FD03C086E495E002C083E495E03B
:106620009F938F938DE097E09F938F930E94D99BC8
:1066300086E097E09F938F930E94D99B60912D14E1
:1066400070912E1480912F14909130140E94A429DF
:106650000E94F1110F900F900F900F900F900F90DC
:10666000779B03C086E495E002C083E495E09F93A6
:106670008F938DEF96E09F938F930E94D99B0E94FA
:10668000740E0E9445119F938F937F936F938FEEAB
:1066900096E09F938F930E94D99B0E94F4109F9342
:1066A0008F937F936F9381EE96E09F938F930E94D9
:1066B000D99B81E090E00E944228809128369091F9
:1066C0002936A0912A36B0912B36BF93AF939F9372
:1066D0008F9383ED96E09F938F930E94D99B809137
:1066E0003D368F9380913C368F9380913B368F93CC
:1066F00080913A368F938FEB96E09F938F930E9411
:10670000D99B80912C3690912D36A0912E36B09148
:106710002F36BF93AF939F938F9381EB96E09F9318
:106720008F930E94D99B8DB79EB782960FB6F8942F
:106730009EBF0FBE8DBF809141368F9380914036B2
:106740008F9380913F368F9380913E368F938DE962
:1067500096E09F938F930E94D99B61E070E080E068
:1067600090E00E94FA1161E070E081E090E00E9408
:10677000FA110F900F900F900F900F900F90299992
:1067800003C086E495E002C083E495E09F938F9375
:1067900085E996E09F938F930E94D99B0F900F906D
:1067A0000F900F902A9903C086E495E002C083E41D
:1067B00095E09F938F938DE896E09F938F930E942F
:1067C000D99B8091660290916702A0916802B09176
:1067D00069020F900F900F900F9094FD03C086E414
:1067E00095E002C083E495E09F938F9385E896E05F
:1067F0009F938F930E94D99B0F900F900F900F90B3
:106800000895F89491E2E0E0F0E0909357008491CD
:10681000E2E0F0E0909357002491E4E0F0E0909300
:106820005700E49190E0A0E0B0E0BC015527442778
:10683000822F90E0A0E0B0E0BA2FA92F982F8827F0
:10684000840F951FA61FB71F8E0F911DA11DB11D8F
:106850008093692990936A29A0936B29B0936C293E
:1068600078940895CF93DF93CDB7DEB761970FB6D5
:10687000F894DEBF0FBECDBF48E250E062E270E0A8
:106880008CE59DE10E94869E20915C1D30915D1DEE
:1068900040915E1D50915F1D6091601D7091611D62
:1068A0008091621D9091631DAFEF0E94BB9209F031
:1068B0005DC08DE480935C1D80E880935D1D84E065
:1068C00080935E1D10925F1D1092601D1092611DDD
:1068D0001092621D1092631D8CE390E09093651DF1
:1068E0008093641D1092661D1092671D1092681DA2
:1068F0001092691D10926A1D10926B1D10926C1DF2
:1069000010926D1D10926F1D10926E1D1092701DD1
:106910001092711D1092721D1092731D1092741DB1
:106920001092751D1092761D1092771D1092791D90
:106930001092781D10927A1D10927B1D10927C1D72
:1069400010927D1D10927E1D10927F1D1092801D51
:106950001092811D1092831D1092821D48E250E01A
:1069600062E270E08CE59DE10E94A49E44E050E06C
:106970006EE170E0CE010B960E94869E8B859C8511
:10698000AD85BE858F3F2FEF9207A207B207A9F40E
:106990008AE090E4A0E0B0E0809366029093670202
:1069A000A0936802B093690244E050E06EE170E0A9
:1069B00086E692E00E94A49E08C0809366029093AF
:1069C0006702A0936802B093690280916602909179
:1069D0006702A0916802B0916902A2FF02C02A9AE0
:1069E00003C080E00E949E2944E050E06AE570E028
:1069F000CE010B960E94869E8B859C85AD85BE85BB
:106A00008F3F2FEF9207A207B20789F410922D143F
:106A100010922E1410922F141092301444E050E073
:106A20006AE570E08DE294E10E94A49E08C0809324
:106A30002D1490932E14A0932F14B093301449E08A
:106A400050E06EE070E082E496E30E94869E0E9431
:106A5000281344E050E06EE470E0CE010B960E94F3
:106A6000869E8B859C85AD85BE8544E050E06EE4B6
:106A700070E08F3F9F4FAF4FBF4F29F485E892E002
:106A80000E94A49E04C085E892E00E94869E44E095
:106A900050E06AE470E0CE010B960E94869E8B85E2
:106AA0009C85AD85BE8544E050E06AE470E08F3F90
:106AB0009F4FAF4FBF4F29F481E892E00E94A49E00
:106AC00004C081E892E00E94869E44E050E062E5C6
:106AD00070E0CE010B960E94869E8B859C85AD85CD
:106AE000BE8544E050E062E570E08F3F9F4FAF4FBE
:106AF000BF4F29F489E892E00E94A49E04C089E86F
:106B000092E00E94869E41E050E06DE170E0CE018F
:106B100041960E94869E898941E050E06DE170E0D7
:106B20008F3F29F48AE294E10E94A49E04C08AE285
:106B300094E10E94869E41E050E06CE170E0CE015D
:106B400041960E94869E898941E050E06CE170E0A8
:106B50008F3F29F485E692E00E94A49E04C085E65A
:106B600092E00E94869E41E050E06BE170E0CE0131
:106B700041960E94869E898941E050E06BE170E079
:106B80008F3F29F484E692E00E94A49E04C084E62C
:106B900092E00E94869E4AE050E064E070E0CE0100
:106BA00001960E94869E89814AE050E064E070E090
:106BB0008F3F29F483E49DE10E94A49E04C083E4F6
:106BC0009DE10E94869E44E050E066E570E0CE01C3
:106BD0000B960E94869E8B859C85AD85BE8544E084
:106BE00050E066E570E08F3F9F4FAF4FBF4F29F4F5
:106BF0008DE892E00E94A49E04C08DE892E00E947D
:106C0000869E44E050E067E170E0CE010B960E9462
:106C1000869E8B859C85AD85BE8544E050E067E10E
:106C200070E08F3F9F4FAF4FBF4F29F480E692E057
:106C30000E94A49E04C080E692E00E94869E8091FD
:106C4000600290916102A0916202B091630281386A
:106C50009A41A640B105A0F083EF92E09F938F93F5
:106C60000E94D99B80E197E2A0E0B0E080936002AF
:106C700090936102A0936202B09363020F900F9011
:106C80006091600270916102809162029091630252
:106C90000E94276342E050E062E070E0CE010F9670
:106CA0000E94869E8F85988942E050E062E070E005
:106CB0008F3F910529F483E294E10E94A49E04C0D1
:106CC00083E294E10E94869E42E050E060E070E042
:106CD000CE010F960E94869E8F85988942E050E0F3
:106CE00060E070E08F3F910529F481E294E10E9419
:106CF000A49E04C081E294E10E94869E61960FB634
:106D0000F894DEBF0FBECDBFDF91CF910895CF9233
:106D1000DF92EF92FF9260917E0270917F0280E09D
:106D200090E00E94F99A6AE475E00E941A9B892B10
:106D300009F03BC18DE480935C1D80E880935D1D6C
:106D400084E080935E1D10925F1D1092601D109272
:106D5000611D1092621D1092631D8CE390E0909370
:106D6000651D8093641D1092661D1092671D109220
:106D7000681D1092691D10926A1D10926B1D109271
:106D80006C1D10926D1D10926F1D10926E1D109251
:106D9000701D1092711D1092721D1092731D109231
:106DA000741D1092751D1092761D1092771D109211
:106DB000791D1092781D10927A1D10927B1D1092F1
:106DC0007C1D10927D1D10927E1D10927F1D1092D1
:106DD000801D1092811D1092831D1092821D48E229
:106DE00050E062E270E08CE59DE10E94A49E8AE0A2
:106DF00090E4A0E0B0E08093660290936702A093D5
:106E00006802B093690244E050E06EE170E086E60B
:106E100092E00E94A49E10922D1410922E141092B3
:106E20002F141092301444E050E06AE570E08DE2D7
:106E300094E10E94A49E82E2C82EDD24DA948CECB8
:106E4000E82E8BE3F82EC0928502D0928602E09263
:106E50008702F092880244E050E06EE470E085E83A
:106E600092E00E94A49EC0928102D0928202E0929F
:106E70008302F092840244E050E06AE470E081E82A
:106E800092E00E94A49E87ED94E3AFEEBCE3809372
:106E9000890290938A02A0938B02B0938C0244E003
:106EA00050E062E570E089E892E00E94A49E8AE9E1
:106EB00099E9A9E1B0E480938D0290938E02A093AA
:106EC0008F02B093900244E050E066E570E08DE8F8
:106ED00092E00E94A49E10922A1480E00E94976D76
:106EE00041E050E06DE170E08AE294E10E94A49EEE
:106EF0008AE1809365020E94706C41E050E06CE191
:106F000070E085E692E00E94A49E8FE08093640288
:106F100041E050E06BE170E084E692E00E94A49EC4
:106F20008AE0E3E4FDE1DF011D928A95E9F74AE09A
:106F300050E064E070E0CF010E94A49E80E197E2FF
:106F4000A0E0B0E08093600290936102A09362029F
:106F5000B093630244E050E067E170E080E692E0C5
:106F60000E94A49E109224141092231442E050E038
:106F700062E070E083E294E10E94A49E10922214E9
:106F80001092211442E050E060E070E081E294E170
:106F90000E94A49E81E00E94682980E090E0FF901A
:106FA000EF90DF90CF900C943D13FF90EF90DF9027
:106FB000CF9008950E948E696C9A6B9A6A9A6F9A24
:106FC000729A749A739A779A809880B3897F80BBFB
:106FD0008398849887E080937E00549A0E940134BD
:106FE0000E9432348091660290916702A0916802FB
:106FF000B091690294FD0E949D690E94E20E80E0BA
:1070000090E00E943D136091600270916102809156
:107010006202909163020E9427630E94F4106093C1
:107020007B3170937C3180937D3190937E31809160
:10703000660286FD239A219A229A239A0E94F70ECD
:107040001D9B05C010922C1410922B14089581E002
:1070500090E090932C1480932B140895CF93DF939A
:1070600090E040912D1450912E1460912F14709146
:10707000301441FD08C02091660220FD04C021FFAC
:107080008CC01D9B8AC02DE8289FE001299FD00D50
:107090001124CE018759914E9F938F9381E595E0FE
:1070A0009F938F930E94C59BFE01EE59F14EDF0125
:1070B000AA57BF4F2C910F900F900F900F904381C4
:1070C00054816581768180917F3190918031A0914A
:1070D0008131B0918231841B950BA60BB70B222313
:1070E000D1F1BF93AF939F938F93DF01A257BF4F0F
:1070F00011968C9111978F938C918F931297119673
:107100008C9111978F938C918F9313978C911F92E1
:107110008F9311978C911F928F9313968C911F923E
:107120008F9311978C911F928F93E957FF4F808116
:107130001F928F931F922F9387E595E09F938F93D4
:107140000E94C59B8DB79EB746960FB6F8949EBF1A
:107150000FBE8DBF10C0BF93AF939F938F938EE9E7
:1071600095E09F938F930E94C59B0F900F900F9077
:107170000F900F900F900E94F11180918002882350
:1071800061F01F928F9380EF92E09F938F930E9404
:10719000D99B0F900F900F900F90DF91CF91089592
:1071A0008091621E882341F08091631E90E00E94CE
:1071B0002E380E94E80FF4CF0895CF93DF93EC01AF
:1071C0008881998183332FE09207F1F018F4892B9D
:1071D000C1F04BC08B332FE0920709F44CC08F33C2
:1071E0009F4009F042C084EE9AE00E94D571892B3D
:1071F00009F43FC084EE9AE00E94C17180E00E94D1
:10720000982983E39FE02EC0623199F5299A409135
:107210002114509122145695542F44275795479581
:1072200060E070E084EE9AE00E94B77180912D14C6
:1072300090912E14A0912F14B0913014A0FF10C083
:10724000809122148F93809121148F9383E092E197
:107250009F938F930E94D99B0F900F900F900F9048
:107260008BE39FE09983888304C01982188283E0AE
:1072700019C081E017C084EE9AE00E94D571892B75
:10728000C1F384EE9AE00E94C1710E94D03840E2BE
:1072900050E060E070E084EE9AE00E94B7718FE306
:1072A0009FE0E0CFDF91CF9108952F923F924F92D0
:1072B0005F926F927F928F929F92AF92BF92CF9286
:1072C000DF92EF92FF920F931F93CF93DF93CDB78F
:1072D000DEB72B970FB6F894DEBF0FBECDBF9B87EE
:1072E0008A873A01FC0180819181892B11F00C94ED
:1072F000FF4D60917E0270917F02CA010E94F99A4F
:1073000060E870E0C3010E94399B009759F46091D6
:10731000B73A7091B83A8AE090E00E948D9B81E084
:107320000C94044E8130910561F4F3011081912E8B
:10733000990C9908892C092D292C392C492C592C68
:10734000B9C082309105B9F4F3018081082E000C98
:10735000990B982F88272181820F911D27FD9A95DF
:10736000182F992E892E880C8808082D282C382C47
:10737000482C582C9FC083309105B1F5F301208132
:10738000922F990F990B392F492F592F692F792F48
:10739000892F00E10E945D9219012A014B01B82F4B
:1073A000A92F2181922F990F990B392F492F592FEE
:1073B000692F792F892F08E00E945D9259016A0197
:1073C0007B018C019101A201B4018B2F9A2F0E94A5
:1073D0009492A2801A2D110F110BB12EC12ED12E15
:1073E000E12EF12E012F55C004970CF45BC0F30180
:1073F0002081922F990F990B392F492F592F692FDF
:10740000792F892F08E10E945D9219012A014B0111
:10741000B82FA92F2181922F990F990B392F492F1E
:10742000592F692F792F892F00E10E945D92590110
:107430006A017B018C019101A201B4018B2F9A2F6B
:107440000E949492A3801A2D110F110BB12EC12E00
:10745000D12EE12EF12E012F0E94949219012A01C2
:107460004B01B82FA92F2281922F990F990B392FF9
:10747000492F592F692F792F892F08E00E945D929B
:1074800059016A017B018C019101A201B4018B2F8A
:107490009A2F0E949492122F932E842E052F1B0157
:1074A0002C0108C01AE0912C812C00E0212C312CF9
:1074B000412C512C0E94F111212F392D482D502F94
:1074C000B101C2012537F3E63F07FDE64F0751053D
:1074D000610571058105910511F40C946E482537FD
:1074E000E3E63E07EDE64E075105610571058105AE
:1074F000910511F008F0B2C12337F2E73F074105CB
:107500005105610571058105910511F40C94074B36
:107510002337E2E73E074105510561057105810505
:10752000910511F008F0B9C02536F4E63F07410592
:107530005105610571058105910509F4D1C725360D
:10754000E4E63E0741055105610571058105910598
:1075500011F008F041C0A6E70E94BB9211F40C9410
:10756000F2440E94BB9209F070F4A8E60E94BB921C
:1075700011F40C94C142A5E70E94BB9211F40C9443
:10758000DC440C94FD4D212F392D482D502FB10195
:10759000C2012436F1E63F07410551056105710539
:1075A0008105910511F40C942F4B2537E2E63E0737
:1075B00041055105610571058105910509F431C544
:1075C0002A33364241055105610571058105910552
:1075D00009F430C30C94FD4D212F392D482D502F27
:1075E000B101C2012737EFE63E07410551056105AC
:1075F00071058105910511F40C94D4482737FFE6F5
:107600003F0741055105610571058105910509F0A7
:10761000C8F42436E9E63E074105510561057105C8
:107620008105910511F40C94B54425363E4641057B
:107630005105610571058105910511F40C94084906
:107640000C94FD4D212F392D482D502FB101C20131
:107650002536E2E73E0741055105610571058105C3
:10766000910511F40C94D4492936F2E73F074105FE
:107670005105610571058105910511F40C94B64A17
:107680002333314741055105610571058105910598
:1076900011F00C94FD4D0C942F4B212F392D482DBA
:1076A000502FB101C2012236F5E63F07F4E64F073D
:1076B0005105610571058105910509F411C722364F
:1076C000E5E63E07E4E64E075105610571058105D3
:1076D000910511F008F05BC02133F4E63F07F1E6B5
:1076E0004F075105610571058105910509F4B6C281
:1076F0002133E4E63E07E1E64E07510561057105D9
:107700008105910509F0C0F42337F3E73F074105F0
:107710005105610571058105910511F40C941B4B10
:1077200028373447410551056105710581059105EB
:1077300009F480C20C94FD4D212F392D482D502F76
:10774000B101C2012837F4E63F07F1E64F075105C2
:10775000610571058105910509F47CC22C36E5E7C8
:107760003E07E2E64E075105610571058105910569
:1077700009F457C423363446414651056105710565
:107780008105910511F00C94FD4D0C942F4B212F88
:10779000392D482D502FB101C2012D36E5E73E07A6
:1077A000E8E64E075105610571058105910511F463
:1077B0000C94454B2D36F5E73F07F8E64F0751058A
:1077C000610571058105910509F0E0F42237E2E7D2
:1077D0003E07E5E64E0751056105710581059105F6
:1077E00011F40C941F4823363D4648465105610567
:1077F00071058105910511F00C94FD4D0E94181D35
:107800000C94FF4D212F392D482D502FB101C2016D
:107810002436E3E63E07ECE64E07510561057105A7
:107820008105910511F40C9482472736FFE63F0746
:10783000FCE64F075105610571058105910511F4BD
:107840000C9485472336324349465105610571053D
:107850008105910511F00C94FD4D20C2212F392D89
:10786000482D502FB101C2012037FCE63F07F5E655
:107870004F07F8E65F07610571058105910509F479
:1078800080C62037ECE63E07E5E64E07E8E65E07F1
:10789000610571058105910511F008F0E0C02437FC
:1078A000F8E73F07F4E74F075105610571058105CA
:1078B000910511F40C945E452437E8E73E07E4E7B0
:1078C0004E075105610571058105910511F008F01C
:1078D0005DC02033F1E33F07F1E74F075105610534
:1078E00071058105910511F40C941F482033E1E3E3
:1078F0003E07E1E74E0751056105710581059105D8
:1079000009F0C0F42133F2E63F07F0E74F075105D5
:10791000610571058105910509F498C2223332464B
:1079200040475105610571058105910509F4E3C2E0
:107930000C94FD4D212F392D482D502FB101C2013E
:107940002037F5E63F07F2E74F075105610571055E
:107950008105910511F40C94D4492C36E4E73E07D7
:107960004E075105610571058105910511F40C94CF
:107970001A4D213331434147510561057105810598
:10798000910511F00C94FD4D0C946E48212F392D6A
:10799000482D502FB101C2012B36ECE63E07E5E73A
:1079A0004E07E2E65E07610571058105910509F460
:1079B00038C32B36FCE63F07F5E74F07F2E65F07D3
:1079C000610571058105910509F0E0F42437E4E6CD
:1079D0003E07E7E74E0751056105710581059105F1
:1079E00011F40C94684D24373F464F4652466105CA
:1079F00071058105910511F00C94FD4D0C9400006A
:107A00000C94FF4D212F392D482D502FB101C2016B
:107A10002E36E1E63E07E8E64E07E3E65E0761053F
:107A200071058105910511F40C9432452633F9E670
:107A30003F07F5E74F07F5E65F076105710581052B
:107A4000910509F4A2C529363C46414653466105D5
:107A500071058105910511F00C94FD4D7FC3212F17
:107A6000392D482D502FB101C2012437F3E73F07CC
:107A7000F5E64F07F2E75F0761057105810591059E
:107A800011F40C9484492437E3E73E07E5E64E07FA
:107A9000E2E75E07610571058105910511F008F0C7
:107AA00062C02337F5E63F07F2E74F07F0E75F07CD
:107AB000610571058105910511F40C94F54B23378F
:107AC000E5E63E07E2E74E07E0E75E076105710580
:107AD0008105910509F0D0F42136FDE63F07F5E771
:107AE0004F07F8E65F07610571058105910511F4FF
:107AF0000C94F248223737474047504761057105DB
:107B00008105910509F45CC20C94FD4D212F392D9E
:107B1000482D502FB101C2012436FDE63F07F3E6A0
:107B20004F07F2E75F07610571058105910509F4CB
:107B300037C62136ECE63E07E5E64E07E2E75E078C
:107B4000610571058105910509F43CC5233732476C
:107B500047475047610571058105910511F00C9467
:107B6000FD4D0C948749212F392D482D502FB101FF
:107B7000C2012437E2E73E07E1E64E07E5E75E078C
:107B8000610571058105910509F465C62437F2E7A1
:107B90003F07F1E64F07F5E75F07610571058105CE
:107BA000910509F0C8F42437E3E73E07E5E64E0700
:107BB000E4E75E07610571058105910509F4A9C730
:107BC00027373047484754476105710581059105BE
:107BD00009F41EC70C94FD4D212F392D482D502F2F
:107BE000B101C2012F36ECE63E07EFE54E07E6E7AE
:107BF0005E07610571058105910509F47CC52C3688
:107C0000F1E63F07F4E74F07F8E75F076105710505
:107C10008105910511F40C94E74C22373746404713
:107C20005547610571058105910511F00C94FD4DD5
:107C30000C945E4783E08093303610923236109277
:107C4000313640E356E362E182E492E00E944773FA
:107C50000C94FF4D0E94A11C0C94FF4D21E042E1C9
:107C600061E080ED0E94046521E042E161E080ED89
:107C70000E94046521E042E161E080ED0E9404651C
:107C800021E042E161E080ED0E94046521E042E1F3
:107C900061E080ED0E9404650C94FF4D60917E02CE
:107CA00070917F0280E090E00E94F99A6AEA75E0A4
:107CB0000E941A9B892B09F0C5C060917E027091C9
:107CC0007F0280E090E00E94F99A8C01009709F40D
:107CD00097C062E773E00E941A9B892BE1F488EE5B
:107CE00093E0A0E0B0E08093600290936102A093E3
:107CF0006202B093630268EE73E080E090E00E945D
:107D0000276344E050E067E170E080E692E00E9483
:107D1000A49E0C94FF4D60EB75E0C8010E941A9B75
:107D2000892BE1F480E197E2A0E0B0E0809360026B
:107D300090936102A0936202B093630260E177E2E4
:107D400080E090E00E94276344E050E067E170E04B
:107D500080E692E00E94A49E0C94FF4D63EB75E0D8
:107D6000C8010E941A9B892BE1F480EA96E8A1E001
:107D7000B0E08093600290936102A0936202B0939E
:107D8000630260EA76E881E090E00E94276344E0C5
:107D900050E067E170E080E692E00E94A49E0C94BF
:107DA000FF4D67EB75E0C8010E941A9B892BE1F437
:107DB00080E89AE1A6E0B0E08093600290936102CF
:107DC000A0936202B093630260E87AE186E090E0FB
:107DD0000E94276344E050E067E170E080E692E0B3
:107DE0000E94A49E0C94FF4D8FEA94E09F938F9382
:107DF0000E94D99B0E94F1110F900F900C94FF4D9F
:107E000060916002709161028091620290916302C0
:107E100028EE33E040E050E00E9488905F934F935B
:107E20003F932F938BEA94E09F938F930E94D99B6B
:107E30000E94F1110F900F900F900F900F900F90E4
:107E40000C94FF4D0E94E5160C94FF4D60917E024C
:107E500070917F0280E090E00E94F99A8C0163E4C7
:107E600075E00E941A9B892BA1F480916602909183
:107E70006702A0916802B0916902A26080936602D5
:107E800090936702A0936802B0936902299A0C94B8
:107E9000FF4D66E475E0C8010E941A9B892BB1F47E
:107EA0008091660290916702A0916802B091690288
:107EB000AD7F8093660290936702A0936802B093AF
:107EC000690280E00E9498290C94FF4D299903C013
:107ED00086E495E002C083E495E09F938F9383EA64
:107EE00094E09F938F930E94D99B0F900F900F90D7
:107EF0000F900C94FF4D60917E0270917F0280E0A4
:107F000090E00E94F99A8C0163E475E00E941A9B4C
:107F1000892BE1F48091660290916702A09168023A
:107F2000B0916902A4608093660290936702A09367
:107F30006802B09369022A9A44E050E06EE170E072
:107F400086E692E00E94A49E0C94FF4D66E475E0E4
:107F5000C8010E941A9B892BF1F4809166029091CE
:107F60006702A0916802B0916902AB7F80936602BC
:107F700090936702A0936802B093690280E00E9428
:107F80009E2944E050E06EE170E086E692E00E94B7
:107F9000A49E0C94FF4D2A9903C086E495E002C08C
:107FA00083E495E09F938F938BE994E09F938F9365
:107FB0000E94D99B0F900F900F900F900C94FF4D43
:107FC00060917E0270917F0280E090E00E94F99AB9
:107FD0008C0163E475E00E941A9B892B19F4779851
:107FE0000C94FF4D66E475E0C8010E941A9B892B32
:107FF00019F4779A0C94FF4D779B03C086E495E0C3
:1080000002C083E495E09F938F938FE696E09F9361
:108010008F930E94D99B0F900F900F900F900C940C
:10802000FF4D60917E0270917F0280E090E00E949F
:10803000F99A8C016BEB75E00E941A9B892BD1F4A5
:108040008091621E1F928F938091641E1F928F9366
:108050008091631E1F928F931F9284E18F9381E71B
:1080600094E09F938F930E94D99B0FB6F894DEBF44
:108070000FBECDBF60EC75E0C8010E941A9B892B32
:1080800019F40E94D03866C068EC75E0C8010E94FF
:108090001A9B892BF1F560917E0270917F0280E03E
:1080A00090E00E94F99A009709F454C00E94E69962
:1080B0008531910528F5909324148093231442E090
:1080C00050E062E070E083E294E10E94A49E60913F
:1080D0007E0270917F0280E090E00E94F99A009702
:1080E000C9F10E94E699909322148093211442E0F2
:1080F00050E060E070E081E294E10E94A49E2AC01A
:108100008FE594E09F938F930E94D99B0F900F90DF
:1081100021C0809124148F93809123148F9386E53E
:1081200094E09F938F930E94D99B0E94F1118091BC
:1081300022148F93809121148F9387E494E09F936E
:108140008F930E94D99B0E94F1110FB6F894DEBF65
:108150000FBECDBF0E94F1110C94FF4D60917E02C5
:1081600070917F0280E090E00E94F99A8C016CEEA1
:1081700074E00E941A9B892B09F077C060917E02FF
:1081800070917F0280E090E00E94F99A8C01009744
:1081900011F40C94FF4D66EC75E00E941A9B892B3C
:1081A000B1F482E29FEFACECBBE380938502909345
:1081B0008602A0938702B093880244E050E06EE408
:1081C00070E085E892E00E94A49E0C94FF4D6CEC58
:1081D00075E0C8010E941A9B892BB1F482E29FEFDF
:1081E000ACECBAE38093850290938602A093870259
:1081F000B093880244E050E06EE470E085E892E0DD
:108200000E94A49E0C94FF4DC8010E94E2992B018C
:108210003C0120E030E0A9010E94A6938823D9F018
:1082200081E00E9492109B01AC01C301B2010E9447
:10823000AB9360938502709386028093870290933C
:10824000880244E050E06EE470E085E892E00E942D
:10825000A49E0C94FF4D8AE394E09F938F930E9419
:10826000D99B0F900F900C94FF4D6FEE74E0C801F6
:108270000E941A9B892B09F077C060917E02709151
:108280007F0280E090E00E94F99A8C01009711F43F
:108290000C94FF4D66EC75E00E941A9B892BB1F49B
:1082A00082E29FEFACECBBE3809381029093820269
:1082B000A0938302B093840244E050E06AE470E04B
:1082C00081E892E00E94A49E0C94FF4D6CEC75E056
:1082D000C8010E941A9B892BB1F482E29FEFACEC9B
:1082E000BAE38093810290938202A0938302B093B9
:1082F000840244E050E06AE470E081E892E00E9489
:10830000A49E0C94FF4DC8010E94E2992B013C01F0
:1083100020E030E0A9010E94A6938823D9F082E0F2
:108320000E9492109B01AC01C301B2010E94AB9369
:1083300060938102709382028093830290938402FF
:1083400044E050E06AE470E081E892E00E94A49E7C
:108350000C94FF4D8DE294E09F938F930E94D99BE4
:108360000F900F900C94FF4D67EE74E0C8010E94CF
:108370001A9B892B09F073C060917E0270917F0275
:1083800080E090E00E94F99A8C01009711F40C941F
:10839000FF4D66EC75E00E941A9B892BB1F487EDC6
:1083A00094E3AFEEBCE38093890290938A02A0939A
:1083B0008B02B0938C0244E050E062E570E089E803
:1083C00092E00E94A49E0C94FF4D6CEC75E0C801F5
:1083D0000E941A9B892B51F48EE194E09F938F9316
:1083E0000E94D99B0F900F900C94FF4DC8010E94E2
:1083F000E2992B013C0120E030E0A9010E94A69304
:10840000882319F180E00E9492104B015C0121EE5B
:108410003AE744E95EE3C301B2010E94C792A501B5
:1084200094010E94AB936093890270938A028093B7
:108430008B0290938C0244E050E062E570E089E8A2
:1084400092E00E94A49E0C94FF4D81E194E09F93E2
:108450008F930E94D99B0F900F900C94FF4D0E9418
:10846000E0109F938F937F936F938AE094E09F93A4
:108470008F930E94D99B82E00E94921020918102EA
:108480003091820240918302509184020E9457965B
:10849000162F072FF82EE92E81E00E949210EF92FE
:1084A000FF920F931F932091850230918602409195
:1084B0008702509188020E9457969F938F937F93D3
:1084C0006F938EEF93E09F938F930E94D99B0E94AE
:1084D000F1110FB6F894DEBF0FBECDBF0C94FF4D67
:1084E00060917E0270917F0280E090E00E94F99A94
:1084F000009711F10E94972A00912D1410912E14CB
:1085000020912F1430913014601771078207930760
:1085100039F160932D1470932E1480932F1490933F
:10852000301444E050E06AE570E08DE294E10E948E
:10853000A49E88E696E002C081E696E09F938F9322
:108540000E94D99B60912D1470912E1480912F144C
:10855000909130140E94A4290E94F1110F900F9065
:1085600086E596E09F938F930E94D99B6FEF7FEFF4
:10857000CB010E94A4290E94F1110F900F900C943E
:10858000FF4D0E9485260C94FF4DF30184818433B6
:1085900029F440E061E080E00E94BB1880918002F5
:1085A000882311F40C94FF4D1F928F9383E596E07E
:1085B0009F938F930E94D99B0F900F900F900F90D5
:1085C0000C94FF4DF3018481893709F080C06091DC
:1085D0007E0270917F0280E090E00E94F99A8C0107
:1085E00063E475E00E941A9B892B51F48091660226
:1085F00090916702A0916802B0916902906410C0E6
:1086000066E475E0C8010E941A9B892BD1F4809121
:10861000660290916702A0916802B09169029F7B07
:108620008093660290936702A0936802B0936902F8
:1086300044E050E06EE170E086E692E00E94A49E85
:1086400046C061ED75E0C8010E941A9B892B21F597
:1086500080915B1D8F9380915A1D8F938091591D3E
:108660008F938091581D8F938091571D8F93809188
:10867000561D8F938091551D8F938091541D8F931C
:1086800083ED93E09F938F930E94D99B0FB6F8944C
:10869000DEBF0FBECDBF1BC0809166029091670206
:1086A000A0916802B091690296FD03C086E495E04E
:1086B00002C083E495E09F938F938FEC93E09F93A8
:1086C0008F930E94D99B0F900F900F900F908091E5
:1086D0008002882311F40C94FF4D1F928F9380E544
:1086E00096E09F938F930E94D99B0F900F900F90CD
:1086F0000F900C94FF4DF30184818737E9F5609169
:108700007E0270917F0280E090E00E94F99A0097CB
:10871000D9F00E94E2992B013C0120E030E0A90150
:108720000E94A693882381F040928D0250928E027F
:1087300060928F027092900244E050E066E570E033
:108740008DE892E00E94A49E809190028F93809188
:108750008F028F9380918E028F9380918D028F93E1
:1087600081EC93E09F938F930E94D99B0F900F9081
:108770000F900F900F900F9080918002882311F43A
:108780000C94FF4D1F928F938DE496E09F938F93EF
:108790000E94D99B0F900F900F900F900C94FF4D5B
:1087A00060917E0270917F0280E090E00E94F99AD1
:1087B0008C0163E475E00E941A9B40906602509021
:1087C00067026090680270906902892B19F46894BE
:1087D00057F809C066E475E0C8010E941A9B892B0E
:1087E00099F4E89457F840926602509267026092BA
:1087F00068027092690244E050E06EE170E086E643
:1088000092E00E94A49E13C057FC03C086E495E04A
:1088100002C083E495E09F938F938DEB93E09F9349
:108820008F930E94D99B0F900F900F900F90809183
:108830008002882311F40C94FF4D1F928F938AE4D9
:1088400096E09F938F930E94D99B0F900F900F906B
:108850000F900C94FF4D60917E0270917F0280E03A
:1088600090E00E94F99A8C0167ED75E00E941A9BD6
:10887000892B11F489E108C06BED75E0C8010E94F5
:108880001A9B892B49F480E18093C4001092C500A3
:1088900082E08093C00055C06FED75E0C8010E9472
:1088A0001A9B892B11F488E0EFCF64EE75E0C801C4
:1088B0000E941A9B892B39F069EE75E0C8010E946D
:1088C0001A9B892B11F483E0DFCF8091C40089319A
:1088D00041F488EB93E09F938F930E94D99B0F9074
:1088E0000F908091C400803141F483EB93E09F931B
:1088F0008F930E94D99B0F900F908091C400883075
:1089000041F48DEA93E09F938F930E94D99B0F903F
:108910000F908091C400833041F487EA93E09F93E5
:108920008F930E94D99B0F900F908091C400883044
:1089300041F481EA93E09F938F930E94D99B0F901B
:108940000F9080918002882311F40C94FF4D1F92A8
:108950008F9387E496E09F938F930E94D99B0F900B
:108960000F900F900F900C94FF4D60917E027091CC
:108970007F0280E090E00E94F99A66EC75E00E9428
:108980001A9B892B11F481E001C080E00E946829C4
:1089900080918002882311F40C94FF4D1F928F93D5
:1089A00084E496E09F938F930E94D99B0F900F9041
:1089B0000F900F900C94FF4D0E948C2780918002A5
:1089C000882311F40C94FF4D1F928F9381E496E05D
:1089D0009F938F930E94D99B0F900F900F900F90B1
:1089E0000C94FF4D0E94882780918002882311F407
:1089F0000C94FF4D1F928F938EE396E09F938F937D
:108A00000E94D99B0F900F900F900F900C94FF4DE8
:108A100060917E0270917F0280E090E00E94F99A5E
:108A20000E94E699803170F480932A140E94976D19
:108A300041E050E06DE170E08AE294E10E94A49E82
:108A40000C94FF4D80912A141F928F9387E993E035
:108A50009F938F930E94D99B0F900F900F900F9030
:108A60000C94FF4D60917E0270917F0280E090E057
:108A70000E94F99A0E94E69995EF980F903170F450
:108A8000809365020E94706C41E050E06CE170E000
:108A900085E692E00E94A49E0C94FF4D80916502B1
:108AA0001F928F938EE893E09F938F930E94D99BA0
:108AB0000F900F900F900F900C94FF4D60917E02DD
:108AC00070917F0280E090E00E94F99A009789F00F
:108AD0004AE050E0BC0183E49DE10E942A9B4AE009
:108AE00050E064E070E083E49DE10E94A49E0C9459
:108AF000FF4D83E49DE19F938F938EEE95E09F93CE
:108B00008F930E94C59B0F900F900F900F900C9425
:108B1000FF4D60917E0270917F0280E090E00E94A4
:108B2000F99A8C0162E773E00E941A9B892BE1F4A9
:108B3000219A8091660290916702A0916802B0919B
:108B4000690280618093660290936702A093680235
:108B5000B093690244E050E06EE170E086E692E096
:108B60000E94A49E0C94FF4D60EF74E0C8010E9427
:108B70001A9B892BE1F4229A8091660290916702F8
:108B8000A0916802B091690280628093660290931E
:108B90006702A0936802B093690244E050E06EE17E
:108BA00070E086E692E00E94A49E0C94FF4D64E57E
:108BB00073E0C8010E941A9B892BE1F4239A8091EB
:108BC000660290916702A0916802B0916902806488
:108BD0008093660290936702A0936802B093690243
:108BE00044E050E06EE170E086E692E00E94A49ED0
:108BF0000C94FF4D63E974E0C8010E941A9B892B15
:108C0000E1F4239A8091660290916702A091680234
:108C1000B091690280688093660290936702A09386
:108C20006802B093690244E050E06EE170E086E6CD
:108C300092E00E94A49E0C94FF4D68E07AE0C80187
:108C40000E941A9B892B71F581E0809394318CE509
:108C50009DE19093963180939531109298311092C6
:108C600097318091660290916702A0916802B0915D
:108C7000690291608093660290936702A0936802F4
:108C8000B093690244E050E06EE170E086E692E065
:108C90000E94A49E44E951E362E182E492E00E94D2
:108CA0004773ADC76BE773E0C8010E941A9B892B1D
:108CB00011F5ECE8FDE1119211922DE1EC3AF20789
:108CC000D1F78091660290916702A0916802B091FD
:108CD000690292608093660290936702A093680293
:108CE000B093690244E050E06EE170E086E692E005
:108CF0000E94A49E84C766E475E0C8010E941A9B86
:108D00004091660250916702609168027091690219
:108D1000892BC1F44F705C7F4093660250936702C9
:108D200060936802709369022B9A44E050E06EE110
:108D300070E086E692E00E94A49E809139360E94FF
:108D4000856C5DC744FD03C086E495E002C083E402
:108D500095E09F938F9383E893E09F938F930E9476
:108D6000D99B809166020F900F900F900F9085FD18
:108D700003C086E495E002C083E495E09F938F935F
:108D800088E793E09F938F930E94D99B809166021E
:108D90000F900F900F900F9086FD03C086E495E032
:108DA00002C083E495E09F938F938DE693E09F93B9
:108DB0008F930E94D99B809166020F900F900F9025
:108DC0000F9087FD03C086E495E002C083E495E040
:108DD0009F938F9382E693E09F938F930E94D99BFA
:108DE0008091660290916702A0916802B091690239
:108DF0000F900F900F900F9090FD03C086E495E0C8
:108E000002C083E495E09F938F9387E593E09F935F
:108E10008F930E94D99B8091660290916702A091E6
:108E20006802B09169020F900F900F900F9091FD22
:108E300003C086E495E002C083E495E09F938F939E
:108E40008CE493E09F938F930E94D99B809166025C
:108E500090916702A0916802B09169020F900F9003
:108E60000F900F9091FFCBC686EF95E00E94019C7A
:108E70009CE8E92E9DE1F92E00E010E02EEF822E15
:108E800025E0922EF70180819181F2E0EF0EF11C36
:108E90009F938F93C8010B969F938F939F928F926E
:108EA0000E94C59B0F5F1F4F0F900F900F900F9068
:108EB0000F900F900031110529F7A1C68AE396E0C3
:108EC0009F938F930E94D99B809180020F900F9067
:108ED000882361F01F928F9387E396E09F938F938F
:108EE0000E94D99B0F900F900F900F90F89498E0EC
:108EF00088E10FB6F894A895809360000FBE909318
:108F00006000FFCF0E94B5647AC660917E027091C6
:108F10007F0280E090E00E94F99A8C0163E475E0A2
:108F20000E941A9B892BE9F40E94746B809166025F
:108F300090916702A0916802B09169028D7F816073
:108F40008093660290936702A0936802B0936902CF
:108F500044E050E06EE170E086E692E00E94A49E5C
:108F60004EC666E475E0C8010E941A9B892BE1F4A5
:108F70000E94AA6A8091660290916702A09168029D
:108F8000B09169028C7F8093660290936702A093F0
:108F90006802B093690244E050E06EE170E086E65A
:108FA00092E00E94A49E2BC669E076E0C8010E9470
:108FB0001A9B892BE9F40E94AA6A8091660290911B
:108FC0006702A0916802B09169028E7F82608093EF
:108FD000660290936702A0936802B093690244E02E
:108FE00050E06EE170E086E692E00E94A49E07C623
:108FF0008091660281FF0FC089E096E09F938F9376
:1090000088E493E09F938F930E94D99B0F900F90D9
:109010000F900F90F4C580FD03C086E495E002C078
:1090200083E495E09F938F9384E493E09F938F93E1
:109030000E94D99B0F900F900F900F90E0C58091E8
:1090400092318F93809191318F93809190318F9352
:1090500080918F318F9380918E318F9380918D315C
:109060008F9380918C318F9380918B318F938091EE
:109070008A318F93809189318F93809188318F933A
:10908000809187318F93809186318F938091853144
:109090008F93809184318F93809183318F938BE074
:1090A00096E09F938F930E94D99B0E94F11180912B
:1090B00080020FB6F894DEBF0FBECDBF882309F43F
:1090C0009EC51F928F9388E096E09F938F930E9496
:1090D000D99B0F900F900F900F9091C5F89489E055
:1090E00021E030E0F90180935700C895E02C20E0A2
:1090F00030E0F90180935700C895F02C7894F894EB
:1091000023E030E0F90180935700C895002D22E05C
:1091100030E0F90180935700C895102D7894809124
:109120006C298F9380916B298F9380916A298F93FB
:10913000809169298F938EEF95E09F938F930E9482
:10914000D99B1F92EF921F92FF921F920F931F9233
:109150001F9387ED95E09F938F930E94D99B0E9468
:109160002628809166001F928F938BEC95E09F9349
:109170008F930E94D99B0E94F111809180020FB6BB
:10918000F894DEBF0FBECDBF882309F438C51F9207
:109190008F9388EC95E09F938F930E94D99B0F90BB
:1091A0000F900F900F902BC560E070E080E090E092
:1091B0000E94FA1160E070E081E090E00E94FA11F4
:1091C00080918002882309F41AC51F928F9385EC41
:1091D00095E09F938F930E94D99B0F900F900F90D3
:1091E0000F900DC50E9448260E94F11180918002C7
:1091F000882309F404C51F928F9382EC95E09F9316
:109200008F930E94D99B0F900F900F900F90F7C4EF
:1092100060917E0270917F0280E090E00E94F99A56
:1092200060EC75E00E941A9B892B31F5F8948FE170
:109230009BE00E9420748C01892B69F0C8010F9675
:109240000E948D70B80188E092E00E94D174C8013C
:109250000E948574F0CF8FE19BE00E947874892B87
:1092600029F08FE19BE00E943474F5CF8FE19BE001
:109270000E941C74789436C08FE19BE00E94207499
:109280008C018EE0E82E86E0F82E0115110551F1D3
:10929000F80186811F928F9380851F928F9385811D
:1092A0001F928F9381851F928F9387811F928F9337
:1092B00084811F928F9383811F928F9382811F924B
:1092C0008F9382851F928F93FF92EF920E94C59B8E
:1092D000C8010E9485748C010FB6F894DEBF0FBEE2
:1092E000CDBFD3CF80918002882309F488C41F9218
:1092F0008F938FEB95E09F938F930E94D99B0F9054
:109300000F900F900F907BC40E94873678C46091B5
:109310007E0270917F0280E090E00E94F99A8C01B9
:109320006DE476E00E941A9B892BD1F4809166024D
:1093300090916702A0916802B0916902977F809333
:10934000660290936702A0936802B093690244E0BA
:1093500050E06EE170E086E692E00E94A49E4FC469
:109360006CEC75E0C8010E941A9B892BD1F48091A6
:10937000660290916702A0916802B09169029860BC
:109380008093660290936702A0936802B09369028B
:1093900044E050E06EE170E086E692E00E94A49E18
:1093A0002EC40E94740E2BC460917E0270917F02C5
:1093B00080E090E00E94F99AFC0120812332C1F400
:1093C0004AE050E060E070E001960E9480977B8365
:1093D0006A8360917E0270917F0280E090E00E943B
:1093E000F99A2A813B81243031050CF096C002C0E5
:1093F0001B821A82009709F490C01982BE016F5F28
:109400007F4F0E94662F19013A014B01B82FA92FF7
:109410008AE02A813B81829FF001839FF00D112415
:10942000E45AF24E4080518032813C8383818D83A7
:1094300094819E8325812F83368138878781898710
:109440009101A301B4018B2F9A2F5201CC80DD80B2
:10945000EE80FF80088519850E94B29209F460C0F1
:109460008981811103C0208231822AC0181684F4B8
:10947000422853289C81692A2D81722A3E81832AA1
:109480008F81982A9885B92B2985A22B408217C0F5
:10949000209430946094709480949094B095A095AA
:1094A000242053203C8163228D8178229E81892251
:1094B0002F8192223885B3238985A8232082518267
:1094C0006282738284829582B683A78348E250E0E9
:1094D00062E270E08CE59DE10E94A49E87EB95E03E
:1094E0009F938F930E94D99B8AE02A813B81829F20
:1094F000F001839FF00D1124E45AF24E2081318156
:109500004281538164817581868197810E94502BAD
:109510000E94F1110F900F9003C082E00E94403131
:109520008BEA95E09F938F930E94D99B2FEF3FEF9B
:109530004FEF5FEF6FEF7FEF8FEF9FEF0E94502BAA
:109540000E94F111809180020F900F90882309F4FE
:1095500056C31F928F9388EA95E09F938F930E9442
:10956000D99B0F900F900F900F9049C360917E028E
:1095700070917F0280E090E00E94F99AFC012081C6
:109580002332A1F44AE050E060E070E001960E94CE
:1095900080978B0160917E0270917F0280E090E065
:1095A0000E94F99A04301105ECF402C000E010E0CA
:1095B0000097C1F04AE050E060E070E00E94AB9894
:1095C0002AE0209FF001219FF00D1124E45AF24E71
:1095D0007187608748E250E062E270E08CE59DE1CF
:1095E0000E94A49E81E00E944031809180028823E5
:1095F00009F405C31F928F9385EA95E09F938F939B
:109600000E94D99B0F900F900F900F90F8C20E946C
:10961000147580918002882309F4F1C21F928F9300
:1096200082EA95E09F938F930E94D99B0F900F90B1
:109630000F900F90E4C20E9405328091800288232F
:1096400009F4DDC21F928F938FE995E09F938F936A
:109650000E94D99B0F900F900F900F90D0C280E086
:1096600090E00E94422880918002882309F4C7C2BA
:109670001F928F938CE995E09F938F930E94D99BC3
:109680000F900F900F900F90BAC28091792D81FFAB
:109690002DC00E94CE25892B49F5809170298F938A
:1096A00080916F298F9380916E298F9380916D297E
:1096B0008F9381E995E09F938F930E94D99B80912E
:1096C0005D368F9380915C368F9380915B368F935C
:1096D00080915A368F9384E895E09F938F930E94F0
:1096E000D99B0FB6F894DEBF0FBECDBF0E94F1111B
:1096F0008091792D90917A2D93FF63C081E090E065
:109700000E9446257B011C0180E090E00E944625D6
:109710004B018C010E94A4243F922F92FF92EF9262
:1097200083E795E09F938F930E94D99B1F930F939C
:109730009F928F9283E695E09F938F930E94D99B8F
:10974000240138019401A80147018101B701C10139
:109750000E9443239F938F937F936F9388E595E0B7
:109760009F938F930E94D99B242D352D462D572DE5
:109770006E2D792D822D912F0E94A4239F938F937C
:109780007F936F938AE495E09F938F930E94D99B78
:10979000242D352D462D572D6E2D792D822D912F6F
:1097A0000E9405249F938F937F936F9387E395E0A7
:1097B0009F938F930E94D99B0FB6F894DEBF0FBE84
:1097C000CDBF0E94F11180918002882309F417C255
:1097D0001F928F9384E395E09F938F930E94D99B70
:1097E0000F900F900F900F900AC28091792D82FFF9
:1097F0003FC021E048E061E083E00E94261A8091AA
:10980000601E8F9380915F1E8F9380915E1E8F9359
:1098100080915D1E8F9380915C1E8F9380915B1E63
:109820008F9380915A1E8F938091591E8F938DE153
:1098300095E09F938F930E94D99B0E94F111809194
:10984000581E8F938091571E8F938091561E8F9331
:109850008091551E8F938FE095E09F938F930E9488
:10986000D99B0E94F1110FB6F894DEBF0FBECDBF99
:109870008091792D85FF58C081E00E94B27D609172
:109880004D3670914E3680914F36909150360E94F1
:109890005F9420E030E048EC52E40E94AB939F9349
:1098A0008F937F936F9382E596E09F938F930E94AF
:1098B000C59B60915136709152368091533690918C
:1098C00054360E945D9420E030E040E85AE30E9464
:1098D00057969F938F937F936F9381E696E09F9324
:1098E0008F930E94C59B609155367091563680913A
:1098F0005736909158360E945D9420E030E040E861
:109900005BE30E9457969F938F937F936F9382E7B9
:1099100096E09F938F930E94C59B0E94F1110FB612
:10992000F894DEBF0FBECDBF8091792D90917A2D36
:1099300094FF3BC00E949D1E20E030E048EC52E4C2
:10994000162F072FF82EE92E0E94579620E836EEA4
:1099500045EC57E40E94AB9321E03EED42E45EE328
:109960000E94C4969B01AC0160E070E080E89FE338
:109970000E94C7922BE43AE34DEB57E30E94AB936E
:109980009F938F937F936F93EF92FF920F931F9309
:1099900086EF94E09F938F930E94D99B0E94F111D0
:1099A0000FB6F894DEBF0FBECDBF80918002882332
:1099B00009F425C11F928F9383EF94E09F938F93B7
:1099C0000E94D99B0F900F900F900F9018C160913B
:1099D0007E0270917F0280E090E00E94F99A62E836
:1099E00076E00E941A9B892B99F460917E02709117
:1099F0007F0280E090E00E94F99A009709F4FFC08E
:109A00000E94E69990915201892B80935201F7C0F0
:109A1000809152018F701F928F9387E393E09F9301
:109A20008F930E94D99B0E94F1110F900F900F907D
:109A30000F90E5C060917E0270917F0280E090E01F
:109A40000E94F99A009711F14AE050E060E070E05E
:109A50000E948097603198F4609364021F926F9324
:109A600086EE94E09F938F930E94D99B41E050E053
:109A70006BE170E084E692E00E94A49E11C08091A8
:109A800064021F928F938DED94E006C08091640272
:109A90001F928F9384ED94E09F938F930E94D99BA4
:109AA0000F900F900F900F900E94F1118091800203
:109AB000882309F4A4C01F928F9381ED94E09F93B3
:109AC0008F930E94D99B0F900F900F900F9097C08B
:109AD00060917E0270917F0280E090E00E94F99A8E
:109AE0008C0163E475E00E941A9B892BE1F40E94CB
:109AF0009D698091660290916702A0916802B09181
:109B0000690290618093660290936702A093680255
:109B1000B093690244E050E06EE170E086E692E0C6
:109B20000E94A49E6CC066E475E0C8010E941A9B66
:109B3000892B99F5F8940E94AA690FB6F894A89514
:109B400080916000886180936000109260000FBE79
:109B500084B7877F84BF80916000886180936000B4
:109B60001092600078948091660290916702A091B3
:109B70006802B09169029F7E8093660290936702AB
:109B8000A0936802B093690244E050E06EE170E097
:109B900086E692E00E94A49E32C067E876E0C801A3
:109BA0000E941A9B40916602509167026091680280
:109BB00070916902892B69F454FF02C0F894FFCFB9
:109BC00086E293E09F938F930E94D99B0F900F9012
:109BD00016C054FD03C086E495E002C083E495E01E
:109BE0009F938F9382E293E09F938F930E94D99BE0
:109BF0000F900F900F900F9002C00E946C26EA8584
:109C0000FB851182108283E02B960FB6F894DEBF9D
:109C10000FBECDBFDF91CF911F910F91FF90EF90BD
:109C2000DF90CF90BF90AF909F908F907F906F907C
:109C30005F904F903F902F900895CF93DF93EC016A
:109C400088819981009741F08536924109F490C04E
:109C50001982188283E097C00E94DA3780916602E9
:109C600080FD05C081FF01C01D9B0E94AA6A8091F2
:109C700070008C7F809370008091B600806280932A
:109C8000B6001092B20082E08093B1008091B600DD
:109C90008770E1F78091700081608093700062E9C5
:109CA0007EE080E090E00E9477690E94882780E053
:109CB0000E9468298FE292E19F938F930E94D99B23
:109CC0000E94E5168091792D90917A2D0F900F903A
:109CD00091FD0E9461648091792D90917A2D93FD80
:109CE0000E945C248091792D90917A2D92FF06C07C
:109CF00021E04CE061E080ED0E94046580912A142F
:109D00000E94976D809165020E94706C0E946D6C3C
:109D100080930F0B809165020E94706C80912A14D1
:109D20001F928F9380910F0B1F928F938CE896E078
:109D30009F938F930E94C59B1092110B1092100B52
:109D40000F900F900F900F900F900F9086E592E07C
:109D500090934C3680934B3683E290E09093261498
:109D60008093251485E692E19983888381E00BC076
:109D70006332E1F748EA51E360E070E080E19BE0A4
:109D80000E945539E3CFDF91CF9108950F931F9330
:109D9000CF93DF93EC018A0188819981009711F1BB
:109DA0008A37924121F01982188283E020C0623103
:109DB000E9F4A80162E170E080E19BE00E9455397E
:109DC00084E0809330361092323610923136109300
:109DD00034360093333640E356E362E182E492E0A6
:109DE0000E9447738AE792E19983888381E0DF913B
:109DF000CF911F910F9108958436910514F19F938F
:109E00008F9382EE96E09F938F930E94C59B8091E3
:109E1000833190918431A0918531B0918631019642
:109E2000A11DB11D8093833190938431A09385311E
:109E3000B09386310F900F900F900F9081E090E0DB
:109E4000089580E090E008952F923F924F925F92A4
:109E50006F927F928F929F92AF92BF92CF92DF923A
:109E6000EF92FF920F931F93CF93DF93CDB7DEB79F
:109E7000CC59D1090FB6F894DEBF0FBECDBFCB567B
:109E8000DF4F99838883C559D0408A01633871F4C4
:109E900084E19BE0C456DF4F6883CC59D0400E94D8
:109EA0006576C456DF4F6881CC59D040CB56DF4F22
:109EB000A881B981C559D0402D913C912231B2E1A0
:109EC0003B0711F40C94FD5D40F42115310581F040
:109ED0002331304109F4AAC49EC4243242E134073C
:109EE00009F478C42B32324111F40C94055E93C40A
:109EF00048EB59E061E870E084E19BE00E944A761B
:109F000083E190E15EC45A01E3E0F0E0EC0FFD1F55
:109F1000E40FF51F1082CA010E94FC4E892B81F7C5
:109F200020E030E040E050E0CC56DF4F6881C4597B
:109F3000D040627070E080E090E0A0E00E94BB92B0
:109F400009F01EC7CE56DF4F2881C259D040287075
:109F500030E040E050E060E070E080E090E0A0E0C1
:109F60000E94BB9299F127E04AE250E06BE270E078
:109F700089E290E00E94E26082E496E30E94B3628C
:109F8000BC01990F880B990B0E945F9420E030E090
:109F900048EC52E40E94AB939F938F937F936F930F
:109FA00086E197E09F938F931F9287E78F93CE016F
:109FB0008A0D9B1D03969F938F930E94319CA80E40
:109FC000B91E0FB6F894DEBF0FBECDBFCE56DF4F21
:109FD0002881C259D040207130E040E050E060E07C
:109FE00070E080E090E0A0E00E94BB92E9F126E002
:109FF0004AE250E06BE270E089E290E00E94E260A9
:10A0000081E090E00E9489118093291485EB9DE105
:10A010000E94B362BC01990F880B990B0E945F9458
:10A0200020E030E048EC52E40E94AB939F938F9382
:10A030007F936F9380E297E09F938F931F9287E7C0
:10A040008F93C501029621E030E02C0F3D1F820F57
:10A05000931F9F938F930E94319CA80EB91E0FB639
:10A06000F894DEBF0FBECDBFC257DF4F2881CE5858
:10A07000D04030E040E050E060E070E080E090E010
:10A08000A0E00E94BB9201F10E9445119F938F9323
:10A090007F936F938BE297E09F938F931F9287E755
:10A0A0008F93C5010296A1E0B0E0AC0FBD1F8A0FEF
:10A0B0009B1F9F938F930E94319CA80EB91E0FB6D1
:10A0C000F894DEBF0FBECDBFCE56DF4F2881C259F8
:10A0D000D040207430E040E050E060E070E080E08C
:10A0E00090E0A0E00E94BB9231F180917E318F938D
:10A0F00080917D318F9380917C318F9380917B31E2
:10A100008F9389E397E09F938F931F9287E78F93B5
:10A11000C501029621E030E02C0F3D1F820F931FF6
:10A120009F938F930E94319CA80EB91E0FB6F8948E
:10A13000DEBF0FBECDBFCE56DF4F2881C259D04003
:10A14000207830E040E050E060E070E080E090E0B7
:10A15000A0E00E94BB9241F1F89480912836909142
:10A160002936A0912A36B0912B367894BF93AF93BD
:10A170009F938F9387E497E09F938F931F9287E736
:10A180008F93C5010296A1E0B0E0AC0FBD1F8A0F0E
:10A190009B1F9F938F930E94319CA80EB91E0FB6F0
:10A1A000F894DEBF0FBECDBF20E0312F317040E00C
:10A1B00050E060E070E080E090E0A0E00E94BB92A0
:10A1C00009F0F0C520E0312F327040E050E060E04F
:10A1D00070E080E090E0A0E00E94BB9209F060C6D1
:10A1E00020E0312F347040E050E060E070E080E02B
:10A1F00090E0A0E00E94BB9209F083C620E0312FDE
:10A20000387040E050E060E070E080E090E0A0E076
:10A210000E94BB9209F0A5C620E0312F307140E0CA
:10A2200050E060E070E080E090E0A0E00E94BB922F
:10A2300009F015C720E0312F307240E050E060E0B7
:10A2400070E080E090E0A0E00E94BB9209F037C788
:10A2500020E030E040E050E0CC56DF4F6881C45948
:10A26000D040647070E080E090E0A0E00E94BB927B
:10A2700009F053C720E0C856DF4F3881C859D04095
:10A2800040E050E060E070E080E090E0A0E00E94FC
:10A29000BB9209F0AFC720E0C756DF4F3881C959DC
:10A2A000D04040E050E060E070E080E090E0A0E06E
:10A2B0000E94BB9209F0CCC7502F5170952E20E020
:10A2C00030E0452F50E060E070E080E090E0A0E0FA
:10A2D0000E94BB9209F0EBC720E030E0402F4270B3
:10A2E00050E060E070E080E090E0A0E00E94BB926F
:10A2F00011F00C948B5920E030E0C657DF4F4881B5
:10A30000CA58D04050E060E070E080E090E0A0E00B
:10A310000E94BB9211F00C94BF5920E030E040E065
:10A3200050E0CC56DF4F6881C459D040687070E06F
:10A3300080E090E0A0E00E94BB9211F00C94EA59FA
:10A3400020E030E040E050E0CC56DF4F6881C45957
:10A35000D040607170E080E090E0A0E00E94BB928D
:10A3600011F00C94165A20E030E0402F487050E075
:10A3700060E070E080E090E0A0E00E94BB9211F00D
:10A380000C94425A20E030E0402F407150E060E0F1
:10A3900070E080E090E0A0E00E94BB9211F00C948D
:10A3A000775A20E030E0402F407250E060E070E0EB
:10A3B00080E090E0A0E00E94BB9211F00C94AC5AB7
:10A3C00020E030E0402F407450E060E070E080E03A
:10A3D00090E0A0E00E94BB9211F00C94E15AF02FA3
:10A3E000F0787F2E20E030E04F2F50E060E070E00A
:10A3F00080E090E0A0E00E94BB9211F00C94165B0C
:10A40000CD56DF4F2881C359D0402170622E20E005
:10A4100030E040E0562D60E070E080E090E0A0E0A9
:10A420000E94BB9211F40C94185E8091792D82FDEC
:10A4300002C00C945E5B21E046E061E083E00E9494
:10A44000261A20E030E0472D50E060E070E080E028
:10A4500090E0A0E00E94BB9211F40C945E5B8091AE
:10A46000792D82FF02C00C94235B20E030E040E0B5
:10A47000CD56DF4F5881C359D040527060E070E034
:10A4800080E090E0A0E00E94BB9211F00C94935BFE
:10A4900020E030E040E0CD56DF4F5881C359D04036
:10A4A000547060E070E080E090E0A0E00E94BB9219
:10A4B00011F00C94C65B20E030E040E0CD56DF4F59
:10A4C0005881C359D040507160E070E080E090E066
:10A4D000A0E00E94BB9211F00C94F95B20E030E008
:10A4E00040E0CD56DF4F5881C359D040507260E0F4
:10A4F00070E080E090E0A0E00E94BB9211F00C942C
:10A50000385C20E030E040E0CD56DF4F5881C35941
:10A51000D040507460E070E080E090E0A0E00E94E5
:10A52000BB9211F00C94775C20E030E040E0CD5617
:10A53000DF4F5881C359D040587060E070E080E030
:10A5400090E0A0E00E94BB9211F00C94B65C20E079
:10A5500030E040E050E0CC56DF4F6881C459D04035
:10A56000607270E080E090E0A0E00E94BB9211F485
:10A570000C94E75C8091792D85FD02C00C94E75C1A
:10A5800081E00E94B27D60914D3670914E3680918F
:10A590004F36909150360E945F9420E030E048ECB6
:10A5A00052E40E94AB939F938F937F936F9380EDC0
:10A5B00098E09F938F931F9287E78F93C501029630
:10A5C00041E050E04C0F5D1F840F951F9F938F93C8
:10A5D0000E94319CA80EB91EC5010E94FC4E0FB608
:10A5E000F894DEBF0FBECDBF892B09F089CCE1E026
:10A5F00020E030E040E050E0CC56DF4F6881C459A5
:10A60000D040607470E080E090E0A0E00E94BB92D7
:10A6100011F00C94EA5C20E030E040E050E0CC56D1
:10A62000DF4F6881C459D040607870E080E090E0EE
:10A63000A0E00E94BB9211F00C942D5D20E030E070
:10A6400040E0C656DF4F5881CA59D04060E070E004
:10A6500080E090E0A0E00E94BB9211F00C946F5D4E
:10A6600020E030E0492D50E060E070E080E090E0D4
:10A67000A0E00E94BB9211F00C949F5DCE56DF4F7C
:10A680002881C259D040312F402FCD56DF4F5881FD
:10A69000C359D040CC56DF4F6881C459D040722D89
:10A6A000832DC956DF4F9881C759D040A0E00E9442
:10A6B000BB9211F00C94AA5D809164028061898341
:10A6C0008091080B8A83FE01EA0DFB1D13828091A5
:10A6D0002D1490912E14A0912F14B0913014850157
:10A6E0000D5F1F4F80FF0CC01F930F938BE199E00C
:10A6F0009F938F930E94C59B0F900F900F900F9088
:10A70000B801CE0101960E9454788091660282FFC2
:10A710000AC028E232E3A801BE016F5F7F4F8EE6D8
:10A7200092E00E94C76380912D1490912E14A09105
:10A730002F14B091301482FD73980E94746B84E1E1
:10A740009BE00E9467768091660290916702A091DB
:10A750006802B091690290FD02C00C94E15D5FEF68
:10A76000A51AB50A0E946D6CF82E89E10E94856CCD
:10A770008091660290916702A0916802B09169028F
:10A7800090FD02C00C94DD5D73988091080B8F5F83
:10A790008093080B8A83B5016F5F7F4FCE010196CE
:10A7A0000E94547884E19BE00E94677640E050E08C
:10A7B00065E880916F15909170150E94477382E152
:10A7C00092E1CB56DF4FA881B981C559D0408D9316
:10A7D0009C931EC08CEF9AE00E94D571892BC1F02A
:10A7E0000E94746B8091660287FD2B9840E450E0D4
:10A7F00060E070E08CEF9AE00E94B7718BE292E12A
:10A80000CB56DF4FE881F981C559D04091838083D1
:10A8100081E00C94285ECB56DF4FA881B981C559E1
:10A82000D0401D921C9283E00C94285E623181F727
:10A830008090660290906702A0906802B0906902D2
:10A8400091FC5ECBF8018081813021F50180F2819D
:10A85000E02D2081CE56DF4F2883C259D040118190
:10A8600002813381CD56DF4F3883C359D0404481B4
:10A87000CC56DF4F4883C459D0402580368057815D
:10A88000C956DF4F5883C759D040C084D184E12CCA
:10A89000F12C55C08230C1F4E380F480C12CD12C5E
:10A8A000B1E0CE56DF4FB883C259D04010E000E08F
:10A8B000E0E8CD56DF4FE883C359D040CC56DF4F98
:10A8C0001882C459D04034C08330D9F0843009F0A4
:10A8D00017CBC12CD12CE12CF12CF5E0CE56DF4F5B
:10A8E000F883C259D04010E000E0CD56DF4F188207
:10A8F000C359D04022E0CC56DF4F2883C459D04002
:10A9000017C0C12CD12CE12CF12C35E0CE56DF4FF5
:10A910003883C259D04010E000E0CD56DF4F188296
:10A92000C359D04041E0CC56DF4F4883C459D04092
:10A93000212C312CC956DF4F1882C759D040409086
:10A940007B3150907C3160907D3170907E31809170
:10A950008D0290918E02A0918F02B0919002C65705
:10A96000DF4F88839983AA83BB83CA58D0402DECDC
:10A970003CEC4CE45EE3BC01CD010E94C8929B011B
:10A98000AC01C301B2010E94849587FD0BC0E8941D
:10A99000A0F88092660290926702A0926802B0923C
:10A9A000690247C0C657DF4F288139814A815B81E0
:10A9B000CA58D040C301B2010E94A69387FF39C094
:10A9C0008091873190918831A0918931B0918A31FD
:10A9D0000196A11DB11D8093873190938831A0937A
:10A9E0008931B0938A31A0FC8BCA6894A0F8809218
:10A9F000660290926702A0926802B092690295E4A2
:10AA0000CE56DF4F9883C259D04010E200E0CD56B9
:10AA1000DF4F1882C359D040A4E0CC56DF4FA88343
:10AA2000C459D040212C312CC956DF4F1882C75948
:10AA3000D040B02FB470C657DF4FB883CA58D0404B
:10AA400020E030E04B2F50E060E070E080E090E0EC
:10AA5000A0E00E94BB9209F08C9ACE56DF4FE881AD
:10AA6000C259D040E072C257DF4FE883CE58D04081
:10AA70002E2F30E040E050E060E070E080E090E0B9
:10AA8000A0E00E94BB9211F00E944511F12FF074DA
:10AA9000C856DF4FF883C859D04020E03F2F40E030
:10AAA00050E060E070E080E090E0A0E00E94BB92A7
:10AAB00011F00E94CE25212F2078C756DF4F288322
:10AAC000C959D04020E0C756DF4F3881C959D0401E
:10AAD00040E050E060E070E080E090E0A0E00E94A4
:10AAE000BB9251F00E94E010609335367093363679
:10AAF0008093373690933836CE56DF4F2881C2592F
:10AB0000D040217030E040E050E060E070E080E054
:10AB100090E0A0E00E94BB92F1F083E49DE19F935E
:10AB20008F9386EF96E09F938F931F9287E78F9383
:10AB3000CE0103969F938F930E94319C4C010E94FB
:10AB4000FC4E0FB6F894DEBF0FBECDBF892B09F0C7
:10AB5000D7C9540102C0A12CB12CCE56DF4F288199
:10AB6000C259D040227030E040E050E060E070E038
:10AB700080E090E0A0E00E94BB92D1F1C501029676
:10AB80006EEF76E0A1E0B0E0AC0FBD1F8A0F9B1F17
:10AB90000E94239BB3E0AB0EB11C22E4622E26E39D
:10ABA000722E34E8832E33E0932E47E7542EF301C0
:10ABB00081913F011F928F939F928F921F925F927C
:10ABC000C501029621E030E02C0F3D1F820F931F3C
:10ABD0009F938F930E94319CA80EB91E0FB6F894D4
:10ABE000DEBF0FBECDBF5AE4651656E37506F9F613
:10ABF000CE56DF4F2881C259D040247030E040E06B
:10AC000050E060E070E080E090E0A0E00E94BB9245
:10AC100009F450C0C501029662E077E0A1E0B0E01F
:10AC2000AC0FBD1F8A0F9B1F0E94239BB4E0AB0E8D
:10AC3000B11C2E01EAE74E0E511C80E1D2011D929B
:10AC40008A95E9F728E0A20168E980EB0E949B164B
:10AC50003201B8E06B0E711C94E8892E93E0992EB6
:10AC600027E7F20181912F011F928F939F928F927C
:10AC70001F922F93C501029641E050E04C0F5D1FDB
:10AC8000840F951F9F938F93C556DF4F2883CB5911
:10AC9000D0400E94319CA80EB91E0FB6F894DEBFBA
:10ACA0000FBECDBFC556DF4F2881CB59D0404614CB
:10ACB0005704B9F6CD56DF4F9881C359D0409078EC
:10ACC000C656DF4F9883CA59D04020E030E040E0BC
:10ACD000592F60E070E080E090E0A0E00E94BB921D
:10ACE000E1F480912B1490912C149F938F9387E023
:10ACF00097E09F938F931F9287E78F93CE018A0DE2
:10AD00009B1D03969F938F930E94319CA80EB91EA2
:10AD10000FB6F894DEBF0FBECDBF20E030E040E0BC
:10AD200050E0CC56DF4F6881C459D040617070E06C
:10AD300080E090E0A0E00E94BB9209F4F1C8E3E05B
:10AD4000F0E0EC0FFD1FEA0DFB1D80E28083A50102
:10AD500083E090E08A199B09FC01E40FF51FE85598
:10AD6000FE4C20814F5F5F4F222309F4CCC8208125
:10AD7000E1E0F0E0EC0FFD1FE40FF51F2283ECCFC4
:10AD8000CE018A0D9B1D6EE077E003960E94239B07
:10AD9000B7E0AB0EB11CC5010E94FC4E892B09F037
:10ADA000AFC8D0C8C114D10409F40CCAF8944090BB
:10ADB00028365090293660902A3670902B36789439
:10ADC0008091AD1D9091AE1DA091AF1DB091B01DB1
:10ADD000A3019201281B390B4A0B5B0BCA01B90175
:10ADE0000E945D94C257DF4F688379838A839B8377
:10ADF000CE58D040B60180E090E00E945D949B0167
:10AE0000AC01C257DF4F688179818A819B81CE581E
:10AE1000D0400E94AB934C019F928F937F936F938E
:10AE200082E597E09F938F931F9287E78F939E0110
:10AE30002A0D3B1D2D5F3F4F3F932F93C456DF4F8D
:10AE40006883CC59D040C556DF4F7883CB59D0406A
:10AE50000E94319CA80EB91EC456DF4F6881CC59A0
:10AE6000D040C556DF4F7881CB59D040862F972FE1
:10AE7000A82DB92D80933A3690933B36A0933C365B
:10AE8000B0933D364092AD1D5092AE1D6092AF1D05
:10AE90007092B01D0FB6F894DEBF0FBECDBF92C941
:10AEA000C114D10409F49CC9F8948091841D909137
:10AEB000851DA091861DB091871D78949F938F93D7
:10AEC00080916D028F9380916C028F938FE597E054
:10AED0009F938F931F9287E78F93C5010296A1E0FE
:10AEE000B0E0AC0FBD1F8A0F9B1F9F938F930E94F2
:10AEF000319CA80EB91E0FB6F894DEBF0FBECDBFB1
:10AF00006FC9F89480912C3690912D36A0912E36F1
:10AF1000B0912F367894BF93AF939F938F938FE622
:10AF200097E09F938F931F9287E78F93C5010296B7
:10AF300021E030E02C0F3D1F820F931F9F938F93D2
:10AF40000E94319CA80EB91EC5010E94FC4E0FB68E
:10AF5000F894DEBF0FBECDBF892B11F00C94804F4B
:10AF60004DC9C114D10409F457C9F89440902C3646
:10AF700050902D3660902E3670902F3678948091B8
:10AF8000B11D9091B21DA091B31DB091B41DA3014C
:10AF90009201281B390B4A0B5B0BCA01B9010E94B5
:10AFA0005D94C257DF4F688379838A839B83CE5831
:10AFB000D040B60180E090E00E945D949B01AC011E
:10AFC000C257DF4F688179818A819B81CE58D040FA
:10AFD0000E94AB934C019F928F937F936F938AE76C
:10AFE00097E09F938F931F9287E78F939E012A0D7F
:10AFF0003B1D2D5F3F4F3F932F93C456DF4F688318
:10B00000CC59D040C556DF4F7883CB59D0400E94F1
:10B01000319CA80EB91EC456DF4F6881CC59D04070
:10B02000C556DF4F7881CB59D040862F972FA82D5A
:10B03000B92D80933E3690933F36A0934036B0931F
:10B0400041364092B11D5092B21D6092B31D709274
:10B05000B41D0FB6F894DEBF0FBECDBFDDC8CD283E
:10B0600009F4E8C8F8948091881D9091891DA091F9
:10B070008A1DB0918B1D78949F938F9380916B0262
:10B080008F9380916A028F9387E897E09F938F93C5
:10B090001F9287E78F93C5010296A1E0B0E0AC0F45
:10B0A000BD1F8A0F9B1F9F938F930E94319CA80EF8
:10B0B000B91E0FB6F894DEBF0FBECDBFBBC88091DE
:10B0C0007F3190918031A0918131B0918231BF93D5
:10B0D000AF939F938F9387E997E09F938F931F92EE
:10B0E00087E78F93C501029621E030E02C0F3D1FCA
:10B0F000820F931F9F938F930E94319CA80EB91EBD
:10B10000C5010E94FC4E0FB6F894DEBF0FBECDBF46
:10B11000892B11F00C94804F9BC880918A318F93BA
:10B12000809189318F93809188318F93809187317D
:10B130008F93809186318F93809185318F93809109
:10B1400084318F93809183318F9382EA97E09F932C
:10B150008F931F9287E7982E9F92C5010296A1E0D8
:10B16000B0E0AC0FBD1F8A0F9B1F9F938F930E946F
:10B17000319CA80EB91EC5010E94FC4E0FB6F89472
:10B18000DEBF0FBECDBF892B11F00C94804F809194
:10B19000792D90917A2D93FF6DC880918E318F9388
:10B1A00080918D318F9380918C318F9380918B31F1
:10B1B0008F9386EC97E09F938F931F929F92C50188
:10B1C000029621E030E02C0F3D1F820F931F9F93CA
:10B1D0008F930E94319CA80EB91EC5010E94FC4E9F
:10B1E0000FB6F894DEBF0FBECDBF892B11F00C94C3
:10B1F000804F40C8809170298F9380916F298F93E1
:10B2000080916E298F9380916D298F9388ED97E0BF
:10B210009F938F931F9287E78F93C5010296A1E0BA
:10B22000B0E0AC0FBD1F8A0F9B1F9F938F930E94AE
:10B23000319CA80EB91EC5010E94FC4E0FB6F894B1
:10B24000DEBF0FBECDBF892B11F00C94804F23C8F9
:10B25000809138368F93809137368F938091363630
:10B260008F93809135368F9383EE97E09F938F93E2
:10B270001F9287E78F93C501029621E030E02C0FE3
:10B280003D1F820F931F9F938F930E94319CA80EA6
:10B29000B91EC5010E94FC4E0FB6F894DEBF0FBE6A
:10B2A000CDBF892B11F00C94804F0C945C5181E040
:10B2B0000E9492102091850230918602409187026F
:10B2C000509188020E9457969F938F937F936F931C
:10B2D00080EF97E09F938F931F9287E78F93C5012D
:10B2E0000296A1E0B0E0AC0FBD1F8A0F9B1F9F9399
:10B2F0008F930E94319CA80EB91EC5010E94FC4E7E
:10B300000FB6F894DEBF0FBECDBF892B11F00C94A1
:10B31000804F0C946C5182E00E9492102091810227
:10B320003091820240918302509184020E9457968C
:10B330009F938F937F936F938DEF97E09F938F935E
:10B340001F9287E78F93C501029621E030E02C0F12
:10B350003D1F820F931F9F938F930E94319CA80ED5
:10B36000B91EC5010E94FC4E0FB6F894DEBF0FBE99
:10B37000CDBF892B11F00C94804F0C947B5183E04E
:10B380000E9492109F938F937F936F938AE098E02F
:10B390009F938F931F9287E78F93C5010296A1E039
:10B3A000B0E0AC0FBD1F8A0F9B1F9F938F930E942D
:10B3B000319CA80EB91E8C98C5010E94FC4E0FB698
:10B3C000F894DEBF0FBECDBF892B11F00C94804FD7
:10B3D0000C948D51299903C086E495E002C083E462
:10B3E00095E09F938F9387E198E09F938F931F92AF
:10B3F00087E78F93C501029621E030E02C0F3D1FB7
:10B40000820F931F9F938F930E94319CA80EB91EA9
:10B41000C5010E94FC4E0FB6F894DEBF0FBECDBF33
:10B42000892B11F00C94804F0C94A0512A9903C0E1
:10B4300086E495E002C083E495E09F938F938FE1CB
:10B4400098E09F938F931F9287E78F93C501029691
:10B45000A1E0B0E0AC0FBD1F8A0F9B1F9F938F939D
:10B460000E94319CA80EB91EC5010E94FC4E0FB669
:10B47000F894DEBF0FBECDBF892B11F00C94804F26
:10B480000C94B3518091792D90917A2D92FD02C048
:10B490000C94C25121E042E161E080ED0E9404651C
:10B4A0009F938F937F936F9387E298E09F938F93FF
:10B4B0001F9287E78F93C501029621E030E02C0FA1
:10B4C0003D1F820F931F9F938F930E94319CA80E64
:10B4D000B91EC5010E94FC4E0FB6F894DEBF0FBE28
:10B4E000CDBF892B11F00C94804F0C94C2518091E8
:10B4F000792D90917A2D92FD02C00C94D15121E0CA
:10B5000042E162E080ED0E9404659F938F937F93F8
:10B510006F9385E398E09F938F931F9287E78F93B4
:10B52000C5010296A1E0B0E0AC0FBD1F8A0F9B1FC2
:10B530009F938F930E94319CA80EB91EC5010E9453
:10B54000FC4E0FB6F894DEBF0FBECDBF892B11F0B5
:10B550000C94804F0C94D1518091792D90917A2D3B
:10B5600092FD02C00C94E05121E042E163E080EDE5
:10B570000E9404659F938F937F936F9383E498E079
:10B580009F938F931F9287E78F93C501029621E0C7
:10B5900030E02C0F3D1F820F931F9F938F930E94CB
:10B5A000319CA80EB91EC5010E94FC4E0FB6F8943E
:10B5B000DEBF0FBECDBF892B11F00C94804F0C94D1
:10B5C000E0518091792D90917A2D92FD02C00C94DA
:10B5D000EF5121E042E164E080ED0E9404659F9319
:10B5E0008F937F936F9381E598E09F938F931F9242
:10B5F00087E78F93C5010296A1E0B0E0AC0FBD1FB5
:10B600008A0F9B1F9F938F930E94319CA80EB91E97
:10B61000C5010E94FC4E0FB6F894DEBF0FBECDBF31
:10B62000892B11F00C94804F0C94EF518091792D5F
:10B6300082FD02C00C94005246E061E083E00E946B
:10B64000261A0C94005280915C1E8F9380915B1E91
:10B650008F9380915A1E8F938091591E8F938FE5FF
:10B6600098E09F938F931F9287E78F93C50102966F
:10B6700041E050E04C0F5D1F840F951F9F938F9307
:10B680000E94319CA80EB91EC5010E94FC4E0FB647
:10B69000F894DEBF0FBECDBF892B11F00C94804F04
:10B6A00020E030E040E0562D60E070E080E090E087
:10B6B000A0E00E94BB9211F40C9435528091792D38
:10B6C00082FD02C00C9435528091601E8F93809150
:10B6D0005F1E8F9380915E1E8F9380915D1E8F936E
:10B6E00087E698E09F938F931F9287E78F93C5011A
:10B6F0000296E1E0F0E0EC0FFD1F8E0F9F1F9F937D
:10B700008F930E94319CA80EB91EC5010E94FC4E69
:10B710000FB6F894DEBF0FBECDBF892B11F00C948D
:10B72000804F0C9435528091792D90917A2D93FD14
:10B7300002C00C94485280E090E00E9446259F93FE
:10B740008F937F936F9382E798E09F938F931F92DD
:10B7500087E78F93C501029641E050E04C0F5D1FD3
:10B76000840F951F9F938F930E94319CA80EB91E42
:10B77000C5010E94FC4E0FB6F894DEBF0FBECDBFD0
:10B78000892B11F00C94804F0C9448528091792DA4
:10B7900090917A2D93FD02C00C945B5281E090E071
:10B7A0000E9446259F938F937F936F9382E898E042
:10B7B0009F938F931F9287E78F93C5010296E1E0D5
:10B7C000F0E0EC0FFD1F8E0F9F1F9F938F930E9441
:10B7D000319CA80EB91EC5010E94FC4E0FB6F8940C
:10B7E000DEBF0FBECDBF892B11F00C94804F0C949F
:10B7F0005B528091792D90917A2D93FD02C00C942B
:10B800006E5281E090E00E9446252B013C0180E0D1
:10B8100090E00E9446259B01AC01C301B2010E9449
:10B8200043239F938F937F936F9383E998E09F9334
:10B830008F931F9287E78F93C501029641E050E0F6
:10B840004C0F5D1F840F951F9F938F930E94319C17
:10B85000A80EB91EC5010E94FC4E0FB6F894DEBFBB
:10B860000FBECDBF892B11F00C94804F0C946E52FB
:10B870008091792D90917A2D93FD02C00C94815284
:10B8800081E090E00E9446252B013C0180E090E0A1
:10B890000E9446259B01AC01C301B2010E94A42372
:10B8A0009F938F937F936F938EE998E09F938F93ED
:10B8B0001F9287E78F93C5010296E1E0F0E0EC0F5D
:10B8C000FD1F8E0F9F1F9F938F930E94319CA80E88
:10B8D000B91EC5010E94FC4E0FB6F894DEBF0FBE24
:10B8E000CDBF892B11F00C94804F0C948152809124
:10B8F000792D90917A2D93FD02C00C94945281E0A1
:10B9000090E00E9446252B013C0180E090E00E94DF
:10B9100046259B01AC01C301B2010E9405249F93FF
:10B920008F937F936F938CEA98E09F938F931F92EE
:10B9300087E78F93C501029641E050E04C0F5D1FF1
:10B94000840F951F9F938F930E94319CA80EB91E60
:10B95000C5010E94FC4E0FB6F894DEBF0FBECDBFEE
:10B96000892B11F00C94804F0C9494528091792D76
:10B9700090917A2D94FD02C00C94A7520E949D1EB6
:10B980009F938F937F936F938FEB98E09F938F9309
:10B990001F9287E78F93C5010296E1E0F0E0EC0F7C
:10B9A000FD1F8E0F9F1F9F938F930E94319CA80EA7
:10B9B000B91EC5010E94FC4E0FB6F894DEBF0FBE43
:10B9C000CDBF892B11F00C94804F0C94A752E0E06E
:10B9D0000C94F8528091792D85FD02C00C940B5384
:10B9E000E11103C081E00E94B27D609151367091F7
:10B9F000523680915336909154360E945D9420E0E7
:10BA000030E040E85AE30E9457969F938F937F93CC
:10BA10006F9381EE98E09F938F931F9287E78F93A8
:10BA2000C5010296E1E0F0E0EC0FFD1F8E0F9F1FB5
:10BA30009F938F930E94319CA80EB91EC5010E944E
:10BA4000FC4E0FB6F894DEBF0FBECDBF892B11F0B0
:10BA50000C94804FE1E00C940B538091792D85FD7F
:10BA600002C00C941E53E11103C081E00E94B27D1C
:10BA70006091553670915636809157369091583670
:10BA80000E945D9420E030E040E85BE30E9457961E
:10BA90009F938F937F936F9383EF98E09F938F9300
:10BAA0001F9287E78F93C501029641E050E04C0F4B
:10BAB0005D1F840F951F9F938F930E94319CA80E4A
:10BAC000B91EC5010E94FC4E0FB6F894DEBF0FBE32
:10BAD000CDBF892B11F00C94804F0C941E53F701AD
:10BAE00086811F928F9385811F928F9383811F92EE
:10BAF0008F9382811F928F9384E099E09F938F931D
:10BB00001F9287E78F93C501029621E030E02C0F4A
:10BB10003D1F820F931F9F938F930E94319CA80E0D
:10BB2000B91EC5010E94FC4E0FB6F894DEBF0FBED1
:10BB3000CDBF892B11F00C94804F0C943053779A21
:10BB400080912D1490912E14A0912F14B091301447
:10BB500092FD749A80912D1490912E14A0912F141F
:10BB6000B091301482FD0CC08091660280FD08C047
:10BB700081FD02C00C945C531D9902C00C945C536F
:10BB800040E050E060E070E0CE0101960E94FD0EC2
:10BB90008091621E90E0209123143091241482172A
:10BBA000930710F40C945C5340E050E062E180E1B4
:10BBB00092E00E9447730C945C538F2D0E94856C19
:10BBC000739A80912B1490912C14892B11F00E9460
:10BBD000AA6A8091080B8F5F8093080B80912D14C7
:10BBE00090912E14A0912F14B091301482FD02C0B8
:10BBF0000C94804F739A0C94804F653811F00C941C
:10BC00000854A12CB12C0C94B8538CEF9AE00E94EC
:10BC1000D571892B11F40C9408540E94AA6A809162
:10BC2000660287FD02C00C94804F2B9A0C94804FC3
:10BC300020E030E0472D50E060E070E080E090E0F0
:10BC4000A0E00E94BB9211F00C942F520C9435523C
:10BC5000C456DF4F0FB6F894DEBF0FBECDBFDF91E5
:10BC6000CF911F910F91FF90EF90DF90CF90BF90F9
:10BC7000AF909F908F907F906F905F904F903F908C
:10BC80002F9008950C94FD754F925F926F927F9262
:10BC90009F92AF92BF92CF92DF92EF92FF920F935B
:10BCA0001F93CF93DF93CDB7DEB760970FB6F894AD
:10BCB000DEBF0FBECDBF5B010E946D6CE82FF0E0D0
:10BCC000EE0FFF1FEA58F24E808191810196918319
:10BCD000808380912D1490912E14A0912F14B091F7
:10BCE000301481FD74984090660250906702609015
:10BCF0006802709069020E94B0776C01FC0180813B
:10BD0000982F92959F70913099F48F7051F4809193
:10BD10005A1D90915B1D019690935B1D80935A1D57
:10BD20003EC1B50183E698E30E946977892B51F003
:10BD30008091581D9091591D01969093591D8093A3
:10BD4000581D2DC1D301C2013EE0B695A795979528
:10BD500087953A95D1F7F82FF1709F2E8FE19BE0F0
:10BD60000E9420747C01892B09F44BC0B501C701E6
:10BD700002960E946977892B09F43FC087012CEA5B
:10BD80003EE040E054E660E070E0C7010F960E949C
:10BD90005570F6019181F7018481981321C0828545
:10BDA0008F5F82878091561D9091571D01969093C9
:10BDB000571D8093561D84E00E94A078F7012085CE
:10BDC00030E02817390708F07AC184E00E94A07893
:10BDD000F7018087F60180818F70F7018187DFC0CE
:10BDE000F701128684E00E94A078F7018087F601AF
:10BDF00080818F70F701818763C1C7010E948574BC
:10BE0000B1CF88E092E00E94AC747C01892B09F4E8
:10BE1000C6C0B501C70102960E946277F601818112
:10BE20008150F701848380E091E0A0E0B0E0838757
:10BE30009487A587B687128684E00E94A078F701D0
:10BE40008087F60180818F70F7018187B7018FE1CC
:10BE50009BE00E945F7487012CEA3EE040E054E6DC
:10BE600060E070E0C7010F960E94557011E0F60186
:10BE70008181F7018483F60180818F70F7018783C8
:10BE800084E00E94A078F701858383E00E94A07877
:10BE9000F701868387818F3009F010E0F601418039
:10BEA000F7018481481A512C612C712C86E0440CD6
:10BEB000551C661C771C8A95D1F7238534854585EA
:10BEC0005685A0ECB0E00E94EF90BB27A92F982FD9
:10BED000872F480E591E6A1E7B1E43865486658630
:10BEE0007686A501B701C6010E94FD0E8091621EF3
:10BEF00090E020912314309124148217930738F096
:10BF000040E050E062E180E192E00E94477380915E
:10BF1000231490912414029708F44DC08091792D38
:10BF200090917A2D91FF2AC00E945364C601059614
:10BF30000E941F64F60181811F928F93F701868111
:10BF40001F928F9385811F928F938CE299E09F932C
:10BF50008F931F9280E18F93CE0101965C019F9396
:10BF60008F930E94319C82E00E943964C5010E9437
:10BF70001F640FB6F894DEBF0FBECDBF809166027E
:10BF800090916702A0916802B091690297FD4DC03F
:10BF90008091231490912414029708F47AC0809120
:10BFA0002D1490912E14A0912F14B091301481FF74
:10BFB00089C0749A87C08091660290916702A091AF
:10BFC0006802B091690296FFA9CF992009F4A6CF23
:10BFD000F6018081982F9F709230E8F09150807F19
:10BFE000892B808384E19BE00E94425E8091541DF6
:10BFF0009091551D01969093551D8093541D8091ED
:10C000002D1490912E14A0912F14B091301496FFFE
:10C0100085CF739883CF80915A1D90915B1D0196B7
:10C0200090935B1D80935A1D79CF83E49DE120910D
:10C03000431D222309F4ACCF9F938F938FE399E0A4
:10C040009F938F93CE0101963C019F938F930E9403
:10C050006E9C5C01B301C60102960E94449B0F9046
:10C060000F900F900F900F900F90009709F490CFC2
:10C07000EFEFAE1ABE0A8A0D9B1DAC010196FA01C4
:10C0800020812032D1F362E18AE192E00E9447737D
:10C090007FCF112309F483CF82E0809394311092F3
:10C0A000963110929531F0929831E092973144E9AF
:10C0B00051E362E182E492E00E94477370CF912CD9
:10C0C00010E0D5CE60960FB6F894DEBF0FBECDBFA0
:10C0D000DF91CF911F910F91FF90EF90DF90CF9064
:10C0E000BF90AF909F907F906F905F904F9008951A
:10C0F0008115910511F00197F1F70895E0916136EE
:10C10000F091623690818091603689230895E091A4
:10C110005E36F0915F36908180916036892B808306
:10C12000E0916336F0916436908180916036892B7E
:10C13000808308951F93CF93DF93E0915E36F09153
:10C140005F36908180916036809589238083E0916D
:10C150006336F0916436908180916036892B8083BC
:10C160008FE897E00E9478601FB7F894E0916336FB
:10C17000F091643690818091603680958923808328
:10C1800089E091E00E947860E0916136F09162363A
:10C19000D081C09160361FBF789485E896E00E94F8
:10C1A0007860E0916136F0916236808190916036DE
:10C1B000982319F08D2F8C2301C081E0DF91CF915E
:10C1C0001F910895509364364093633670935F36A1
:10C1D00060935E36909362368093613681E001C051
:10C1E000880F2A95EAF7809360360C949A60CF9373
:10C1F000DF93C82FDFB7F894E0916336F09164368F
:10C20000908180916036892B808387E090E00E9446
:10C210007860CC2351F0E0916336F09164369081E0
:10C220008091603680958923808384E390E00E942A
:10C230007860E0916136F09162369081809160364D
:10C24000892309F4C0E085EB90E00E947860E091DA
:10C250006336F091643690818091603680958923B1
:10C260008083DFBF88E790E00E9478608C2FDF91A9
:10C27000CF910895CF93DF93C82FD8E08C2F817092
:10C280000E94F760C6958111C068D150B9F78C2F14
:10C29000DF91CF9108958FEF0C943A61DF92EF9286
:10C2A000FF920F931F93CF93DF93E82E8B010E9491
:10C2B0009A60811135C080EF0E943A61D0E0C0E4FD
:10C2C00088EFD82EDC0E81E00E94F760F82E81E026
:10C2D0000E94F760882319F0FF2071F023C0F1104D
:10C2E0000BC0CE1530F0F801808180FF05C0EC1640
:10C2F00019F0DC2FFF24F3948F2D0E94F760F801D2
:10C3000090819695FF2011F09068F8019083C150BC
:10C31000CD11D9CF0F5F1F4FC111D2CF8D2F03C0C9
:10C320008FEF01C08EEFDF91CF911F910F91FF90A2
:10C33000EF90DF900895EF92FF921F93CF93DF93DA
:10C34000182FEB010E949A60209771F085E50E94FA
:10C350003A617E0188E0E80EF11C89910E943A6101
:10C36000CE15DF05D1F703C08CEC0E943A61812F16
:10C37000DF91CF911F91FF90EF900C943A610F9352
:10C380001F93CF93DF93DB01EC9111969C91119752
:10C39000F0E0F92B803179F4EE7F63E0EE0FFF1FC0
:10C3A0006A95E1F716969C9116976CE070E0691B10
:10C3B0007109E60FF71FF7FF07C091E0EA019883C4
:10C3C000F195E195F10902C0EA011882883279F409
:10C3D00014968C91982F9076903649F086FF02C083
:10C3E000EE7F05C085FF02C0EC7F01C0E87FCF0172
:10C3F00044E0969587954A95E1F7D9018C93EF70C3
:10C40000E801E88380E0DF91CF911F910F910895BB
:10C410000F931F93CF93DF93EC018B01B8018881B9
:10C420000E944E6188839FEF980F9D3F30F4F80182
:10C430009081983211F0903189F7DF91CF911F915F
:10C440000F910895CF93DF93EC010E949A60BE0193
:10C4500084EB0E949B6181E00E94F760C82F0E94DC
:10C460009A6081E0C11101C080E0DF91CF91089511
:10C470001F93CF93DF931F921F92CDB7DEB7182F74
:10C4800069837A830E949A600E947E6069817A81C2
:10C49000882341F084E40E949B61113029F00E94BE
:10C4A000876002C082E001C080E00F900F90DF91B2
:10C4B000CF911F9108955F926F927F928F929F927A
:10C4C000AF92BF92CF92DF92EF92FF920F931F93A2
:10C4D000CF93DF93CDB7DEB729970FB6F894DEBFC1
:10C4E0000FBECDBF5C014B013A0189010E949A60E9
:10C4F000B5018EEB0E949B61CE0101967C016C011F
:10C5000099E0592E5E0C0E944B61F60181936F01F8
:10C510005E12F9CF69E070E0C7010E946881D82EF1
:10C52000811108C09301A401B701F50180810E9427
:10C53000BF6102C083E0D82E8D2D29960FB6F894E6
:10C54000DEBF0FBECDBFDF91CF911F910F91FF9046
:10C55000EF90DF90CF90BF90AF909F908F907F90A3
:10C560006F905F9008950F931F93CF93DF93CDB794
:10C57000DEB72B970FB6F894DEBF0FBECDBF182FD6
:10C58000092F682F792F88E0810F0E943862882355
:10C5900019F084E391E243C06CE872E88EE190E028
:10C5A0000E941A639E01275F3F4FAE01465F5F4FB7
:10C5B000BE01655F7F4F812F902F0E945B628111CA
:10C5C000E8CF88E0E1EEF2E0DE01119601900D92F5
:10C5D0008A95E1F7298541E752E0249FC001259F14
:10C5E000900D112464E670E00E9474908A8594E6B0
:10C5F000899F600D711D1124FE01319688E08E0F18
:10C600009191291303C06F5F7F4F02C08E13F8CF43
:10C610008B85882319F0719561957109CB012B9653
:10C620000FB6F894DEBF0FBECDBFDF91CF911F9143
:10C630000F910895DC01CB0181159105A105B1058C
:10C6400029F081509040A040B040D9F708959B0157
:10C65000AC011092B90060E074E284EF90E00E94B7
:10C660008890DA01C9014097A109B109B695A7954B
:10C67000979587958093B800089594EA9093BC00AD
:10C6800040EA56E861E070E09091BC0097FD07C079
:10C690004150510961097109B9F781E008959091FC
:10C6A000B900987F983011F09031B9F78093BB00B2
:10C6B00084E88093BC0080EA96E8A1E0B0E0209195
:10C6C000BC0027FD05C00197A109B109C1F7E5CF5D
:10C6D0008091B900887F883111F08034F1F680E0D4
:10C6E000089524EA34E844E92093BC009091BC000A
:10C6F00097FFFCCF9091B900987F983011F090315E
:10C7000099F78093BB003093BC009091BC0097FFD9
:10C71000FCCF9091B900987F903211F0983539F4A0
:10C720004093BC009091BC0094FDFCCFDDCF0895F8
:10C730000C943D6384E98093BC008091BC0084FD2F
:10C74000FCCF08958093BB0084E88093BC00809167
:10C75000BC0087FFFCCF9091B900987F81E09832B0
:10C7600009F480E0089584EC8093BC008091BC00C3
:10C7700087FFFCCF8091BB00089584E88093BC00C4
:10C780008091BC0087FFFCCF8091BB000895CF93C0
:10C79000DF93FC017096EC01A991CE01A0933F01BB
:10C7A000CE17DF07C1F780913C018F7D80933C015C
:10C7B00080913C01877F80933C01DB015096FB0117
:10C7C000819180933E01EA17FB07D1F780913C01EC
:10C7D000806880933C0180913D0180FFFCCF4051F7
:10C7E000510980913C01806280933C0180913C0121
:10C7F000877F80933C01141615069CF4FB01819100
:10C8000080933E01EA17FB07D1F780913C018068D5
:10C8100080933C0180913D0180FFFCCF4051510944
:10C82000EACFF901C901409620913E012193E81712
:10C83000F907D1F781E090E0DF91CF9108950F9350
:10C840001F93CF93DF93EC018CE70E9471638CE719
:10C850000E94A2638E01005F1F4F89910E94A26314
:10C86000C017D107D1F7DF91CF911F910F910C9491
:10C870009A63813019F440E050E002C040EC50E08F
:10C8800060E070E08CE790E00C948316813019F43E
:10C890004EE050E002C048E050E060E070E08CE71D
:10C8A00090E00C94831641E050E060E070E08CE78B
:10C8B00090E00E94831664ED74E180E090E00C94B7
:10C8C0001A6348E350E060E070E08CE790E00E947B
:10C8D000831649E350E060E070E08CE790E00E944E
:10C8E000831644E150E060E070E08CE790E00E9445
:10C8F000831648E750E060E070E08CE790E00E942B
:10C9000083164EE550E060E070E08CE790E00E9416
:10C9100083164DE650E060E070E08CE790E00E9406
:10C92000831668E374E38CE090E00E941A634CE0A5
:10C9300050E060E070E08CE790E00E94831641E0F8
:10C9400050E060E070E08CE790E00E94831646E0E3
:10C9500050E060E070E08CE790E00E94831664EDA8
:10C9600074E180E090E00C941A63CF93DF93CDB72D
:10C97000DEB7A2970FB6F894DEBF0FBECDBF81E140
:10C98000EEECF9E0DE01529601900D928A95E1F706
:10C9900081E1EFEDF9E0DE01119601900D928A95AB
:10C9A000E1F70E946164CE0142960E941F6482E01A
:10C9B0000E94396464ED74E180E090E00E941A63A3
:10C9C000CE0101960E941F6460E27CE581E590E063
:10C9D0000E941A6380E00E94466460E27CE581E583
:10C9E00090E00E941A634EE050E060E070E08CE757
:10C9F00090E00E948316A2960FB6F894DEBF0FBE99
:10CA0000CDBFDF91CF910895CF92DF92EF92FF9249
:10CA10000F931F93CF93DF9300D0CDB7DEB7042FD2
:10CA2000122F213061F0223031F0243031F02830E3
:10CA300031F493E005C091E003C092E001C090E0C2
:10CA4000E82FF0E08160F82E0C3009F4E0C00E30E1
:10CA500011F49460DCC0003111F49860D8C0023148
:10CA600009F0D5C0613009F4B7C09C60623011F4A0
:10CA7000906207C0633011F4906403C0643009F41D
:10CA800090669068692F70E023E030E0AE014F5F60
:10CA90005F4FCF010E949B1662E174E380E090E05B
:10CAA0000E941A638F2D0E943D630E94B3638983A5
:10CAB0000E94B3638A83023119F40E94B3638B83AB
:10CAC0000E94B36387FDF1CF0E94BD630E949A6309
:10CAD00062E174E380E090E00E941A638F2D0E946F
:10CAE0003D630E94B36389830E94B3638A830231EA
:10CAF00019F40E94BD638B830E94BD630E949A63F8
:10CB000069812A81023139F5862F90E0A0E0B0E0FA
:10CB10004B81DC019927882730E0322F2227820FB2
:10CB2000931FA11DB11D61FF09C0840F911DA11D9F
:10CB3000B11DBC01CD018C6F9F6F06C0BC01CD0142
:10CB4000640F711D811D911D0E945F9420E83FEFCD
:10CB50004FEF57E41FC070E0762F6627620F711DFC
:10CB6000072E000C880B990B0E945F940C3029F45F
:10CB700020E030EE4FEF54E40DC00E3029F420E0F9
:10CB800038EF4FEF55E406C0003131F420E03EEFBE
:10CB90004FEF56E40E94AB932FE632E143E050E4BE
:10CBA0000E9457966B017C01612F70E080E090E05D
:10CBB0000E945F949B01AC01C701B6010E94AB9338
:10CBC0000F900F900F90DF91CF911F910F91FF90D9
:10CBD000EF90DF90CF9008959C68692F70E023E07C
:10CBE00030E0AE014F5F5F4FCF010E949B1662E1C4
:10CBF00074E380E090E00E941A638F2D0E943D63F1
:10CC00000E94B36389830E94B3638A8356CF6130E5
:10CC100009F02CCF9068692F70E023E030E0AE017E
:10CC20004F5F5F4FCF010E949B1662E174E380E08B
:10CC300090E00E941A638F2D0E943D630E94B363AF
:10CC400089830E94B3638A833BCFCF93E6E4F1E00C
:10CC5000208190818081C081C295C695C695C370A0
:10CC6000207CC20F969596959073C90F82958C7013
:10CC7000C80F1F92CF938CE493E19F938F930E94F0
:10CC8000D99B0F900F900F900F908C2FCF910895FC
:10CC90001F93CF93DF9346E069E180E00E94306903
:10CCA00080E00E9485690E94136804B600FE08C0F7
:10CCB0008BE393E19F938F930E94D99B0F900F90EA
:10CCC00004B601FE08C08AE293E19F938F930E940D
:10CCD000D99B0F900F9004B602FE08C089E193E142
:10CCE0009F938F930E94D99B0F900F9004B603FEE1
:10CCF00008C088E093E19F938F930E94D99B0F9087
:10CD00000F9004B604FE08C08BEF92E19F938F93BF
:10CD10000E94D99B0F900F9080EF99E09F938F9383
:10CD200080EE92E19F938F930E94D99B0E94A27301
:10CD30000E94D37260E070E085EB92E00E94757310
:10CD40000E944970E091340AF091350A19950E94C9
:10CD5000256690E00E94B6690E947A7782E080930F
:10CD60006338809364380E940B6843E658E3BC0143
:10CD70008DEC9BEA0E948A6C0E947B670E94706C1B
:10CD80000E940F680E94976D0E94B978E091AA0AEC
:10CD9000F091AB0A1995E091820AF091830A1995F6
:10CDA000E091740AF091750A19950E94996D182FF7
:10CDB000C091B60AD091B70AFE0119950F900F9055
:10CDC0000F900F90892B49F0FE011995BC0180E866
:10CDD00090E00E946090EB0102C0C0E8D0E00E94A9
:10CDE0006D6C1F921F93DF93CF931F928F9380914F
:10CDF000A90A8F938091A80A8F938091810A8F93BB
:10CE00008091800A8F938EEA92E19F938F930E9484
:10CE1000D99B81EA92E19F938F930E94D99B80E9ED
:10CE200092E19F938F930E94D99B60E070E087ED21
:10CE300092E00E9475738CEB99E00E94D46F88E8B1
:10CE400092E19F938F930E94D99B8DB79EB7429694
:10CE50000FB6F8949EBF0FBE8DBFDF91CF911F918B
:10CE6000089580E880936100109261000E944866F6
:10CE7000C6E7D2E105E612E184E5E82E82E1F82E6C
:10CE800093E4C92E92E1D92E25E3A22E22E1B22EFF
:10CE900004B600FE06C0DF93CF930E94D99B0F908B
:10CEA0000F9004B601FE06C01F930F930E94D99BFA
:10CEB0000F900F9004B602FE06C0FF92EF920E9400
:10CEC000D99B0F900F9004B603FE06C0DF92CF925D
:10CED0000E94D99B0F900F9004B604FE06C0BF922B
:10CEE000AF920E94D99B0F900F9014BE0E94E372E4
:10CEF0000E94A869CDCFDF92EF92FF920F931F930C
:10CF0000CF93DF93CDB7DEB7A0970FB6F894DEBF0F
:10CF10000FBECDBF83E690E00E949E9E182F282F63
:10CF200035EF380F303108F0982F9095291709F414
:10CF300063C08BE593E19F938F930E94D99BE0EAB6
:10CF4000F3E18E010F5F1F4F0F900F90D801D02E8D
:10CF5000E12EF02E88E0800F94919D9331968A13F4
:10CF6000FBCFF89448E050E06FE770E0C8010E9402
:10CF7000A49EE2E9F3E1D8018EE08F0D94919D9398
:10CF800031968A13FBCF4EE050E061E770E0C801B4
:10CF90000E94A49EE8E8F3E12AE02F0D8491D801D5
:10CFA0008D938D0131962A13F9CF4AE050E067E660
:10CFB00070E08D2D9E2D0E94A49E6DEC7BEA81E693
:10CFC00090E00E94BC9E60E070E08FE590E00E94DF
:10CFD000BC9E60E08EE590E00E94AE9E60E070E056
:10CFE00085E690E00E94BC9E1AE16AE175EE83E658
:10CFF00090E00E94BC9E7894812FA0960FB6F89482
:10D00000DEBF0FBECDBFDF91CF911F910F91FF907B
:10D01000EF90DF9008958FE590E00C949E9E8EE552
:10D0200090E00C94969EF8941092B60016BC89E796
:10D0300087BD82E084BD95E095BD95B395BB809397
:10D040006E00789408950F931F936091331470913C
:10D05000341480913514909136140091331410914A
:10D0600034142091351430913614601771078207FB
:10D07000930759F71F910F9108950F931F93609194
:10D080006D3670916E3680916F369091703600914A
:10D090006D3610916E3620916F3630917036601774
:10D0A00071078207930759F71F910F9108951F92F7
:10D0B0000F920FB60F9211240BB60F922F933F933E
:10D0C0004F935F936F937F938F939F93AF93BF9390
:10D0D000EF93FF938091331490913414A091351401
:10D0E000B09136140196A11DB11D80933314909315
:10D0F0003414A0933514B0933614809132148F5F9A
:10D100008093321487FF15C01092321480916D36CF
:10D1100090916E36A0916F36B09170360196A11D38
:10D12000B11D80936D3690936E36A0936F36B09399
:10D13000703680910C388823E1F0809131148F5F34
:10D140008093311487FF15C0109231148091653699
:10D1500090916636A0916736B09168360196A11D10
:10D16000B11D8093653690936636A0936736B09371
:10D1700068360E94E071892B11F00E940171FF91C5
:10D18000EF91BF91AF919F918F917F916F915F913F
:10D190004F913F912F910F900BBE0F900FBE0F90AC
:10D1A0001F9018951F920F920FB60F9211240BB675
:10D1B0000F922F933F934F935F936F937F938F9330
:10D1C0009F93AF93BF93EF93FF938091C600E0913D
:10D1D0007336F0917436309709F01995FF91EF91FD
:10D1E000BF91AF919F918F917F916F915F914F917F
:10D1F0003F912F910F900BBE0F900FBE0F901F907D
:10D2000018951F920F920FB60F9211240BB60F9222
:10D210002F933F934F935F936F937F938F939F933E
:10D22000AF93BF93EF93FF938091CE00E09171365F
:10D23000F0917236309709F01995FF91EF91BF91F7
:10D24000AF919F918F917F916F915F914F913F919E
:10D250002F910F900BBE0F900FBE0F901F9018953F
:10D2600081110EC01092C5006093C40088E98093BC
:10D27000C1004093C2001092743610927336089524
:10D28000813069F41092CD006093CC0088E98093DE
:10D29000C9004093CA0010927236109271360895F8
:10D2A000811107C08091C00085FFFCCF6093C6004C
:10D2B0000895813031F48091C80085FFFCCF6093E0
:10D2C000CE000895CF93C82F8A3031F46DE080915D
:10D2D00037140E94506902C08D3029F06C2F809164
:10D2E00037140E94506980E090E0CF910895811139
:10D2F00005C070937436609373360895813021F4BD
:10D30000709372366093713608958093371483E971
:10D3100092E09093B83A8093B73A089584B7877FA4
:10D3200084BF0FB6F894A8958091600088618093BF
:10D330006000109260000FBE08959FE088E10FB674
:10D34000F894A895809360000FBE909360000895B4
:10D35000A89508950FB6F894A8958091600088610B
:10D3600080936000109260000FBE08950C94759732
:10D370000C94719780917A3690E0089580913901EC
:10D3800081FF09C0809139018D7F8093390189E146
:10D3900090E00197F1F723E040E06FE182E491E053
:10D3A0000E94F46E85E090E00197F1F70895909166
:10D3B000390191FD0AC0282F803108F02FE040E0AC
:10D3C0006FE085E491E00C94F46E0895809139014A
:10D3D00081FD0EC040E06FE181E491E00E94E96EC2
:10D3E000282F2F7E81E090E0213021F080E0089509
:10D3F00080E090E008958091390181FF02C081E0D2
:10D40000089540E06FE181E491E00E94E96E8F3180
:10D4100021F08F7E8150823090F780E008958091D6
:10D42000390181FD04C00E94FB698823C1F308957E
:10D4300010920C388091390181FD8BC00E940F6AD7
:10D440008091390181FD85C00E94BE6980913901BA
:10D45000826080933901809144388823D9F180918A
:10D46000940090919500409155385091563884170A
:10D470009507A0F48091213890912238A09123380B
:10D48000B0912438875F924CAF4FBF4F80932138C3
:10D4900090932238A0932338B0932438209194009D
:10D4A00030919500241B350B8091213890912238C2
:10D4B000A0912338B0912438820F931FA11DB11D74
:10D4C0008093213890932238A0932338B093243846
:10D4D00010924438809146388823D9F18091940085
:10D4E000909195004091593850915A38841795077A
:10D4F000A0F48091293890912A38A0912B38B091CE
:10D500002C38875F924CAF4FBF4F80932938909350
:10D510002A38A0932B38B0932C3820919400309166
:10D520009500241B350B8091293890912A38A091C1
:10D530002B38B0912C38820F931FA11DB11D809301
:10D54000293890932A38A0932B38B0932C38109216
:10D550004638089580910C38882321F00E94FB6999
:10D560000E94186A80E090E0089522E0260F27FFCD
:10D570000CC080910A3890910B38019690930B382B
:10D5800080930A388FEF9FEF0895AB01BC0188E3C9
:10D5900094E10E940A9B80E090E0089540E06FE1F2
:10D5A00081E491E00C94E96E282F40E06FEF86E56E
:10D5B00091E00E94F46E0895CF93DF9398EF980F57
:10D5C000923038F0982F9F7E963019F0893109F00B
:10D5D00049C09091390191FD48C0C82F0E940F6A3F
:10D5E0000E94CE6AD82FC81709F442C0C83029F467
:10D5F000809139010E94BE6927C0C93119F4863172
:10D6000081F404C0C63169F4893159F429E040E05D
:10D610006FE182E491E00E94F46E85E090E0019772
:10D62000F1F72C2F40E06FE182E491E00E94F46E6C
:10D63000D83031F48FEF0E94D46A81ED92E002C0BD
:10D6400085E090E00197F1F70E94CE6A8C1781F097
:10D65000C63019F4813079F40BC0C63161F48131E0
:10D6600051F406C082E490E008C084E490E005C074
:10D6700080E490E002C083E490E0DF91CF910895D0
:10D68000809194009091950090935A3880935938E6
:10D6900081E08093463880930C389091390191FF56
:10D6A0001EC02091940030919500309356382093FD
:10D6B000553880934438809307382FB778948091F9
:10D6C0003901809139018D7F8093390180E197E2A2
:10D6D00030910738332311F00197D1F72FBF86E13E
:10D6E0000E94DC6A0C940F6A80910C38811102C090
:10D6F0000E94406B81E090E008950F931F93CF93B9
:10D70000DF931F92CDB7DEB780910C38882361F08C
:10D710008091390181FF02C080E07BC00E94FB69DB
:10D720008823D1F300E003C00E94746B01E0809174
:10D73000940090919500909354388093533811E061
:10D740001093433880E88093550186E00E94DC6A9C
:10D7500010937B368FB7898378941092470180911C
:10D760007B368111FCCF89818FBF8091470111E009
:10D770008E3008F010E0119586E10E94DC6A10926C
:10D780005501809143388823D9F18091940090917C
:10D790009500409153385091543884179507A0F460
:10D7A00080911D3890911E38A0911F38B09120387B
:10D7B000875F924CAF4FBF4F80931D3890931E38B8
:10D7C000A0931F38B0932038209194003091950099
:10D7D000241B350B80911D3890911E38A0911F3865
:10D7E000B0912038820F931FA11DB11D80931D3869
:10D7F00090931E38A0931F38B0932038109243386E
:10D8000001110E94AA6A812F829586958695837060
:10D81000817090E00F90DF91CF911F910F9108954B
:10D820008FEF80934E0121E044E060EF8CE691E0C1
:10D830000E94F46E25E041E06EE08CE691E00E94EB
:10D84000F46E80E880936F018091460180936D01B2
:10D8500021E045E060E284E491E00C94F46ECF9323
:10D86000DF93C9EFD7E0CE010197F1F70E94E86E90
:10D8700010928136109203371092853710928036BD
:10D8800010927F36E9E3F1E080818E7F8083808192
:10D890008D7F808381EC93E00197F1F78081816037
:10D8A000808323E040E06FE182E491E00E94F46E27
:10D8B0002197F1F780915D0180915E010E94106CCB
:10D8C00060E070E081EA92E00E9475730E94406B14
:10D8D00081E090E0DF91CF9108958091B91408958F
:10D8E000CF93DF931F92CDB7DEB789830E940F6A73
:10D8F00089818093B914282F40E06FE188E491E09A
:10D900000F90DF91CF910C94F46E0E94706C86E0C2
:10D910000C94DC6AEF92FF920F931F93CF93DF93E7
:10D920001F921F92CDB7DEB78C017A017F936F9360
:10D930001F938F938AE09AE09F938F9369837A83F2
:10D940000E94C59B009362011093630169816093FB
:10D9500060017A81709361010F900F900F900F908A
:10D960000F900F90E114F104C9F0F70180818093CA
:10D970006B01818180936A01828180936901838137
:10D98000809368018481809367018581809366011B
:10D990008681809365018781809364010F900F9049
:10D9A000DF91CF911F910F91FF90EF90089581EA41
:10D9B00092E00E94967381E080937A3680917C3663
:10D9C00090917D36019690937D3680937C3681E0F0
:10D9D00090E008950F931F93CF9320918036C2E873
:10D9E000C29F90011124F901EF57F94C4081442363
:10D9F00009F451C047FD09C0433038F050E08A01B6
:10DA0000025011096017710710F4108244C0B90167
:10DA10006E57794C0E940A9B80918036C89FF00116
:10DA20001124EF57F94CDF01A058BF4F9C91909300
:10DA3000753610828F5F833018F48093803602C071
:10DA400010928036E091803682E8E89FF001112440
:10DA5000EF57F94C8081882319F00E94D76C02C0DF
:10DA600010927A368091470180937636909179367C
:10DA7000992311F0891710F48093793660917636E6
:10DA800070E084E00E9495786091753670E083E0E4
:10DA90000E94957802C000E010E0C801CF911F916C
:10DAA0000F9108950F931F93CF93DF931F92CDB7DC
:10DAB000DEB78C01FC0180819181009709F18334EC
:10DAC000954029F0F8011182108283E02AC0623863
:10DAD000E1F40E9441788FB78983F8940E94B0776F
:10DAE00060E870E00E94EA6C29812FBF18161906C1
:10DAF00074F40E94AB77E091B00AF091B10A1995E5
:10DB000083E495E0F8019183808381E00AC08091ED
:10DB10007736909178360196909378368093773661
:10DB2000EFCF0F90DF91CF911F910F9108950C943B
:10DB3000D7698091390181FD06C040E06FE085E43E
:10DB400091E00C94E96E80E10895EF92FF921F93AB
:10DB5000CF93DF931F92CDB7DEB7182F8091390195
:10DB600081FD07C00E940F6A80910C3881111CC092
:10DB70005AC080919400909195009093563880936C
:10DB8000553881E08093443880930738809139017B
:10DB90008D7F8093390180E197E22091073822231D
:10DBA00009F30197D1F7DECF809146388823D9F168
:10DBB00080919400909195004091593850915A3835
:10DBC00084179507A0F48091293890912A38A09164
:10DBD0002B38B0912C38875F924CAF4FBF4F80935A
:10DBE000293890932A38A0932B38B0932C38209161
:10DBF000940030919500241B350B80912938909129
:10DC00002A38A0912B38B0912C38820F931FA11D78
:10DC1000B11D8093293890932A38A0932B38B09364
:10DC20002C381092463889E10E94DC6A86E00E9416
:10DC3000A078892B51F00E94996DE82E86E00E9411
:10DC4000A07881500E94D76902C0E12CF12C80910C
:10DC5000940090919500909358388093573881E0C4
:10DC6000809345388FB78983F89480913901826019
:10DC700080933901809139018D7F8093390162E071
:10DC8000610F88E394E10E943B6F89818FBF80918F
:10DC90000838909109380196909309388093083894
:10DCA0000E940F6A45E060EE82E491E00E94E96E16
:10DCB000182F86E00E94A078892B19F08E2D0E94E3
:10DCC000D769809145388823D9F18091940090914B
:10DCD0009500409157385091583884179507A0F413
:10DCE0008091253890912638A0912738B091283816
:10DCF000875F924CAF4FBF4F809325389093263863
:10DD0000A0932738B0932838209194003091950043
:10DD1000241B350B8091253890912638A091273807
:10DD2000B0912838820F931FA11DB11D8093253813
:10DD300090932638A0932738B0932838109245380E
:10DD400080910C38882371F0809194009091950017
:10DD500090935A388093593881E0809346380E94D6
:10DD6000406B02C00E94186A123028F48CE00E94B6
:10DD7000A07810E00BC0133031F0153031F01730BF
:10DD800029F411E003C012E001C013E0812F90E0FC
:10DD90000F90DF91CF911F91FF90EF900895CF9357
:10DDA000DF93EB010E94B56A009729F4CE010E942F
:10DDB000A56D009751F020910A3830910B382F5FF4
:10DDC0003F4F30930B3820930A38DF91CF9108955D
:10DDD0000895FC0180816823862F90E002C095950C
:10DDE00087954A95E2F70895CF93DF931F92CDB7B9
:10DDF000DEB7FC01922F8FB78983F8942081362FEC
:10DE00003095522F5323292F01C0220F4A95EAF74C
:10DE10002623252B208389818FBF0F90DF91CF91FF
:10DE20000895CF93DF93E0917B012DEF2E0F2D37D7
:10DE300040F0FC011082E058FF4F108231961082B2
:10DE400017C0EC01E993A0E8B1E020E82E0F3C9167
:10DE5000399311962A13FBCFE150F0E0E058FE4FC2
:10DE60002181FC01E058FF4F2083319681E08083BF
:10DE7000DF91CF91089560938001E1E8F1E061586E
:10DE8000DC012D91CD01208331966E13F9CF0895D9
:10DE90001F920F920FB60F9211240BB60F922F9371
:10DEA0003F934F935F936F937F938F939F93AF9322
:10DEB000BF93EF93FF9380914701809376368091D3
:10DEC0007F3622E8829FC00111248F57994C0E940F
:10DED000116F80917F368F5F833018F480937F3687
:10DEE00002C010927F360E94D76CFF91EF91BF91D4
:10DEF000AF919F918F917F916F915F914F913F91E2
:10DF00002F910F900BBE0F900FBE0F901F90189582
:10DF10001F920F920FB60F9211240F900FBE0F9009
:10DF20001F9018951F920F920FB60F9211240F9009
:10DF30000FBE0F901F9018951F920F920FB60F9261
:10DF400011240F900FBE0F901F9018951F920F92E3
:10DF50000FB60F921124109207380F900FBE0F903A
:10DF60001F9018951F920F920FB60F9211241092C6
:10DF70007E360F900FBE0F901F9018951F920F9234
:10DF80000FB60F9211240F900FBE0F901F9018958F
:10DF90001F920F920FB60F92112410927B360F90A2
:10DFA0000FBE0F901F901895CF93DF93EC018991CE
:10DFB0009991009729F060E070E00E947573F7CFA7
:10DFC000DF91CF910895EF92FF920F931F93CF931C
:10DFD000DF938C017A01FC0180819181009741F0EF
:10DFE0008A34910511F1F8011182108283E04AC050
:10DFF0008BEB94E10E942074EC01209761F04E813C
:10E000005F8168857985CE0102960E94B77109907B
:10E01000D881C02DF2CF81E08093BA148AE490E0D9
:10E02000F8019183808381E02DC06838E1F78BEBA4
:10E0300094E10E942074EC01209781F3CE010296B6
:10E04000E816F906D9F4BE018BEB94E10E94407406
:10E05000E0906F15F09070158E859F8590937015E8
:10E0600080936F15E889F989309719F08A899B891F
:10E070001995F0927015E0926F15D0CF0990D88164
:10E08000C02DDACFDF91CF911F910F91FF90EF90CC
:10E0900008951092BA148BEB94E10E941C7460E016
:10E0A00070E08BEA92E00C947573EF92FF920F93FD
:10E0B0001F93CF93DF93EC01E0906F15F0907015F4
:10E0C000FF86EE86398B288B1B8B0A8B8091BA14C6
:10E0D000882379F08BEA92E09093701580936F1506
:10E0E000CE0102960E94B771F0927015E0926F1502
:10E0F00004C04E835F8368877987BE018BEB94E110
:10E100000E944074BE018BEB94E1DF91CF911F918F
:10E110000F91FF90EF900C945F74CF93DF93EC011D
:10E120008091BA14882329F0CE0102960E94EB71E7
:10E1300004C01B861A861D861C86BE018BEB94E1EB
:10E14000DF91CF910C944074CF92DF92EF92FF92C7
:10E150000F931F938091C1149091C214892B49F49D
:10E160001092BD141092BE141092BF141092C014DD
:10E1700041C00E9423688B019C01E091C114F09181
:10E18000C214448155816681778180819181A28109
:10E19000B381840F951FA61FB71F801B910BA20B85
:10E1A000B30B0084F185E02D3097C1F0C480D58099
:10E1B000E680F78040815181628173814C0D5D1D45
:10E1C0006E1D7F1D401B510B620B730B48175907C7
:10E1D0006A077B0730F7DB01CA01E3CF800F911F8D
:10E1E000A21FB31F8093BD149093BE14A093BF14BD
:10E1F000B093C0141F910F91FF90EF90DF90CF90DC
:10E20000089585EB92E00C949673EF92FF920F9332
:10E210001F93CF93DF938C01FC0180819181009744
:10E2200099F089359105D9F0F8011182108283E0C7
:10E2300068C0828593858417950709F049C00084DA
:10E24000F185E02D3097A9F71092C2141092C114F5
:10E2500089E590E0F8019183808381E052C06738BE
:10E2600091F16238A9F7C091C114D091C214E12C88
:10E27000F12C209769F3CE010E94F173892BF1F004
:10E28000AE0168E88A859B850E944773892BA1F4BB
:10E290001B861A8688859985E114F10421F0F7011F
:10E2A0009187808704C09093C2148093C11419860B
:10E2B00018860E94A470D7CF0E9401717E01088445
:10E2C000D985C02DD6CFE091C114F091C214BACF38
:10E2D000F093C214E093C114A085B185109709F49E
:10E2E000B7CF1A968D919C911B978417950739F497
:10E2F00018968D919C91199791878087EDCFFD019C
:10E30000EBCFDF91CF911F910F91FF90EF90089588
:10E31000CF93DF93EC010E9401712A853B85909198
:10E32000C1148091C214232B91F0E92FF82F30975C
:10E3300071F0EC17FD0739F480916F15909170150D
:10E340009387828710C00084F185E02DF0CF209163
:10E350006F15309170153B872A8798878987D093EE
:10E36000C214C093C114DF91CF910C94A470CF93C9
:10E37000DF93EC010E94C373CE01DF91CF910C9427
:10E380008871CF93DF93EC010E94D373CE01DF91AC
:10E39000CF910C948871CF93DF93EC010E94E573C9
:10E3A000CE01DF91CF910C94887121E030E0FC0127
:10E3B00082859385892B11F020E030E0C901089512
:10E3C00081E090E02091C1143091C214232B11F40C
:10E3D00080E090E00895CF93DF93EC01E091C114C9
:10E3E000F091C2148E179F0769F4888599859093E0
:10E3F000C2148093C1140DC0808591858C179D0730
:10E4000021F0FC013097C1F706C088859985918776
:10E4100080870E94A470198618861B861A86DF9151
:10E42000CF9108951F93CF93DF93DC011496ED9164
:10E43000FC9115973097E1F0162FEC019093701531
:10E4400080936F1582E08887CD0106961995082E76
:10E45000000C990B0297029710F0133839F4BE01A3
:10E46000CE01DF91CF911F910C94427281E0888799
:10E47000DF91CF911F910895FC01208520FD0C9420
:10E4800012720895CF92DF92EF92FF920F931F9333
:10E49000CF93DF93E0906F15F0907015C0907115D9
:10E4A000D0907215F601E817F90739F0309709F4A2
:10E4B0004BC00190F081E02DF6CF009709F444C0E5
:10E4C0008B01EC018885882309F11886C114D104D9
:10E4D00061F0CC15DD0529F0AE0167E8C6010E94A8
:10E4E0003C72F601C080D180F1CFEC81FD81309784
:10E4F00069F0C017D10751F0D0937015C0936F1514
:10E5000040E050E063E8CE0106961995E091711560
:10E51000F0917215CE17DF0741F4888199819093AD
:10E520007215809371150CC0FC01309749F0808101
:10E5300091818C179D07C1F7888199819183808390
:10E54000F0927015E0926F15DF91CF911F910F91AE
:10E55000FF90EF90DF90CF9008951F93CF93DF93BC
:10E560001092CB14C0917115D091721511E02097C3
:10E5700079F08985882341F01887198640E050E0BA
:10E5800062E8CE010E9412720990D881C02DEFCFAF
:10E59000DF91CF911F91089580916E1591E0980FB2
:10E5A00090936E1508958AE880936E1510926C15FD
:10E5B00010926D15109272151092711510927015BF
:10E5C00010926F1508958091CB1481110E94AD7245
:10E5D00050916D15552309F452C0E0916C152E2F02
:10E5E00030E085E0E89FF0011124E453FB4E6081A8
:10E5F0006093CA14A181B281B093C914A093C814C6
:10E60000838194819093C7148093C6142F5F3F4FEA
:10E610002F71332720936C15515050936D1500972F
:10E6200031F580917115909172159093C514809376
:10E63000C4148091C4149091C514892B01F1809168
:10E64000CB1481110E94AD724091C8145091C9142D
:10E650006091CA148091C4149091C5140E943C72B8
:10E66000E091C414F091C51480819181DECF6138AE
:10E6700019F421E0FC012087AD010E943C728091D9
:10E68000CB1420916D1590E0820F911D08959C018F
:10E6900090916D159032B9F0E0916C15E90FEF7122
:10E6A000E093C31485E0E89FF0011124E453FB4E8E
:10E6B000608352834183348323839F5F90936D15DE
:10E6C00080E090E0089581E090E00895CF93DF939B
:10E6D000C0916F15D09170150E943C72D093701547
:10E6E000C0936F15DF91CF910895AB0130917115F3
:10E6F00020917215E32FF22FE817F907B1F0309748
:10E7000021F00190F081E02DF7CF009771F0FC012E
:10E7100030832183909372158093711521E02087B7
:10E720001782168261E80C9466730895009749F089
:10E73000FC0120852150223020F421E02187209304
:10E74000CB1408950C94F8818091731590917415F1
:10E750000097C1F01092741510927315DC01149695
:10E760006D917C9115971296ED91FC9113971995E7
:10E77000E0917315F0917415309721F080819181AB
:10E780000C9412820895CF93DF93EC014C835D8348
:10E790006E837F830E942368688379838A839B8347
:10E7A000DF91CF910895FC01408151816281738195
:10E7B00084819581A681B781840F951FA61FB71FFD
:10E7C00080839183A283B3830895CF93DF93EC0179
:10E7D0000E942368688379838A839B83DF91CF912A
:10E7E0000895CF92DF92EF92FF92CF93DF93EC01E7
:10E7F0000E942368C880D980EA80FB80DC01CB01BD
:10E800008C199D09AE09BF090196A11DB11D21E01A
:10E8100030E0CC80DD80EE80FF80C816D906EA06A5
:10E82000FB0610F020E030E0C901DF91CF91FF90AE
:10E83000EF90DF90CF900895FC011182108208952F
:10E84000FC01808191810895DC01ED91FC9130976C
:10E8500041F080819181009711F0FC01FACFCF0146
:10E86000089580E090E00895DC01ED91FC9111970E
:10E87000309721F0208131812D933C93CF01089571
:10E88000DC01ED91FC913097C9F0A0E0B0E0E61713
:10E89000F70761F4FB0120813181109709F4DC0155
:10E8A0002D933C93FB0111821082089520813181C8
:10E8B000DF012115310511F0F901E9CF08950F931A
:10E8C0001F93CF93DF938C01EB010E944074198258
:10E8D0001882C8010E942474009711F4F80101C045
:10E8E000FC01D183C083DF91CF911F910F910895D7
:10E8F000DC01ED91FC9180E090E0309729F00196E9
:10E900000190F081E02DF9CF0895009721F0FC01EE
:10E9100080819181089580E090E00895CF93DF9306
:10E92000EC014A815B8160E070E08C819D810E94F6
:10E93000139B2A813B8188819981289FA001299F6F
:10E94000500D389F500D112460E070E08E819F8142
:10E95000DF91CF910C94139BFC018281938120E085
:10E9600030E028173907D1F0A481B581A20FB31F79
:10E970004C91411110C081E08C9380819181289F3E
:10E98000A001299F500D389F500D11248681978139
:10E99000840F951F08952F5F3F4FE3CF80E090E0F5
:10E9A0000895FC01868197814281538120E030E007
:10E9B00024173507D1F08617970781F4A481B58114
:10E9C000A20FB31F8C91181614F481508C9384817C
:10E9D0009581FC01E20FF31F80810895A081B18130
:10E9E0008A0F9B1F2F5F3F4FE3CF8FEF0895FC01EE
:10E9F0002681378162177307A0F0A081B18142811F
:10EA00005381A49FC001A59F900DB49F900D112428
:10EA1000280F391F81E090E06217730720F080E033
:10EA2000089580E090E008952F923F924F925F9278
:10EA30006F927F928F929F92AF92BF92CF92DF920E
:10EA4000EF92FF920F931F93CF93DF93CDB7DEB773
:10EA500068970FB6F894DEBF0FBECDBFEDE0F8E3C8
:10EA600024A535A546A557A550A441A432A423A4A6
:10EA7000948C858C768C678C808D8983918D9A831C
:10EA8000828D8B83938D9C8384898D8395899E83CE
:10EA900086898F83978998878089898791899A87C2
:10EAA00082898B8793899C8784858D8795859E87AE
:10EAB00086858F879785988B8085898B91859A8BA2
:10EAC000B284A384F480E580D680C78080818F8B58
:10EAD0009181988F128103812B8B3C8B4D8B5E8BA8
:10EAE0000E943D685E895F934D894F933C893F93B7
:10EAF0002B892F932F923F924F925F926F927F922A
:10EB00008F929F922C812F932B812F932A812F9369
:10EB100029812F9328852F932F812F932E812F9337
:10EB20002D812F932C852F932B852F932A852F931F
:10EB300029852F9328892F932F852F932E852F9307
:10EB40002D852F93AF92BF922A892F9329892F93D6
:10EB5000CF92DF92EF92FF920F931F93288D2F9306
:10EB60002F892F939F938F937F936F93E3E6F8E31F
:10EB700081811F928F9380811F928F9388EA93E106
:10EB80009F938F930E94D99B0FB6F894DEBF0FBE60
:10EB9000CDBF68960FB6F894DEBF0FBECDBFDF9134
:10EBA000CF911F910F91FF90EF90DF90CF90BF908A
:10EBB000AF909F908F907F906F905F904F903F901D
:10EBC0002F900895EF92FF920F931F93CF93DF93AF
:10EBD0008C01EB017A010E947876F801F086E782D9
:10EBE00063E67AE0CE01DF91CF911F910F91FF9004
:10EBF000EF900C949C760C9480760C943477DC0126
:10EC00001796ED91FC9118970190F081E02D3097C7
:10EC100009F019940895DC011796ED91FC9118976D
:10EC20000280F381E02D309709F019940895DC01FA
:10EC30001996ED91FC911A970280F381E02D30979F
:10EC400009F0199408950F931F93CF93DF931F92A8
:10EC50001F92CDB7DEB78C0188E10E94B378BC016A
:10EC6000CE0101960E946277D8011996ED91FC9130
:10EC70001A970190F081E02D309729F0BE016F5F67
:10EC80007F4FC80119950F900F90DF91CF911F9181
:10EC90000F910895EF92FF920F931F93CF93DF93FD
:10ECA0008C01EB017A0145E65AE00E94E275F80119
:10ECB000F286E18669E67AE0CE01DF91CF911F917D
:10ECC0000F91FF90EF900C949C760C94FB75CF9372
:10ECD000DF93EC0163E678E388E10E94A978CE0136
:10ECE000DF91CF910C94FD7585E795E10C941C7430
:10ECF000FC0173836283BC0185E795E10C945F742A
:10ED0000BC0185E795E10C944074CF93DF93EC014F
:10ED100085E795E10E942074009749F0FC0122816B
:10ED200033812C173D0729F00E948574F5CF80E0D0
:10ED300090E0DF91CF9108950F931F93CF93DF93CE
:10ED40008B010E948576EC01892B31F01D830C83A9
:10ED5000C8010E94C58B8E83DF91CF911F910F91C7
:10ED60000895CF92DF92EF92FF920F931F93CF936C
:10ED7000DF937C018B016A0187E795E10E94207493
:10ED8000EC01892B51F0EC81FD81309711F0C80125
:10ED90001995CE010E948574F3CFA601B801C70171
:10EDA000DF91CF911F910F91FF90EF90DF90CF9067
:10EDB0000C940B760F931F93CF93DF931F921F92A8
:10EDC000CDB7DEB70E94978B8C0187E795E10E9453
:10EDD0002074009779F0DC011296ED91FC91139765
:10EDE000309729F089839A8319959A8189810E94A5
:10EDF0008574EFCF0115110549F0C8010F900F90F0
:10EE0000DF91CF911F910F910C94FF750F900F9090
:10EE1000DF91CF911F910F910895CF92DF92EF92E2
:10EE2000FF920F931F930E94B9780E9441780E942D
:10EE30002C8A0E94958BC12C88E0D82E87E0E82E82
:10EE4000F12C00E01EE120E030E040E052E060E024
:10EE500070E082E090E00E945C8B1F910F91FF9028
:10EE6000EF90DF90CF900895CF93DF93EC010E9455
:10EE7000AA8B009761F00E94C977E091840AF09113
:10EE8000850ABE0181EB96E7199581E090E0DF915C
:10EE9000CF910895E091AC0AF091AD0A1994E091F8
:10EEA000760AF091770A1994E091B20AF091B30AC8
:10EEB0001994E091B40AF091B50A199480E090E0B9
:10EEC00008950895FB0120813181FC013183208365
:10EED000089542E050E00E94FD9A21E030E0892B45
:10EEE00011F020E030E0C9010895BC0183E698E309
:10EEF0000C946277E091340AF091350A1995E0910B
:10EF0000AA0AF091AB0A1995E091820AF091830A5E
:10EF10001995E091740AF091750A199420913016B0
:10EF2000309131162817390798F040912E165091DC
:10EF30002F16480F591F50932F1640932E16281B3B
:10EF4000390B309331162093301681E090E008950C
:10EF500080E090E0089590933116809330160895E4
:10EF600080912E1690912F1685559A4E0895809176
:10EF70002D1690E085589A4E089581E090E02091FA
:10EF8000791530917A152B5A354111F480E090E0D3
:10EF900008950E94BD77892B61F060917915709179
:10EFA0007A1540913016509131168BEA95E10C9408
:10EFB0000A9B20912E1630912F1621153105B9F09C
:10EFC0008091301690913116C096EBEAF5E1AF01D1
:10EFD0004B5755414817590734F4DF01A20FB31FAF
:10EFE0004C914193F4CF10922F1610922E16089543
:10EFF0008091301690913116089580912D1690E3EE
:10F00000981B2091301630913116A901490F511DDE
:10F01000CA0108950F931F93CF938C01C0912D16B1
:10F020008C2F90E0801791076CF00E94FD77800F85
:10F03000911F8138910530F4C01BC0932D1681E0DB
:10F0400090E002C080E090E0CF911F910F91089571
:10F05000CF93DF93EDE6F8E31192119288E3ED3957
:10F06000F807D1F7C5E6D8E36EE87AE0CE010E9452
:10F070006277229688E3CD36D807B1F7DF91CF913A
:10F08000089510922F1610922E161092311610928B
:10F09000301680E380932D168BEA95E190937A15D4
:10F0A000809379150C942878EF92FF920F931F9319
:10F0B000CF93DF931F921F92CDB7DEB78C01698388
:10F0C0007A830E9441786981E62E7A81F72E81E861
:10F0D000E816F10418F080E8E82EF12CA701B80139
:10F0E0008091791590917A150E940A9BF0923116C1
:10F0F000E0923016C7010F900F90DF91CF911F91D2
:10F100000F91FF90EF900895FC0190E3ADE6B8E316
:10F1100001900D929A95E1F788E0FB01A5E6B8E32E
:10F1200001900D928A95E1F70895E82FF0E0EE0F37
:10F13000FF1FE359F74C7183608381E090E00895ED
:10F14000E82FF0E0EE0FFF1FE359F74C808191812B
:10F15000089590E0880F991F8B5C974C0E9462770E
:10F1600081E090E0089590E0880F991F8B5C974CA8
:10F1700008958FEB92E00E948E748FEC92E00E94D3
:10F180008E7487EC92E00C948E740F931F93CF9340
:10F19000DF93EC01BC018FEC92E00E94F774892BA5
:10F1A000A9F00990D881C02DFE0161917191CF0124
:10F1B0000E945478BE016E547F4FCE018E579F4FF0
:10F1C000DF91CF911F910F910C948478BE0187EC51
:10F1D00092E00E94F774892BD1F00E9441786881F7
:10F1E00079818A819B810E9454788CA990E00E9449
:10F1F0000A780CA910E00E94B777BE016C5F7F4FC0
:10F20000A801DF91CF911F910F910C940A9BDF9180
:10F21000CF911F910F91089585EA9CE10E94D571CD
:10F22000892B21F085EA9CE10C94CB710895E09143
:10F23000911CF091921C309709F0199480E0089588
:10F24000EF92FF920F931F93CF93DF938C01EA010C
:10F25000FC0180819181009741F08A33934081F1D4
:10F26000F8011182108283E0F8C080E024E0829FE0
:10F27000F0011124ED56F34E118210828F5F84301D
:10F28000A9F78093901C80916F15909170159093C1
:10F29000A41C8093A31C0E94CC7280939D3840E4F0
:10F2A00050E060E070E085EA9CE10E94B7710E9446
:10F2B000D9828AE393E0F8019183808381E0CDC015
:10F2C0006230D9F480919E3890919F38892B89F3D0
:10F2D0008091AF38863029F48091C73881FD0E9433
:10F2E0000C7981E00E94208380919E3890919F3814
:10F2F000892BF9F20E947A7ADCCF633060F56111D4
:10F3000014C02097B1F2D0939C39C0939B3983E00D
:10F310000E94208380919E3890919F38892B11F014
:10F320000E9417790E940C79C4CF613011F62097A2
:10F3300009F4BFCFD0939839C093973985E00E94E4
:10F34000208380919E3890919F38892B09F4B1CF0A
:10F350000E941779AECF673809F040C010928F1C19
:10F3600083E9E82E8CE1F82E80918F1C8430C0F464
:10F37000F701828193818C179D0749F480819181E7
:10F380000E940583F7011182108213821282F4E039
:10F39000EF0EF11C80918F1C8F5F80938F1CE4CF48
:10F3A000E6EBF9E3838194818C179D0719F41482AD
:10F3B00013821082B0962AE3E633F20799F7E3E36B
:10F3C000FAE3818592858C179D0711F415821482CA
:10F3D0003D968AE3E53BF807A1F76BCF683809F063
:10F3E00068CFC55ADC4109F064CF85EA9CE10E94F0
:10F3F000D571892B09F45DCF10928F1CE0918F1C81
:10F40000E43008F056CF20E2E29FF0011124E356E9
:10F41000F64C818D8823D9F085EA9CE10E94CB715E
:10F4200080918F1CE0E28E9FC00111248356964C80
:10F4300090939C3980939B3982E00E942083809135
:10F440009E3890919F38892B11F00E9417798091F6
:10F450008F1C8F5F80938F1CD1CFDF91CF911F9135
:10F460000F91FF90EF900895CF93DF93A0919B3978
:10F47000B0919C39109719F0ED016C9605C0C091C0
:10F480009739D091983929968091963986FF23C073
:10F4900010928E1C80E0E3E9FCE18430C1F04081F1
:10F4A000518114962D913C9115974217530761F4A1
:10F4B000228133812115310539F080938E1C3983E7
:10F4C00028831B821A8205C034968F5FE6CF809313
:10F4D0008E1C0E940C7988819981009741F04A81A5
:10F4E0005B8160919D38DF91CF910C946673DF91C1
:10F4F000CF9108950F931F93CF93DF938091AF38EF
:10F50000863009F07AC080919E3890919F38803F74
:10F51000910508F472C08897EC01D695C7959E01B5
:10F52000220F331F8E012817390710F40F5F1F4F6A
:10F53000CE01889690939F3880939E389093A838F8
:10F540008093A9381092CB381092CA380E94D38287
:10F55000809590959093CB388093CA381092B138AB
:10F560001092B0380E94C282809590959093B138E5
:10F570008093B0380E941779C801889690939F387D
:10F5800080939E389093A8388093A93880919939B8
:10F5900090919A39BC016C0F7D1FA8010E940A9BB3
:10F5A000BE018EEB98E30E946F828091A238809317
:10F5B000BE388091A3388093BF388091A43880935F
:10F5C000C0388091A5388093C1381092CB38109202
:10F5D000CA380E94D382809590959093CB388093BF
:10F5E000CA381092B1381092B0380E94C282809509
:10F5F00090959093B1388093B038DF91CF911F915F
:10F600000F910C941779E091440AF091450A1994EE
:10F6100080E090E00895AF92BF92CF92DF92EF9298
:10F62000FF920F931F93CF93DF93CDB7DEB7E19790
:10F630000FB6F894DEBF0FBECDBF7C016B01CE01CB
:10F6400001965C0181E3F50111928A95E9F781E069
:10F6500089838CE00E94A0788C831D821F82809118
:10F66000B11C91E0980F9093B11C898713E0188723
:10F670008DEC9BEA9B878A8789E10E94B3786EE8CC
:10F680007AE00E946977892B31F082E08E838FEFD8
:10F690008C878D8709C089E10E94B378BC01CE01B7
:10F6A0000C960E9462771E838DEC9BEA9D8B8C8B5F
:10F6B00063E678E3CE0146960E9462770E94B077B7
:10F6C0009FA78EA70E94F87799AB88ABC5010E94CF
:10F6D0000D8C8C011127C8010E940A78892B31F109
:10F6E0000E94B777A801BC01C5010E94308C00912F
:10F6F0003A0A10913B0A0E94FD775C010E94B7779D
:10F70000B501F8011995E114F10481F0009739F081
:10F71000019761F441E050E064E070E004C041E032
:10F7200050E060E070E0C601F7011995E1960FB670
:10F73000F894DEBF0FBECDBFDF91CF911F910F9127
:10F74000FF90EF90DF90CF90BF90AF9008950F9310
:10F750001F93CF93DF934115510579F0FA018B0187
:10F76000EC01828193810E94C578B801CE01DF91BE
:10F77000CF911F910F910C940B7BDF91CF911F9133
:10F780000F9108950F931F93CF93DF93CDB7DEB7FB
:10F79000E1970FB6F894DEBF0FBECDBF0E94F87799
:10F7A0008C010E94B077AE014F5F5F4FB8010E949D
:10F7B000238D892B09F443C088A999A99801281B96
:10F7C000390BC9010E948E77892BC9F18E81811175
:10F7D0000CC0BE016A5E7F4F88E10E94A978E0916B
:10F7E000860AF091870A19952AC02A853B852D3C07
:10F7F0009BEA390719F02F3F3F4F09F5823019F086
:10F8000088E090E002C082E090E0019710F3E1E030
:10F81000F0E0EC0FFD1FE80FF91F23852F3FA9F340
:10F82000BE01645F7F4F89E10E94A97889E10E944F
:10F83000B37863E678E30E946977892B51F6E19605
:10F840000FB6F894DEBF0FBECDBFDF91CF911F91F1
:10F850000F9108950E94B8698093B11CE091440A09
:10F86000F091450A1994892B29F0E091440AF0910E
:10F87000450A04C0E091460AF091470A19948F9214
:10F880009F92AF92BF92CF92DF92EF92FF92E2EB04
:10F89000FCE1408151814A01A12CB12C6B017C011A
:10F8A00024E0F594E794D794C7942A95D1F7C81823
:10F8B000D908EA08FB08DC01CB0133E0B595A79530
:10F8C000979587953A95D1F7B501A401440F551F37
:10F8D000661F771F4C015D01841A950AA60AB70AB4
:10F8E000A5019401A281B3810E94FA904B015C01B1
:10F8F0003BE0B594A794979487943A95D1F7A701E4
:10F900009601C701B6010E9444909B01AC016CE0D6
:10F9100055954795379527956A95D1F7A481B58177
:10F920000E94FA90DC01CB017EE0B595A7959795F2
:10F9300087957A95D1F7A5019401280F391F4A1FA1
:10F940005B1F21A332A343A354A3A5E0B0E00E9410
:10F95000EF90DC01CB0180589F4FAF4FBF4F692F15
:10F960007A2F8B2F992787FD9A95FF90EF90DF9044
:10F97000CF90BF90AF909F908F900895EF92FF929D
:10F980001F93CF93DF93CDB7DEB76A970FB6F89486
:10F99000DEBF0FBECDBF182F21E030E0CE010196B3
:10F9A0007C01AC0160ED70E08EEE90E00E949B1651
:10F9B0008981803609F0CAC046EB50E060EE70E005
:10F9C0008EEE90E00E94831668E374E38CE090E092
:10F9D0000E941A638AE1F70111928A95E9F72AE1F8
:10F9E00030E0A70168E870E08EEE90E00E949B1680
:10F9F0008A8190E0982F88272981822B9093B31CCD
:10FA00008093B21C8C8190E0982F88272B81822BC9
:10FA10009093B51C8093B41C8E8190E0982F88271A
:10FA20002D81822B9093B71C8093B61C888590E023
:10FA3000982F88272F81822B9093B91C8093B81C14
:10FA40008A8590E0982F88272985822B9093BB1C6C
:10FA50008093BA1C8C8590E0982F88272B85822B69
:10FA60009093BD1C8093BC1C8E8590E0982F8827B6
:10FA70002D85822B9093BF1C8093BE1C888990E0BB
:10FA8000982F88272F85822B9093C11C8093C01CB0
:10FA90008A8990E0982F88272989822B9093C31C0C
:10FAA0008093C21C8C8990E0982F88272B89822B09
:10FAB0009093C51C8093C41C8E8990E0982F882752
:10FAC0002D89822B9093C71C8093C61C288D30E013
:10FAD000322F22278F89282B3093C91C2093C81CD2
:10FAE0008A8D8093CA1C28E030E0A70161EE70E0A7
:10FAF0008EEE90E00E949B162A8130E0322F222762
:10FB00008981282B3093CC1C2093CB1C8B81809334
:10FB1000CD1C8C81F0E18F9FC00111242D812F70AD
:10FB2000822B9093CF1C8093CE1C8F8120E1829FEB
:10FB3000C00111242E812F70822B9093D11C8093B1
:10FB4000D01C88858093D21C1093D71C6A960FB660
:10FB5000F894DEBF0FBECDBFDF91CF911F91FF9014
:10FB6000EF9008952F923F924F925F926F927F9203
:10FB70008F929F92AF92BF92CF92DF92EF92FF92BD
:10FB80000F931F93CF93DF93CDB7DEB7AD970FB62B
:10FB9000F894DEBF0FBECDBF9E012F5F3F4F7901AE
:10FBA00098E0F90111929A95E9F7813009F077C34D
:10FBB0008091D71C813009F072C341E050E062EFC0
:10FBC00070E08EEE90E00E94831640E050E065EF1A
:10FBD00070E08EEE90E00E94831646E250E064EF03
:10FBE00070E08EEE90E00E9483160CE211E021E0BE
:10FBF00030E0AE01475F5F4F64EF70E08EEE90E063
:10FC00000E949B16898583708987882351F06AE654
:10FC10007AE080E090E00E941A630150110939F700
:10FC20003EC328E030E0A70167EF70E08EEE90E081
:10FC30000E949B16E981E8A7FA81F9A72B812AA7E0
:10FC4000CF80D12CE12CF12CFE2CED2CDC2CCC2403
:10FC50008885C82A6D81862F90E0A0E0B0E0AC01D5
:10FC6000BD01E4E0440F551F661F771FEA95D1F7E9
:10FC70008C8190E0A0E0B0E0FCE0880F991FAA1F03
:10FC8000BB1FFA95D1F7842B952BA62BB72B2E8172
:10FC900022952F70BC01CD01622B0E943F7C6093A6
:10FCA0004D3670934E3680934F36909350368090F9
:10FCB000D31C9090D41CA090D51CB090D61C2401CD
:10FCC00035013CE2531A31E0630A7108AEE0CC0C16
:10FCD000DD1CEE1CFF1CAA95D1F78091CE1C9091E3
:10FCE000CF1C092E000CAA0BBB0B14E1880F991F27
:10FCF000AA1FBB1F1A95D1F7C81AD90AEA0AFB0A2C
:10FD0000A091D01CB091D11CA30192010E94FA9045
:10FD1000C61AD70AE80AF90A40E4D40EE11CF11C1D
:10FD20000FE0F594E794D794C7940A95D1F7A09182
:10FD3000D21C0A2E000CBB0BA30192010E94FA9068
:10FD40009B01AC018AE055954795379527958A9593
:10FD5000D1F72A873B874C875D87A091CD1CB0E007
:10FD6000A30192010E94EF90DC01CB012BE0B5953D
:10FD7000A795979587952A95D1F7BC01CD01705825
:10FD80008F4F9F4F2A853B854C855D850E9444900F
:10FD9000DC01CB013AE0B595A795979587953A9503
:10FDA000D1F79C01AD01405E5F4FA091CB1CB0919B
:10FDB000CC1C0E94FA90DC01CB01905EAF4FBF4F8C
:10FDC000BC01CD014EE095958795779567954A954D
:10FDD000D1F7A70196010E9444906B017C015FE07E
:10FDE00095958795779567955A95D1F79B01AC01C5
:10FDF0000E9444909B01AC0167E05595479537956B
:10FE000027956A95D1F7A091CA1CB0E00E94EF90A7
:10FE1000DC01CB0174E0B595A795979587957A9508
:10FE2000D1F7A7019601281B390B4A0B5B0BDA01AE
:10FE3000C90157FF03C080E090E0DC0181309105EB
:10FE4000A10539E1B30724F080E090E0A0E0B9E13A
:10FE50002CE0B595A795979587952A95D1F780932E
:10FE6000513690935236A0935336B0935436750161
:10FE70006401FF0CCC08DC2C76019401A5016C2DEB
:10FE80007C2D8C2D9C2D345F4140510961097109F5
:10FE9000810991092A873E874F87588B698B7A8B16
:10FEA0008B8B9C8B59016A017B018C010E94029112
:10FEB00028A339A34AA35BA36CA37DA38EA39FA30E
:10FEC0004091C21C4BA75091C31C5D8B8091C01CFC
:10FED0008CA7E091C11CEE8BF091BE1CFDA7209178
:10FEE000BF1C2F8BB090BB1CA090BA1C1B2D110FF8
:10FEF000110BC12ED12EE12EF12E012F2A853E8528
:10FF00004F85588969897A898B899C890E940291D9
:10FF10000CE00E945D9219012A013B014C01B09056
:10FF2000BD1CA090BC1C1B2D110F110BC12ED12E7E
:10FF3000E12EF12E012F28A139A14AA15BA16CA1CC
:10FF40007DA18EA19FA10E94029108E00E9476925D
:10FF500051016201730184010E94949270588F4F85
:10FF60009F4F2090B81C3090B91C5101C12CD12C4E
:10FF7000E12CF12C00E010E00E94029101E20E94CD
:10FF80007692288F398F4A8F5B8F6C8F7D8F8E8F03
:10FF90009F8FA0E00E94BB9209F475C1ABA41D899C
:10FFA000110F110BBD88C12ED12EE12EF12E012F84
:10FFB00028A139A14AA15BA16CA17DA18EA19FA11D
:10FFC0000E94029119012A013B014C01ACA41E8937
:10FFD000110F110BBE88C12ED12EE12EF12E012F53
:10FFE0002A853E854F85588969897A898B899C89BC
:10FFF0000E94029101E10E945D9259016A017B0118
:020000021000EC
:100000008C019101A201B301C4010E9494921901D3
:100010002A013B014C01F9A54F2F50E060E070E050
:10002000E4E0440F551F661F771FEA95D1F78AA5B4
:1000300082958F708A019B01082B88A5482F50E07C
:1000400060E070E0DB01CA01FCE0880F991FAA1F85
:10005000BB1FFA95D1F7B901A801482B592B6A2B80
:100060007B2B80E090E0A0E1B0E0841B950BA60B19
:10007000B70B6C017D01FF0CCC08DC2C76019C01D8
:10008000AD016C2D7C2D8C2D9C2D0FE10E945D927D
:10009000B22FA32FF42FE52F6A877E878F87988B47
:1000A0002DA59F89990F990B3F89492F592F692FAA
:1000B000792F892F03E20E945D9259016A017B0129
:1000C0008C019101A201B301C4010E9494925901D3
:1000D0006A017B018C012B2F3A2F4F2F5E2F6A85EF
:1000E0007E858F8598890E94A99239014A01B62F91
:1000F000A72FF82FE92F03E00E945D9253016401BE
:10010000EB2EFA2E0F2F1E2F0E94A99259016A0181
:100110007B01582E192F03E00E945D92052D0E944D
:10012000A99203E00E945D9253016401EB2EFA2E26
:100130000F2F1E2F0E94A99202E00E945D920F2FA6
:100140000E94A99201E00E945D920F2F0E94A99245
:10015000A88CB98CCA8CDB8CEC8CFD8C0E8D1F8D21
:100160000E9488912A873E874F87588B698B7A8BAC
:100170008B8B9C8B0DE00E947692922E832E742E98
:10018000652E562E472E382E292E3091C91C2091CF
:10019000C81C932F990F990BA92CB82CC72CD62CBF
:1001A000E52CF42C032D122D492F592F692F792F6F
:1001B000892F0E9402910E94029109E10E94769289
:1001C00059016A017B018C012A853E854F8558893A
:1001D00069897A898B899C890E94949219012A01E4
:1001E0003B014C013091C71C2091C61C932F990FE5
:1001F000990BAA84BE84CF84D888E988FA880B89B1
:100200001C89492F592F692F792F892F0E9402911C
:1002100003E10E94769259016A017B018C019101F0
:10022000A201B301C4010E94949208E00E94769258
:10023000322E432E542E652E762E872E982EB92FD1
:100240003091C51C2091C41C932F990F990B492FF5
:10025000592F692F792F892F04E00E945D9259014F
:100260006A017B018C01232D342D452D562D672DE0
:10027000782D892D9B2F0E949492722F632F942F9B
:10028000852F9B0104C030E020E090E080E03093B7
:100290005536209356369093573680935836AD9600
:1002A0000FB6F894DEBF0FBECDBFDF91CF911F9187
:1002B0000F91FF90EF90DF90CF90BF90AF909F9005
:1002C0008F907F906F905F904F903F902F90089508
:1002D000FC01680F791F80E048E1E617F70781F01D
:1002E000219198E0322F3827532F517030FD842709
:1002F0008695513009F480682695915099F7EDCF95
:1003000008951F920F920FB60F9211240BB60F9201
:100310002F933F934F935F936F937F938F939F930D
:10032000AF93BF93EF93FF938091940090919500CA
:100330009093503880934F3881E08093413880917A
:100340007100807D809371000E94A4738091413878
:100350008823D9F1809194009091950040914F3875
:100360005091503884179507A0F4809115389091DA
:100370001638A0911738B0911838875F924CAF4F5C
:10038000BF4F8093153890931638A0931738B093C9
:1003900018382091940030919500241B350B8091E2
:1003A000153890911638A0911738B0911838820FEF
:1003B000931FA11DB11D8093153890931638A093FB
:1003C0001738B093183810924138FF91EF91BF91D0
:1003D000AF919F918F917F916F915F914F913F91DD
:1003E0002F910F900BBE0F900FBE0F901F9018957E
:1003F0009FB7F894E1E7F0E08081807D808388B347
:100400008F6288BB10929000E1E9F0E010821092B8
:1004100092001092950010929400808185608083F4
:100420009FBF08959C019FB7F89430939900209343
:10043000980088B38F6288BBE1E7F0E0808182603A
:1004400080839FBF0895FB0141505109460F571FFC
:10045000E417F50778F4208130E0322F22276181FC
:10046000260F311D820F931F8217930708F4019600
:100470003296EECFE417F50751F4208130E0322FA9
:100480002227820F931F8217930708F4019608957D
:10049000CF93DF93C091A938D0E064972091A8381A
:1004A00030E0322F2227C20FD31F48E050E062EB2A
:1004B00078E39E01280F311DC9010E942382AE01FD
:1004C0006AEB78E30E942382009721F0982789271E
:1004D000982702C08FEF9FEFDF91CF910895FC0125
:1004E0002381260F2093A538A72FBB2792819A0F2F
:1004F0009093A43831813093A33840814093A2383F
:10050000E92FF0E0EA17FB0748F481E0830F8093BE
:10051000A338811103C04F5F4093A23830E07727A2
:100520002617370788F49F5F9093A43891110CC069
:100530008091A3388F5F8093A338811105C080918B
:10054000A2388F5F8093A238089520919B39309113
:100550009C39BC01C90108960E946F82E0919B39C9
:10056000F0919C39A2EAB8E38C91808711968C9126
:100570001197818712968C911297828713968C918E
:100580008387089544E150E066EA78E380E090E0F4
:100590000E942382009721F09827892798270895A1
:1005A0008FEF9FEF089586E00C94488281E10C94D0
:1005B000488280E0E82FF0E0EE0FFF1FE35EF54C8D
:1005C000118210828F5F8430A9F780E090E2899FCA
:1005D000F0011124E356F64C118E8F5F8430B1F791
:1005E00080E094E09093DD1C8093DC1C80E09DE033
:1005F000989FF0011124ED5CF54C158214828F5FF9
:100600008A30B1F78093DB1C08959C0190E0943010
:10061000A1F0E92FF0E081E0890FEE0FFF1FE35E0C
:10062000F54C408151814217530729F49093DB1C0C
:10063000118210820895982FEACF9093DB1C0895C1
:10064000AF92BF92CF92DF92EF92FF920F931F93E0
:10065000CF93DF93C0919B39D0919C39843009F4BA
:10066000DBC12EEC38E330939A39209399393093DB
:10067000A1382093A038833059F4898D8F7083304E
:1006800009F06AC088899989892B09F0D4C67EC08F
:10069000823009F07FC08091E11C8F5F8093E11C64
:1006A000811113C08091E01C8F5F8093E01C811149
:1006B0000CC08091DF1C8F5F8093DF1C811105C00F
:1006C0008091DE1C8F5F8093DE1C10929F38109209
:1006D0009E381092323A1092313A898D982F9D7F30
:1006E000953041F48A8D8F5F8A8F843109F0A3C6DB
:1006F000198EA1C6882309F49EC628893989232B1F
:1007000009F440C09A8D2FEF290F2A8F911193C6BB
:100710009B8D983031F02FEF280F223048F4953020
:1007200039F4198E80E8809396390E94347A3DC559
:10073000953038F423E0092E01C0220F0A94EAF71D
:1007400001C020E32A8F9F5F9B8F8F708330A1F0C1
:1007500048F4813009F444C3823009F06CC6109229
:10076000C73841C3863009F4BCC4883009F4B9C421
:10077000843009F060C6B5C484E0809396390E9445
:10078000347A45C58F70833009F055C688E0809370
:10079000963900C5853019F5E0919739F09198396F
:1007A00084819581892B09F446C610929C39109258
:1007B0009B3982EC98E390939A398093993990937E
:1007C000A1388093A0381092323A1092313A1092A8
:1007D0009F3810929E3888E0809396391BC1809193
:1007E000A638853409F027C60091A83810E0102FEC
:1007F00000278091A938080F111D80919E38909193
:100800009F388017910708F416C610939F380093FD
:100810009E388091AC388F7309F00DC6F090AD38DA
:10082000F11009C680912D3A90912E3AC091B80AE4
:10083000D091B90A8C179D0759F440912F3A5091E5
:10084000303A2091BA0A3091BB0A42175307A1F0FF
:100850002091B6383091B7382817390709F0EBC521
:100860002091B8383091B93880912F3A9091303A30
:100870002817390709F0DFC50E94C282019609F0E6
:10088000DAC58091AF38863009F429C18131E9F1A8
:10089000813009F0D0C58091BA38883009F0CBC5D5
:1008A0001092BA388091BC389091BD38873F6FEF75
:1008B000960710F0099601C008969093BD38809372
:1008C000BC388091B2389091B338A091B438B091CF
:1008D000B5388093B6389093B738A093B838B093B2
:1008E000B93880912D3A90912E3AA0912F3AB0913B
:1008F000303A8093B2389093B338A093B438B09321
:10090000B53880E48093AE3873C50C51110910934B
:100910009F3800939E3882EC98E390939A398093A5
:1009200099398091C0389091C138892B29F00E9463
:10093000D682019609F07FC52091BC383091BD3830
:100940002115310509F477C583E39AE3909398392B
:1009500080939739A090BA38B090BB384091BC0AC8
:100960005091BD0A6091BE0A7091BF0AA091B23841
:10097000B091B3380091B4381091B538E090BA0A0C
:10098000F090BB0AE0919739F09198398AE3E53B02
:10099000F80708F050C584819581009721F1281748
:1009A000390709F586819781009719F0A816B906CD
:1009B000D1F4808191818C179D0729F4C280D38066
:1009C000CE14DF04B1F08417950729F4C280D380D8
:1009D000C616D70671F0A817B90729F4828193814A
:1009E0000817190731F03D96F0939839E09397393D
:1009F000C9CF10929C3910929B3982E0809396392E
:100A000082EC98E39093A1388093A0381092323A08
:100A10001092313A0E94347A8091313A9091323A70
:100A2000009709F408C59C01245E3F4F30939F381E
:100A300020939E383093A8382093A938E0919739B5
:100A4000F091983920852093AE3821E12093AF387A
:100A500008969827892798279093BF388093BE38A7
:100A60001092C1381092C038848195819093BB3820
:100A70008093BA38868197819093BD388093BC3833
:100A800080912D3A90912E3AA0912F3AB091303A20
:100A90008093B2389093B338A093B438B093B538FC
:100AA00080819181A281B3818093B6389093B738C9
:100AB000A093B838B093B9388EEC98E390939A39F4
:100AC000809399390E94D68280959095009711F471
:100AD0008FEF9FEF9093C1388093C03889C40E94F4
:100AE000D382019609F0A7C44091BC385091BD381B
:100AF0004115510509F49FC48091BA389091BB38D3
:100B0000009709F498C46091B2387091B338E091BD
:100B1000B438F091B538CDE9D9E3298D2223A9F075
:100B2000AC81BD814A175B0781F4AE81BF818A1712
:100B30009B0759F4A881B9816A177B0731F4AA8110
:100B4000BB81EA17FB0709F466C1A0962AE3CD3101
:100B5000D20719F78091C7388F738230D9F4509338
:100B6000D91C4093D81C80E0843091F0E82FF0E04D
:100B7000EE0FFF1FE35EF54C208131818F5F42173E
:100B8000530791F71092DB1C80E0C0E0D0E07CC0FE
:100B90008093DB1C8091C73882FD4DC484E1809333
:100BA000C73888E290E090939F3880939E3880E524
:100BB0008093C6383091C1388091C5388093C13850
:100BC0002091C0388091C4388093C0382093C438B5
:100BD0009091BF388091C3388093BF389093C338C9
:100BE0008091BE388093DB1C4091C2384093BE3860
:100BF0008093C2383F5F3093C53831110DC02F5FED
:100C00002093C438211108C09F5F9093C33891117D
:100C100003C08F5F8093C2388091BA389091BB38FF
:100C20009093D91C8093D81C2091BC383091BD384A
:100C30003093BB382093BA389093BD388093BC383A
:100C40008091B2389091B338A091B438B091B53852
:100C50008093B6389093B738A093B838B093B9382A
:100C600080912D3A90912E3AA0912F3AB091303A3E
:100C70008093B2389093B338A093B438B093B5381A
:100C80009CC3973089F08F5F8430C1F060E2869F0B
:100C900090011124F901E356F64C918D9111F1CF99
:100CA0008093DB1CEF010CC0209721F0428D9A8DC0
:100CB000941748F7E901C356D64CE5CF8093DB1C67
:100CC000209709F4B8C3D0939C39C0939B3983E033
:100CD0008A8F888F1E8A84E08F8B1B8E8091BC3810
:100CE0009091BD389D838C838091BA389091BB38A8
:100CF0009F838E838091B2389091B338A091B4389D
:100D0000B091B53888839983AA83BB8381E0898FAA
:100D10008091DE1C8C878091DF1C8D878091E01C88
:100D20008E878091E11C8F8781E090E0998B888B82
:100D30008091C1388B878091C0388A878091BF3875
:100D400089878091BE38888781E090E00E94A582E3
:100D50008091C638982F907F913508F441C08295D4
:100D60008F7090E00597880F991F880F991F209129
:100D7000DA1CEF2DF0E0E817F90774F5EA55F74CA7
:100D800020A5211103C01092DA1C28C0213011F4D3
:100D9000F394EFCF2230D9F431A53430C1F420934D
:100DA000DA1CF092DB1C82A590E0982F882723A5FF
:100DB000822B9093D91C8093D81C893C910510F00C
:100DC00088EC90E09B8B8A8B9D8B8C8B09C031A526
:100DD000332311F0F30ECDCF2093DA1CF092DB1CFD
:100DE00080E18093C7388091C73882608093C7388C
:100DF00082E08093CE3884E08093CF381092D03850
:100E000088EC8093D1388CE290E090939F38809367
:100E10009E3880E680C2D0939C39C0939B39109253
:100E200096398091C738782F7470F72E82FF03C0EF
:100E3000198E80E219C29091C63892959F70990FD1
:100E4000990F9093DB1C091B110904511109109390
:100E50009F3800939E38922F9F70923029F4982FDC
:100E60009F73923139F41FC0913021F4982F9F73F2
:100E70009230C9F0012B19F4982F9370A1F02091B2
:100E8000BE38988529133DC22091BF389985291312
:100E900038C22091C0389A85291333C22091C138B5
:100EA0009B8529132EC284FF49C068897989611501
:100EB000710509F443C0CE010C960E946F823091F7
:100EC000C2388091A238381339C02091C33880913C
:100ED000A338281333C09091C4388091A438981354
:100EE0002DC08091C5384091A538841327C03C8718
:100EF0002D879E878F878B8D811119C09E89888D44
:100F00002A8D821B292F269526952695821B980FC0
:100F10009E8B87FD81952F89322F36953695231B21
:100F2000820F8F8B969596959695890F888F81E085
:100F300080939639888D8A8F198A188A298DE22F95
:100F4000EF708E2F90E0FC013197E830F10508F04A
:100F500072C28827E656FF4F8F4F0C94C99080913C
:100F6000963980FF14C083E0898F80E4809396399E
:100F7000198A188A80919E3890919F38009709F4B9
:100F800005C122E4209396390E94A582FFC080917A
:100F9000C7388F73823009F04EC222CF80919639C4
:100FA00080FF6AC08091C7388F73823109F064C0B6
:100FB0008091C638982F907F913508F441C0829572
:100FC0008F7090E00597880F991F880F991F2091C7
:100FD000DA1CEF2DF0E0E817F90774F5EA55F74C45
:100FE00020A5211103C01092DA1C28C0213011F471
:100FF000F394EFCF2230D9F431A53430C1F42093EB
:10100000DA1CF092DB1C82A590E0982F882723A59C
:10101000822B9093D91C8093D81C893C910510F0A9
:1010200088EC90E09B8B8A8B9D8B8C8B09C031A5C3
:10103000332311F0F30ECDCF2093DA1CF092DB1C9A
:1010400083E0898F8091BE3888878091BF388987F7
:101050008091C0388A878091C1388B8781E090E089
:101060000E94A58282E480939639198A188A109288
:101070009F3810929E388AC080E2809396390E94F1
:10108000347AE0919B39F0919C39118E83CD809117
:10109000C73880FF28C024FD26C088899989892BFC
:1010A00009F0C9C180919E3890919F3801960E94A5
:1010B000A58280919639982F9061909396392091CE
:1010C0009E3830919F38232B19F082618093963996
:1010D0000E94347A81E090E0998B888B88E0898F38
:1010E0001B8E81E10FC185FF1DC08091CC3890E03F
:1010F000982F88273091CD38832B40919939509182
:101100009A39480F591F50939A3940939939409111
:101110009E3850919F38BA01681B790B70939F38A5
:1011200060939E3840919E3850919F3841155105EB
:1011300051F024FD08C090919639926090939639B1
:10114000CA010E94A5828091C83890E0982F882714
:101150002091C938820F911D9093D91C8093D81C7F
:101160002C893D892817390710F0892B21F43093F9
:10117000D91C2093D81C8091D81C9091D91C9B8B92
:101180008A8B80919639837009F455C11092323A56
:101190001092313A0E94347A8091963985FF07C0C7
:1011A0001092323A1092313A198E84E1ABC084FF2A
:1011B0000AC01092323A1092313A81E090E0998B55
:1011C000888B84E08CCF2091313A3091323A2115CE
:1011D0003105E1F080FF02C0198A188A888999894F
:1011E000009781F48A899B898217930720F4909352
:1011F000323A8093313A8091313A9091323A998BD8
:10120000888B04C09093323A8093313A1B8E809140
:10121000A0389091A13890939A3980939939809110
:10122000313A9091323A892B59F0888999890097FF
:1012300039F0889690939F3880939E3888E10BC050
:101240008091963981FFF7C088E290E090939F38B3
:1012500080939E3880E18093C7385CC08091963936
:1012600080FFE9C0198E80E1809396390E94347A1C
:10127000E2C080919E3890919F38009711F00E94B3
:10128000A5829091C7388091963990FF0BC080FF5E
:1012900006C087E0898F1A8E198A188A19C086E0DD
:1012A000898F16C080FF1EC085E0898F198A188A31
:1012B000C2C080919E3890919F38009711F00E9493
:1012C000A5828091C73880FF0DC087E0898F1A8E74
:1012D00081E090E00E94A58280E1809396390E948F
:1012E000347A0FC080919E3890919F38892B49F4B1
:1012F000A2C08091963980FF9EC087E0898F1A8EA8
:101300009AC080E18093C73888E290E090939F383C
:1013100080939E3880E58093C63888858093C23854
:1013200089858093C3388A858093C4388B85809360
:10133000C5388C858093BE388D858093BF388E8567
:101340008093C0388F858093C13886E08093AF3812
:101350008C819D819093BB388093BA388E819F8118
:101360009093BD388093BC3880912D3A90912E3A5D
:10137000A0912F3AB091303A8093B2389093B3381D
:10138000A093B438B093B53888819981AA81BB8184
:101390008093B6389093B738A093B838B093B938E3
:1013A000898D84FF05C01092C9381092C83805C0D5
:1013B0001092C83888EC8093C93880E48093AE38A6
:1013C00080919E3890919F389093A8388093A93847
:1013D0001092CD381092CC381092CB381092CA3877
:1013E0000E94D382809590959093CB388093CA3891
:1013F00085E48093A6381092A7381092AD381092E9
:10140000AC388091E21C9091E31C01969093E31C10
:101410008093E21C9093AA388093AB381092B13835
:101420001092B0380E94C282809590959093B13806
:101430008093B03804C010929F3810929E3810925A
:101440009639DF91CF911F910F91FF90EF90DF9030
:10145000CF90BF90AF90089586EE9CE10C941C74E1
:101460009093E51C8093E41C089586EE9CE10C9417
:101470002074EF92FF920F931F93CF93DF938C0111
:10148000EB017A0186EE9CE10E9420740097D9F06E
:10149000DC0112962D913C9113972C173D0781F496
:1014A0001696ED91FC911797309769F09701AE0170
:1014B000B801DF91CF911F910F91FF90EF90199498
:1014C0000E948574E3CFDF91CF911F910F91FF9020
:1014D000EF90089508950F931F93CF93DF93C7E282
:1014E000DDE1488159816A817B8100E010E025E9D6
:1014F0003AE887E09DE10E9455700E94B869BC01FE
:1015000080E090E0288139814A815B810E94889047
:10151000AB01BC012AEB3AE883EF9CE10E945570D5
:10152000DF91CF911F910F9108958091271D909188
:10153000281DA091291DB0912A1D4091231D509175
:10154000241D6091251D7091261D880F991FAA1FCB
:10155000BB1F481759076A077B0710F4DB01CA0154
:101560008093271D9093281DA093291DB0932A1DB9
:101570000C946B8ACF93DF930E9441780E94B077DE
:10158000EC01198218820E94358A288139810097DE
:1015900019F1FC0140854423F9F0FC01428153819B
:1015A000F901EE0FFF1FEE0FFF1FEC0FFD1F53831E
:1015B0004283FC01448155812F5F3F4FF901EE0FBB
:1015C000FF1FEE0FFF1FEC0FFD1F51834083398378
:1015D00028830E948574D9CFC901880F991F880F6D
:1015E000991F02960E94AB7788819981892B31F0EF
:1015F00088EE9CE1DF91CF910C946776DF91CF91DB
:101600000895AF92BF92CF92DF92EF92FF920F9325
:101610001F93CF93DF931F921F92CDB7DEB75B016D
:101620000E94B0778C01FC01E080F180FA82E982AF
:101630000E94F8779701220F331F220F331F2E5F6E
:101640003F4F8217930798F0C12CD12CCE14DF04A2
:1016500071F0F8014481558162817381C5010E9456
:10166000398AFFEFCF1ADF0A0C5F1F4FEFCF0F90C1
:101670000F90DF91CF911F910F91FF90EF90DF902E
:10168000CF90BF90AF9008950F93013099F480915F
:101690001B1D90911C1DA0911D1DB0911E1D8093BE
:1016A000271D9093281DA093291DB0932A1D0F91EB
:1016B0000C946B8A0F9108954F925F926F927F9274
:1016C0008F929F92AF92BF92CF92DF92EF92FF9252
:1016D0000F931F932A013B014801590140EC5AE046
:1016E000BC0188EE9CE10E944A76E8EEFCE143AA48
:1016F00054AA65AA76AA87AA90AEA1AEB2AEC3AE2E
:10170000D4AEE5AEF6AE84E49BE81F910F91FF9056
:10171000EF90DF90CF90BF90AF909F908F907F9091
:101720006F905F904F900C94308A0C947476CF93A6
:10173000DF93E091C40AF091C50A1995EC01892B59
:1017400029F06A817B8181E00E949578CE01DF914A
:10175000CF9108950F931F93CF93DF93EC01E09106
:10176000C60AF091C70A19958C016A817B8181E0D4
:101770000E94957881E090E0012B11F480E090E0E8
:10178000DF91CF911F910F910895E091C80AF091D8
:10179000C90A1994CF93DF93FC01DB0185E0EB01CB
:1017A00019928A95E9F78581837011F082E08C9314
:1017B0008781837021F082E012968C931297858145
:1017C000837081F08781837069F0238934898185F2
:1017D00092852817390731F481E0848312961C9290
:1017E000129701C0148285818370823029F0833082
:1017F00011F488E001C080E011968C9311978781E5
:101800008370823029F0833011F488E001C080E0D9
:1018100013968C93DF91CF910895CF93DF9300D0EF
:101820001F921F92CDB7DEB7BE016F5F7F4F0E9440
:10183000CA8B898190E003962A81820F911D2B81AA
:10184000820F911D2C81820F911D2D81820F911D80
:101850000F900F900F900F900F90DF91CF91089500
:101860003F924F925F926F927F928F929F92AF9230
:10187000BF92CF92DF92EF92FF920F931F93CF937D
:10188000DF9300D01F921F92CDB7DEB78C017B0192
:101890003A01BE016F5F7F4F0E94CA8B69817A81D6
:1018A000472F50E0EB813C80232D30E0862F90E0E5
:1018B0000396840F951F8E0F911D820F931FAD818C
:1018C0008A0F911D681679060CF4A4C0D8011196F0
:1018D0008C91119780FB882480F8912C83E0880CF0
:1018E000991C8A95E1F712968C91129780FBAA2495
:1018F000A0F8B12C94E0AA0CBB1C9A95E1F78A28B9
:101900008C918770882A13968C91139780FBCC2436
:10191000C0F8D12CF5E0CC0CDD1CFA95E1F7C82815
:1019200014968C9180FB442440F8512CA6E0440C82
:10193000551CAA95E1F74C28D7014C92D801159671
:101940008C918370B4E08B9F60011124D8011696AE
:101950009C919370B0E19B9FC00111248C29D80108
:101960001796FC9190E4F99FD00111248A2BD7019E
:1019700011968C93D80118968C91D70112968C935E
:10198000623071F4D80119968C91D70113968C931B
:10199000D8011A968C91D70114968C9385E001C0DA
:1019A00083E0780F872F972F941B4115510561F025
:1019B00041505109D801A40FB51F1B968C91D70136
:1019C000A90FB11D8C93EECFE23071F4D701A70FB0
:1019D000B11DF80193899C9391E0970FD701A90F4E
:1019E000B11D8E5F94899C93F32DF80F8F2F821B6E
:1019F0002115310561F021503109D801A20FB31F23
:101A000055969C91D701A80FB11D9C93EFCF8F2FB6
:101A100090E002C080E090E00F900F900F900F9048
:101A20000F90DF91CF911F910F91FF90EF90DF907A
:101A3000CF90BF90AF909F908F907F906F905F906E
:101A40004F903F900895AF92BF92CF92DF92EF9266
:101A5000FF920F931F93CF93DF93633071050CF4C4
:101A6000B3C0EA016B017C01FC01908196FBAA24C2
:101A7000A0F88181282F269526952370B82EB29440
:101A8000B694B69453E0B522392F3770388393FB60
:101A9000332730F9398394FB332730F93A8395FBA8
:101AA000992790F99B83AC822D83829583708E83D6
:101AB000BF8282818887222379F13381848190E0FB
:101AC000982F8827830F911D9A87898787010B5F3D
:101AD0001F4F223071F46EE87AE0CE010B960E941F
:101AE0006277F70186818B8785818C870E5F1F4F18
:101AF0001EC02330E1F4F7013D96DE011B969E01E6
:101B00002D5E3F4F9E2F8F2F42914D93A217B3070B
:101B1000D9F7092F182F0BC087010D5F1F4F6EE8F3
:101B20007AE0CE010B960E9462771A861986BB2056
:101B3000A1F1A1100DC0F8012081818190E0982FC2
:101B40008827820F911D9C8B8B8B0E5F1F4F04C0CB
:101B500089859A859C8B8B8BF2E0BF120EC06EE854
:101B60007AE0CE0145960E946277F80181818D8BE3
:101B700080818E8B0E5F1F4F18C0F3E0BF1215C01F
:101B8000085F1F4FD801FE017596CE014D962E912C
:101B90002193E817F907D9F708C06EE87AE0CE017B
:101BA00045960E9462771C8A1B8A98012E193F096C
:101BB000C601821B930B98AB8FA71EA70DA7C21659
:101BC000D30614F0C90102C080E090E0DF91CF910C
:101BD0001F910F91FF90EF90DF90CF90BF90AF904B
:101BE000089520E030E00296FC01329740814423C2
:101BF00031F0FC0131974081240F311DF4CFC90130
:101C00000895FC01208130E0322F22278181282B8A
